Archive member included to satisfy reference by file (symbol)

c:/renesas/ra/e2studio_v2023-10_fsp_v5.0.0/toolchains/gcc_arm/12.2.mpacbti-rel1/bin/../lib/gcc/arm-none-eabi/12.2.1/thumb/v8-m.main+fp/hard\libgcc.a(_arm_muldf3.o)
                              ./src/adc_temp.o (__aeabi_dmul)
c:/renesas/ra/e2studio_v2023-10_fsp_v5.0.0/toolchains/gcc_arm/12.2.mpacbti-rel1/bin/../lib/gcc/arm-none-eabi/12.2.1/thumb/v8-m.main+fp/hard\libgcc.a(_arm_addsubdf3.o)
                              ./src/adc_temp.o (__aeabi_dsub)
c:/renesas/ra/e2studio_v2023-10_fsp_v5.0.0/toolchains/gcc_arm/12.2.mpacbti-rel1/bin/../lib/gcc/arm-none-eabi/12.2.1/thumb/v8-m.main+fp/hard\libgcc.a(_arm_muldivdf3.o)
                              ./src/adc_temp.o (__aeabi_ddiv)
c:/renesas/ra/e2studio_v2023-10_fsp_v5.0.0/toolchains/gcc_arm/12.2.mpacbti-rel1/bin/../lib/gcc/arm-none-eabi/12.2.1/thumb/v8-m.main+fp/hard\libgcc.a(_arm_cmpdf2.o)
                              ./src/usart.o (__aeabi_dcmpeq)
c:/renesas/ra/e2studio_v2023-10_fsp_v5.0.0/toolchains/gcc_arm/12.2.mpacbti-rel1/bin/../lib/gcc/arm-none-eabi/12.2.1/thumb/v8-m.main+fp/hard\libgcc.a(_arm_unorddf2.o)
                              ./src/usart.o (__aeabi_dcmpun)
c:/renesas/ra/e2studio_v2023-10_fsp_v5.0.0/toolchains/gcc_arm/12.2.mpacbti-rel1/bin/../lib/gcc/arm-none-eabi/12.2.1/thumb/v8-m.main+fp/hard\libgcc.a(_arm_fixdfsi.o)
                              ./src/adc_temp.o (__aeabi_d2iz)
c:/renesas/ra/e2studio_v2023-10_fsp_v5.0.0/toolchains/gcc_arm/12.2.mpacbti-rel1/bin/../lib/gcc/arm-none-eabi/12.2.1/thumb/v8-m.main+fp/hard\libgcc.a(_arm_fixunsdfsi.o)
                              ./src/hal_entry.o (__aeabi_d2uiz)
c:/renesas/ra/e2studio_v2023-10_fsp_v5.0.0/toolchains/gcc_arm/12.2.mpacbti-rel1/bin/../lib/gcc/arm-none-eabi/12.2.1/thumb/v8-m.main+fp/hard\libgcc.a(_aeabi_ldivmod.o)
                              ./src/hal_entry.o (__aeabi_ldivmod)
c:/renesas/ra/e2studio_v2023-10_fsp_v5.0.0/toolchains/gcc_arm/12.2.mpacbti-rel1/bin/../lib/gcc/arm-none-eabi/12.2.1/thumb/v8-m.main+fp/hard\libgcc.a(_udivmoddi4.o)
                              c:/renesas/ra/e2studio_v2023-10_fsp_v5.0.0/toolchains/gcc_arm/12.2.mpacbti-rel1/bin/../lib/gcc/arm-none-eabi/12.2.1/thumb/v8-m.main+fp/hard\libgcc.a(_aeabi_ldivmod.o) (__udivmoddi4)
c:/renesas/ra/e2studio_v2023-10_fsp_v5.0.0/toolchains/gcc_arm/12.2.mpacbti-rel1/bin/../lib/gcc/arm-none-eabi/12.2.1/thumb/v8-m.main+fp/hard\libgcc.a(_dvmd_tls.o)
                              c:/renesas/ra/e2studio_v2023-10_fsp_v5.0.0/toolchains/gcc_arm/12.2.mpacbti-rel1/bin/../lib/gcc/arm-none-eabi/12.2.1/thumb/v8-m.main+fp/hard\libgcc.a(_aeabi_ldivmod.o) (__aeabi_ldiv0)
c:/renesas/ra/e2studio_v2023-10_fsp_v5.0.0/toolchains/gcc_arm/12.2.mpacbti-rel1/bin/../lib/gcc/arm-none-eabi/12.2.1/thumb/v8-m.main+fp/hard\libg_nano.a(libc_a-exit.o)
                              c:/renesas/ra/e2studio_v2023-10_fsp_v5.0.0/toolchains/gcc_arm/12.2.mpacbti-rel1/bin/../lib/gcc/arm-none-eabi/12.2.1/thumb/v8-m.main+fp/hard/rdimon-crt0.o (exit)
c:/renesas/ra/e2studio_v2023-10_fsp_v5.0.0/toolchains/gcc_arm/12.2.mpacbti-rel1/bin/../lib/gcc/arm-none-eabi/12.2.1/thumb/v8-m.main+fp/hard\libg_nano.a(libc_a-itoa.o)
                              ./src/packet.o (__itoa)
c:/renesas/ra/e2studio_v2023-10_fsp_v5.0.0/toolchains/gcc_arm/12.2.mpacbti-rel1/bin/../lib/gcc/arm-none-eabi/12.2.1/thumb/v8-m.main+fp/hard\libg_nano.a(libc_a-strtol.o)
                              ./src/packet.o (strtol)
c:/renesas/ra/e2studio_v2023-10_fsp_v5.0.0/toolchains/gcc_arm/12.2.mpacbti-rel1/bin/../lib/gcc/arm-none-eabi/12.2.1/thumb/v8-m.main+fp/hard\libg_nano.a(libc_a-utoa.o)
                              ./src/packet.o (__utoa)
c:/renesas/ra/e2studio_v2023-10_fsp_v5.0.0/toolchains/gcc_arm/12.2.mpacbti-rel1/bin/../lib/gcc/arm-none-eabi/12.2.1/thumb/v8-m.main+fp/hard\libg_nano.a(libc_a-ctype_.o)
                              c:/renesas/ra/e2studio_v2023-10_fsp_v5.0.0/toolchains/gcc_arm/12.2.mpacbti-rel1/bin/../lib/gcc/arm-none-eabi/12.2.1/thumb/v8-m.main+fp/hard\libg_nano.a(libc_a-strtol.o) (_ctype_)
c:/renesas/ra/e2studio_v2023-10_fsp_v5.0.0/toolchains/gcc_arm/12.2.mpacbti-rel1/bin/../lib/gcc/arm-none-eabi/12.2.1/thumb/v8-m.main+fp/hard\libg_nano.a(libc_a-findfp.o)
                              c:/renesas/ra/e2studio_v2023-10_fsp_v5.0.0/toolchains/gcc_arm/12.2.mpacbti-rel1/bin/../lib/gcc/arm-none-eabi/12.2.1/thumb/v8-m.main+fp/hard\libg_nano.a(libc_a-exit.o) (__stdio_exit_handler)
c:/renesas/ra/e2studio_v2023-10_fsp_v5.0.0/toolchains/gcc_arm/12.2.mpacbti-rel1/bin/../lib/gcc/arm-none-eabi/12.2.1/thumb/v8-m.main+fp/hard\libg_nano.a(libc_a-fwalk.o)
                              c:/renesas/ra/e2studio_v2023-10_fsp_v5.0.0/toolchains/gcc_arm/12.2.mpacbti-rel1/bin/../lib/gcc/arm-none-eabi/12.2.1/thumb/v8-m.main+fp/hard\libg_nano.a(libc_a-findfp.o) (_fwalk_sglue)
c:/renesas/ra/e2studio_v2023-10_fsp_v5.0.0/toolchains/gcc_arm/12.2.mpacbti-rel1/bin/../lib/gcc/arm-none-eabi/12.2.1/thumb/v8-m.main+fp/hard\libg_nano.a(libc_a-stdio.o)
                              c:/renesas/ra/e2studio_v2023-10_fsp_v5.0.0/toolchains/gcc_arm/12.2.mpacbti-rel1/bin/../lib/gcc/arm-none-eabi/12.2.1/thumb/v8-m.main+fp/hard\libg_nano.a(libc_a-findfp.o) (__sread)
c:/renesas/ra/e2studio_v2023-10_fsp_v5.0.0/toolchains/gcc_arm/12.2.mpacbti-rel1/bin/../lib/gcc/arm-none-eabi/12.2.1/thumb/v8-m.main+fp/hard\libg_nano.a(libc_a-memset.o)
                              c:/renesas/ra/e2studio_v2023-10_fsp_v5.0.0/toolchains/gcc_arm/12.2.mpacbti-rel1/bin/../lib/gcc/arm-none-eabi/12.2.1/thumb/v8-m.main+fp/hard/rdimon-crt0.o (memset)
c:/renesas/ra/e2studio_v2023-10_fsp_v5.0.0/toolchains/gcc_arm/12.2.mpacbti-rel1/bin/../lib/gcc/arm-none-eabi/12.2.1/thumb/v8-m.main+fp/hard\libg_nano.a(libc_a-closer.o)
                              c:/renesas/ra/e2studio_v2023-10_fsp_v5.0.0/toolchains/gcc_arm/12.2.mpacbti-rel1/bin/../lib/gcc/arm-none-eabi/12.2.1/thumb/v8-m.main+fp/hard\libg_nano.a(libc_a-stdio.o) (_close_r)
c:/renesas/ra/e2studio_v2023-10_fsp_v5.0.0/toolchains/gcc_arm/12.2.mpacbti-rel1/bin/../lib/gcc/arm-none-eabi/12.2.1/thumb/v8-m.main+fp/hard\libg_nano.a(libc_a-reent.o)
                              c:/renesas/ra/e2studio_v2023-10_fsp_v5.0.0/toolchains/gcc_arm/12.2.mpacbti-rel1/bin/../lib/gcc/arm-none-eabi/12.2.1/thumb/v8-m.main+fp/hard\libg_nano.a(libc_a-closer.o) (errno)
c:/renesas/ra/e2studio_v2023-10_fsp_v5.0.0/toolchains/gcc_arm/12.2.mpacbti-rel1/bin/../lib/gcc/arm-none-eabi/12.2.1/thumb/v8-m.main+fp/hard\libg_nano.a(libc_a-impure.o)
                              c:/renesas/ra/e2studio_v2023-10_fsp_v5.0.0/toolchains/gcc_arm/12.2.mpacbti-rel1/bin/../lib/gcc/arm-none-eabi/12.2.1/thumb/v8-m.main+fp/hard\libg_nano.a(libc_a-strtol.o) (_impure_ptr)
c:/renesas/ra/e2studio_v2023-10_fsp_v5.0.0/toolchains/gcc_arm/12.2.mpacbti-rel1/bin/../lib/gcc/arm-none-eabi/12.2.1/thumb/v8-m.main+fp/hard\libg_nano.a(libc_a-lseekr.o)
                              c:/renesas/ra/e2studio_v2023-10_fsp_v5.0.0/toolchains/gcc_arm/12.2.mpacbti-rel1/bin/../lib/gcc/arm-none-eabi/12.2.1/thumb/v8-m.main+fp/hard\libg_nano.a(libc_a-stdio.o) (_lseek_r)
c:/renesas/ra/e2studio_v2023-10_fsp_v5.0.0/toolchains/gcc_arm/12.2.mpacbti-rel1/bin/../lib/gcc/arm-none-eabi/12.2.1/thumb/v8-m.main+fp/hard\libg_nano.a(libc_a-readr.o)
                              c:/renesas/ra/e2studio_v2023-10_fsp_v5.0.0/toolchains/gcc_arm/12.2.mpacbti-rel1/bin/../lib/gcc/arm-none-eabi/12.2.1/thumb/v8-m.main+fp/hard\libg_nano.a(libc_a-stdio.o) (_read_r)
c:/renesas/ra/e2studio_v2023-10_fsp_v5.0.0/toolchains/gcc_arm/12.2.mpacbti-rel1/bin/../lib/gcc/arm-none-eabi/12.2.1/thumb/v8-m.main+fp/hard\libg_nano.a(libc_a-writer.o)
                              c:/renesas/ra/e2studio_v2023-10_fsp_v5.0.0/toolchains/gcc_arm/12.2.mpacbti-rel1/bin/../lib/gcc/arm-none-eabi/12.2.1/thumb/v8-m.main+fp/hard\libg_nano.a(libc_a-stdio.o) (_write_r)
c:/renesas/ra/e2studio_v2023-10_fsp_v5.0.0/toolchains/gcc_arm/12.2.mpacbti-rel1/bin/../lib/gcc/arm-none-eabi/12.2.1/thumb/v8-m.main+fp/hard\libg_nano.a(libc_a-errno.o)
                              ./ra/fsp/src/bsp/mcu/all/bsp_sbrk.o (__errno)
c:/renesas/ra/e2studio_v2023-10_fsp_v5.0.0/toolchains/gcc_arm/12.2.mpacbti-rel1/bin/../lib/gcc/arm-none-eabi/12.2.1/thumb/v8-m.main+fp/hard\libg_nano.a(libc_a-init.o)
                              c:/renesas/ra/e2studio_v2023-10_fsp_v5.0.0/toolchains/gcc_arm/12.2.mpacbti-rel1/bin/../lib/gcc/arm-none-eabi/12.2.1/thumb/v8-m.main+fp/hard/rdimon-crt0.o (__libc_init_array)
c:/renesas/ra/e2studio_v2023-10_fsp_v5.0.0/toolchains/gcc_arm/12.2.mpacbti-rel1/bin/../lib/gcc/arm-none-eabi/12.2.1/thumb/v8-m.main+fp/hard\libg_nano.a(libc_a-lock.o)
                              c:/renesas/ra/e2studio_v2023-10_fsp_v5.0.0/toolchains/gcc_arm/12.2.mpacbti-rel1/bin/../lib/gcc/arm-none-eabi/12.2.1/thumb/v8-m.main+fp/hard\libg_nano.a(libc_a-findfp.o) (__retarget_lock_init_recursive)
c:/renesas/ra/e2studio_v2023-10_fsp_v5.0.0/toolchains/gcc_arm/12.2.mpacbti-rel1/bin/../lib/gcc/arm-none-eabi/12.2.1/thumb/v8-m.main+fp/hard\libg_nano.a(libc_a-strcpy.o)
                              ./src/packet.o (strcpy)
c:/renesas/ra/e2studio_v2023-10_fsp_v5.0.0/toolchains/gcc_arm/12.2.mpacbti-rel1/bin/../lib/gcc/arm-none-eabi/12.2.1/thumb/v8-m.main+fp/hard\libg_nano.a(libc_a-aeabi_memcpy.o)
                              ./src/usart.o (__aeabi_memcpy4)
c:/renesas/ra/e2studio_v2023-10_fsp_v5.0.0/toolchains/gcc_arm/12.2.mpacbti-rel1/bin/../lib/gcc/arm-none-eabi/12.2.1/thumb/v8-m.main+fp/hard\libg_nano.a(libc_a-aeabi_memclr.o)
                              ./src/packet.o (__aeabi_memclr8)
c:/renesas/ra/e2studio_v2023-10_fsp_v5.0.0/toolchains/gcc_arm/12.2.mpacbti-rel1/bin/../lib/gcc/arm-none-eabi/12.2.1/thumb/v8-m.main+fp/hard\libg_nano.a(libc_a-memcpy-stub.o)
                              ./src/control_table.o (memcpy)
c:/renesas/ra/e2studio_v2023-10_fsp_v5.0.0/toolchains/gcc_arm/12.2.mpacbti-rel1/bin/../lib/gcc/arm-none-eabi/12.2.1/thumb/v8-m.main+fp/hard\libg_nano.a(libc_a-strlen.o)
                              ./src/packet.o (strlen)
c:/renesas/ra/e2studio_v2023-10_fsp_v5.0.0/toolchains/gcc_arm/12.2.mpacbti-rel1/bin/../lib/gcc/arm-none-eabi/12.2.1/thumb/v8-m.main+fp/hard\libg_nano.a(libc_a-freer.o)
                              c:/renesas/ra/e2studio_v2023-10_fsp_v5.0.0/toolchains/gcc_arm/12.2.mpacbti-rel1/bin/../lib/gcc/arm-none-eabi/12.2.1/thumb/v8-m.main+fp/hard\libg_nano.a(libc_a-reent.o) (_free_r)
c:/renesas/ra/e2studio_v2023-10_fsp_v5.0.0/toolchains/gcc_arm/12.2.mpacbti-rel1/bin/../lib/gcc/arm-none-eabi/12.2.1/thumb/v8-m.main+fp/hard\libg_nano.a(libc_a-mallocr.o)
                              c:/renesas/ra/e2studio_v2023-10_fsp_v5.0.0/toolchains/gcc_arm/12.2.mpacbti-rel1/bin/../lib/gcc/arm-none-eabi/12.2.1/thumb/v8-m.main+fp/hard\libg_nano.a(libc_a-findfp.o) (_malloc_r)
c:/renesas/ra/e2studio_v2023-10_fsp_v5.0.0/toolchains/gcc_arm/12.2.mpacbti-rel1/bin/../lib/gcc/arm-none-eabi/12.2.1/thumb/v8-m.main+fp/hard\libg_nano.a(libc_a-mlock.o)
                              c:/renesas/ra/e2studio_v2023-10_fsp_v5.0.0/toolchains/gcc_arm/12.2.mpacbti-rel1/bin/../lib/gcc/arm-none-eabi/12.2.1/thumb/v8-m.main+fp/hard\libg_nano.a(libc_a-freer.o) (__malloc_lock)
c:/renesas/ra/e2studio_v2023-10_fsp_v5.0.0/toolchains/gcc_arm/12.2.mpacbti-rel1/bin/../lib/gcc/arm-none-eabi/12.2.1/thumb/v8-m.main+fp/hard\libg_nano.a(libc_a-fflush.o)
                              c:/renesas/ra/e2studio_v2023-10_fsp_v5.0.0/toolchains/gcc_arm/12.2.mpacbti-rel1/bin/../lib/gcc/arm-none-eabi/12.2.1/thumb/v8-m.main+fp/hard\libg_nano.a(libc_a-findfp.o) (_fflush_r)
c:/renesas/ra/e2studio_v2023-10_fsp_v5.0.0/toolchains/gcc_arm/12.2.mpacbti-rel1/bin/../lib/gcc/arm-none-eabi/12.2.1/thumb/v8-m.main+fp/hard\libg_nano.a(libc_a-sbrkr.o)
                              c:/renesas/ra/e2studio_v2023-10_fsp_v5.0.0/toolchains/gcc_arm/12.2.mpacbti-rel1/bin/../lib/gcc/arm-none-eabi/12.2.1/thumb/v8-m.main+fp/hard\libg_nano.a(libc_a-mallocr.o) (_sbrk_r)
c:/renesas/ra/e2studio_v2023-10_fsp_v5.0.0/toolchains/gcc_arm/12.2.mpacbti-rel1/bin/../lib/gcc/arm-none-eabi/12.2.1/thumb/v8-m.main+fp/hard\libg_nano.a(libc_a-aeabi_memset-soft.o)
                              c:/renesas/ra/e2studio_v2023-10_fsp_v5.0.0/toolchains/gcc_arm/12.2.mpacbti-rel1/bin/../lib/gcc/arm-none-eabi/12.2.1/thumb/v8-m.main+fp/hard\libg_nano.a(libc_a-aeabi_memclr.o) (__aeabi_memset)
c:/renesas/ra/e2studio_v2023-10_fsp_v5.0.0/toolchains/gcc_arm/12.2.mpacbti-rel1/bin/../lib/gcc/arm-none-eabi/12.2.1/thumb/v8-m.main+fp/hard\librdimon_nano.a(arm_librdimon_a-_exit.o)
                              c:/renesas/ra/e2studio_v2023-10_fsp_v5.0.0/toolchains/gcc_arm/12.2.mpacbti-rel1/bin/../lib/gcc/arm-none-eabi/12.2.1/thumb/v8-m.main+fp/hard\libg_nano.a(libc_a-exit.o) (_exit)
c:/renesas/ra/e2studio_v2023-10_fsp_v5.0.0/toolchains/gcc_arm/12.2.mpacbti-rel1/bin/../lib/gcc/arm-none-eabi/12.2.1/thumb/v8-m.main+fp/hard\librdimon_nano.a(arm_librdimon_a-_kill.o)
                              c:/renesas/ra/e2studio_v2023-10_fsp_v5.0.0/toolchains/gcc_arm/12.2.mpacbti-rel1/bin/../lib/gcc/arm-none-eabi/12.2.1/thumb/v8-m.main+fp/hard\librdimon_nano.a(arm_librdimon_a-_exit.o) (_kill_shared)
c:/renesas/ra/e2studio_v2023-10_fsp_v5.0.0/toolchains/gcc_arm/12.2.mpacbti-rel1/bin/../lib/gcc/arm-none-eabi/12.2.1/thumb/v8-m.main+fp/hard\librdimon_nano.a(arm_librdimon_a-syscalls.o)
                              c:/renesas/ra/e2studio_v2023-10_fsp_v5.0.0/toolchains/gcc_arm/12.2.mpacbti-rel1/bin/../lib/gcc/arm-none-eabi/12.2.1/thumb/v8-m.main+fp/hard\libg_nano.a(libc_a-readr.o) (_read)

Discarded input sections

 .text          0x00000000        0x0 c:/renesas/ra/e2studio_v2023-10_fsp_v5.0.0/toolchains/gcc_arm/12.2.mpacbti-rel1/bin/../lib/gcc/arm-none-eabi/12.2.1/thumb/v8-m.main+fp/hard/crti.o
 .data          0x00000000        0x0 c:/renesas/ra/e2studio_v2023-10_fsp_v5.0.0/toolchains/gcc_arm/12.2.mpacbti-rel1/bin/../lib/gcc/arm-none-eabi/12.2.1/thumb/v8-m.main+fp/hard/crti.o
 .bss           0x00000000        0x0 c:/renesas/ra/e2studio_v2023-10_fsp_v5.0.0/toolchains/gcc_arm/12.2.mpacbti-rel1/bin/../lib/gcc/arm-none-eabi/12.2.1/thumb/v8-m.main+fp/hard/crti.o
 .text          0x00000000        0x0 c:/renesas/ra/e2studio_v2023-10_fsp_v5.0.0/toolchains/gcc_arm/12.2.mpacbti-rel1/bin/../lib/gcc/arm-none-eabi/12.2.1/thumb/v8-m.main+fp/hard/crtbegin.o
 .data          0x00000000        0x0 c:/renesas/ra/e2studio_v2023-10_fsp_v5.0.0/toolchains/gcc_arm/12.2.mpacbti-rel1/bin/../lib/gcc/arm-none-eabi/12.2.1/thumb/v8-m.main+fp/hard/crtbegin.o
 .bss           0x00000000        0x0 c:/renesas/ra/e2studio_v2023-10_fsp_v5.0.0/toolchains/gcc_arm/12.2.mpacbti-rel1/bin/../lib/gcc/arm-none-eabi/12.2.1/thumb/v8-m.main+fp/hard/crtbegin.o
 .rodata.all_implied_fbits
                0x00000000       0x24 c:/renesas/ra/e2studio_v2023-10_fsp_v5.0.0/toolchains/gcc_arm/12.2.mpacbti-rel1/bin/../lib/gcc/arm-none-eabi/12.2.1/thumb/v8-m.main+fp/hard/crtbegin.o
 .data.__dso_handle
                0x00000000        0x4 c:/renesas/ra/e2studio_v2023-10_fsp_v5.0.0/toolchains/gcc_arm/12.2.mpacbti-rel1/bin/../lib/gcc/arm-none-eabi/12.2.1/thumb/v8-m.main+fp/hard/crtbegin.o
 .text          0x00000000       0xf8 c:/renesas/ra/e2studio_v2023-10_fsp_v5.0.0/toolchains/gcc_arm/12.2.mpacbti-rel1/bin/../lib/gcc/arm-none-eabi/12.2.1/thumb/v8-m.main+fp/hard/rdimon-crt0.o
 .data          0x00000000      0x118 c:/renesas/ra/e2studio_v2023-10_fsp_v5.0.0/toolchains/gcc_arm/12.2.mpacbti-rel1/bin/../lib/gcc/arm-none-eabi/12.2.1/thumb/v8-m.main+fp/hard/rdimon-crt0.o
 .bss           0x00000000        0x0 c:/renesas/ra/e2studio_v2023-10_fsp_v5.0.0/toolchains/gcc_arm/12.2.mpacbti-rel1/bin/../lib/gcc/arm-none-eabi/12.2.1/thumb/v8-m.main+fp/hard/rdimon-crt0.o
 .ARM.extab     0x00000000        0x0 c:/renesas/ra/e2studio_v2023-10_fsp_v5.0.0/toolchains/gcc_arm/12.2.mpacbti-rel1/bin/../lib/gcc/arm-none-eabi/12.2.1/thumb/v8-m.main+fp/hard/rdimon-crt0.o
 .ARM.exidx     0x00000000       0x10 c:/renesas/ra/e2studio_v2023-10_fsp_v5.0.0/toolchains/gcc_arm/12.2.mpacbti-rel1/bin/../lib/gcc/arm-none-eabi/12.2.1/thumb/v8-m.main+fp/hard/rdimon-crt0.o
 .debug_line_str
                0x00000000       0xea c:/renesas/ra/e2studio_v2023-10_fsp_v5.0.0/toolchains/gcc_arm/12.2.mpacbti-rel1/bin/../lib/gcc/arm-none-eabi/12.2.1/thumb/v8-m.main+fp/hard/rdimon-crt0.o
 .ARM.attributes
                0x00000000       0x24 c:/renesas/ra/e2studio_v2023-10_fsp_v5.0.0/toolchains/gcc_arm/12.2.mpacbti-rel1/bin/../lib/gcc/arm-none-eabi/12.2.1/thumb/v8-m.main+fp/hard/rdimon-crt0.o
 .text          0x00000000        0x0 ./src/adc_temp.o
 .data          0x00000000        0x0 ./src/adc_temp.o
 .bss           0x00000000        0x0 ./src/adc_temp.o
 .text          0x00000000        0x0 ./src/angle.o
 .data          0x00000000        0x0 ./src/angle.o
 .bss           0x00000000        0x0 ./src/angle.o
 .text.tad2141_power
                0x00000000       0x98 ./src/angle.o
 .text.tad2141_EOL_Programming
                0x00000000      0x288 ./src/angle.o
 .text          0x00000000        0x0 ./src/control_table.o
 .data          0x00000000        0x0 ./src/control_table.o
 .bss           0x00000000        0x0 ./src/control_table.o
 .text.get_iteminfosize
                0x00000000        0x4 ./src/control_table.o
 .text          0x00000000        0x0 ./src/crc8.o
 .data          0x00000000        0x0 ./src/crc8.o
 .bss           0x00000000        0x0 ./src/crc8.o
 .text          0x00000000        0x0 ./src/global_variables.o
 .data          0x00000000        0x0 ./src/global_variables.o
 .bss           0x00000000        0x0 ./src/global_variables.o
 .text          0x00000000        0x0 ./src/hal_entry.o
 .data          0x00000000        0x0 ./src/hal_entry.o
 .bss           0x00000000        0x0 ./src/hal_entry.o
 .text.led_toggle
                0x00000000       0x1c ./src/hal_entry.o
 .text          0x00000000        0x0 ./src/interpolation.o
 .data          0x00000000        0x0 ./src/interpolation.o
 .bss           0x00000000        0x0 ./src/interpolation.o
 .text          0x00000000        0x0 ./src/monitor.o
 .data          0x00000000        0x0 ./src/monitor.o
 .bss           0x00000000        0x0 ./src/monitor.o
 .text          0x00000000        0x0 ./src/packet.o
 .data          0x00000000        0x0 ./src/packet.o
 .bss           0x00000000        0x0 ./src/packet.o
 .text          0x00000000        0x0 ./src/pid.o
 .data          0x00000000        0x0 ./src/pid.o
 .bss           0x00000000        0x0 ./src/pid.o
 .text.PIDReset_int
                0x00000000        0xc ./src/pid.o
 .text.PIDUpdate_int
                0x00000000       0x5c ./src/pid.o
 .text          0x00000000        0x0 ./src/power_monitor.o
 .data          0x00000000        0x0 ./src/power_monitor.o
 .bss           0x00000000        0x0 ./src/power_monitor.o
 .text          0x00000000        0x0 ./src/sintable.o
 .data          0x00000000        0x0 ./src/sintable.o
 .bss           0x00000000        0x0 ./src/sintable.o
 .text.my_sin1000
                0x00000000       0xa0 ./src/sintable.o
 .text          0x00000000        0x0 ./src/usart.o
 .data          0x00000000        0x0 ./src/usart.o
 .bss           0x00000000        0x0 ./src/usart.o
 .text.us_putc  0x00000000       0x30 ./src/usart.o
 .text.us_puts  0x00000000       0x78 ./src/usart.o
 .text.us_putsbd
                0x00000000       0x28 ./src/usart.o
 .text.us_rx_purge
                0x00000000       0x3c ./src/usart.o
 .rodata.us_printf.str1.4
                0x00000000       0x10 ./src/usart.o
 .text.us_printf
                0x00000000      0xc50 ./src/usart.o
 .text.us_deinit
                0x00000000       0x20 ./src/usart.o
 .bss.buf.0     0x00000000      0x400 ./src/usart.o
 .text          0x00000000        0x0 ./ra_gen/common_data.o
 .data          0x00000000        0x0 ./ra_gen/common_data.o
 .bss           0x00000000        0x0 ./ra_gen/common_data.o
 .text.g_common_init
                0x00000000        0x4 ./ra_gen/common_data.o
 .text          0x00000000        0x0 ./ra_gen/hal_data.o
 .data          0x00000000        0x0 ./ra_gen/hal_data.o
 .bss           0x00000000        0x0 ./ra_gen/hal_data.o
 .text.g_hal_init
                0x00000000        0x4 ./ra_gen/hal_data.o
 .rodata.g_uart4
                0x00000000        0xc ./ra_gen/hal_data.o
 .rodata.g_i2c3
                0x00000000        0xc ./ra_gen/hal_data.o
 .rodata.g_spi2
                0x00000000        0xc ./ra_gen/hal_data.o
 .rodata.g_timer5
                0x00000000        0xc ./ra_gen/hal_data.o
 .rodata.g_timer0
                0x00000000        0xc ./ra_gen/hal_data.o
 .rodata.g_adc0
                0x00000000       0x10 ./ra_gen/hal_data.o
 .rodata.g_flash0
                0x00000000        0xc ./ra_gen/hal_data.o
 .rodata.g_crc0
                0x00000000        0xc ./ra_gen/hal_data.o
 .rodata.g_rtc0
                0x00000000        0xc ./ra_gen/hal_data.o
 .rodata.g_rtc0_cfg
                0x00000000       0x20 ./ra_gen/hal_data.o
 .rodata.g_rtc0_err_cfg
                0x00000000        0x8 ./ra_gen/hal_data.o
 .bss.g_rtc0_ctrl
                0x00000000       0x18 ./ra_gen/hal_data.o
 .text          0x00000000        0x0 ./ra_gen/main.o
 .data          0x00000000        0x0 ./ra_gen/main.o
 .bss           0x00000000        0x0 ./ra_gen/main.o
 .text          0x00000000        0x0 ./ra_gen/pin_data.o
 .data          0x00000000        0x0 ./ra_gen/pin_data.o
 .bss           0x00000000        0x0 ./ra_gen/pin_data.o
 .text          0x00000000        0x0 ./ra_gen/vector_data.o
 .data          0x00000000        0x0 ./ra_gen/vector_data.o
 .bss           0x00000000        0x0 ./ra_gen/vector_data.o
 .text          0x00000000        0x0 ./ra/fsp/src/r_sci_uart/r_sci_uart.o
 .data          0x00000000        0x0 ./ra/fsp/src/r_sci_uart/r_sci_uart.o
 .bss           0x00000000        0x0 ./ra/fsp/src/r_sci_uart/r_sci_uart.o
 .text.R_SCI_UART_Read
                0x00000000       0x34 ./ra/fsp/src/r_sci_uart/r_sci_uart.o
 .text.R_SCI_UART_CallbackSet
                0x00000000       0x10 ./ra/fsp/src/r_sci_uart/r_sci_uart.o
 .text.R_SCI_UART_InfoGet
                0x00000000       0x28 ./ra/fsp/src/r_sci_uart/r_sci_uart.o
 .text.R_SCI_UART_ReadStop
                0x00000000       0x3c ./ra/fsp/src/r_sci_uart/r_sci_uart.o
 .text.R_SCI_UART_Close
                0x00000000       0xd4 ./ra/fsp/src/r_sci_uart/r_sci_uart.o
 .rodata.g_uart_on_sci
                0x00000000       0x24 ./ra/fsp/src/r_sci_uart/r_sci_uart.o
 .text          0x00000000        0x0 ./ra/fsp/src/r_sci_spi/r_sci_spi.o
 .data          0x00000000        0x0 ./ra/fsp/src/r_sci_spi/r_sci_spi.o
 .bss           0x00000000        0x0 ./ra/fsp/src/r_sci_spi/r_sci_spi.o
 .text.R_SCI_SPI_CallbackSet
                0x00000000       0x10 ./ra/fsp/src/r_sci_spi/r_sci_spi.o
 .text.R_SCI_SPI_Close
                0x00000000       0xd4 ./ra/fsp/src/r_sci_spi/r_sci_spi.o
 .text.R_SCI_SPI_Write
                0x00000000      0x10c ./ra/fsp/src/r_sci_spi/r_sci_spi.o
 .text.R_SCI_SPI_Read
                0x00000000      0x114 ./ra/fsp/src/r_sci_spi/r_sci_spi.o
 .text.R_SCI_SPI_CalculateBitrate
                0x00000000       0xbc ./ra/fsp/src/r_sci_spi/r_sci_spi.o
 .rodata.g_spi_on_sci
                0x00000000       0x18 ./ra/fsp/src/r_sci_spi/r_sci_spi.o
 .text          0x00000000        0x0 ./ra/fsp/src/r_sci_i2c/r_sci_i2c.o
 .data          0x00000000        0x0 ./ra/fsp/src/r_sci_i2c/r_sci_i2c.o
 .bss           0x00000000        0x0 ./ra/fsp/src/r_sci_i2c/r_sci_i2c.o
 .text.R_SCI_I2C_Abort
                0x00000000       0x2c ./ra/fsp/src/r_sci_i2c/r_sci_i2c.o
 .text.R_SCI_I2C_CallbackSet
                0x00000000       0x10 ./ra/fsp/src/r_sci_i2c/r_sci_i2c.o
 .text.R_SCI_I2C_StatusGet
                0x00000000       0x18 ./ra/fsp/src/r_sci_i2c/r_sci_i2c.o
 .text.R_SCI_I2C_Close
                0x00000000       0x58 ./ra/fsp/src/r_sci_i2c/r_sci_i2c.o
 .text.sci_i2c_notify
                0x00000000       0x38 ./ra/fsp/src/r_sci_i2c/r_sci_i2c.o
 .rodata.g_i2c_master_on_sci
                0x00000000       0x20 ./ra/fsp/src/r_sci_i2c/r_sci_i2c.o
 .text          0x00000000        0x0 ./ra/fsp/src/r_rtc/r_rtc.o
 .data          0x00000000        0x0 ./ra/fsp/src/r_rtc/r_rtc.o
 .bss           0x00000000        0x0 ./ra/fsp/src/r_rtc/r_rtc.o
 .text.R_RTC_Close
                0x00000000       0xe8 ./ra/fsp/src/r_rtc/r_rtc.o
 .text.R_RTC_CalendarAlarmSet
                0x00000000      0x210 ./ra/fsp/src/r_rtc/r_rtc.o
 .text.R_RTC_CalendarAlarmGet
                0x00000000       0xd0 ./ra/fsp/src/r_rtc/r_rtc.o
 .text.R_RTC_PeriodicIrqRateSet
                0x00000000       0x7c ./ra/fsp/src/r_rtc/r_rtc.o
 .text.R_RTC_InfoGet
                0x00000000       0x1c ./ra/fsp/src/r_rtc/r_rtc.o
 .text.R_RTC_CallbackSet
                0x00000000       0x10 ./ra/fsp/src/r_rtc/r_rtc.o
 .text.R_RTC_ClockSourceSet
                0x00000000       0x90 ./ra/fsp/src/r_rtc/r_rtc.o
 .text.R_RTC_CalendarTimeGet
                0x00000000      0x188 ./ra/fsp/src/r_rtc/r_rtc.o
 .text.R_RTC_Open
                0x00000000       0x88 ./ra/fsp/src/r_rtc/r_rtc.o
 .text.R_RTC_CalendarTimeSet
                0x00000000      0x1b8 ./ra/fsp/src/r_rtc/r_rtc.o
 .text.R_RTC_ErrorAdjustmentSet
                0x00000000       0x94 ./ra/fsp/src/r_rtc/r_rtc.o
 .text.rtc_alarm_periodic_isr
                0x00000000       0x70 ./ra/fsp/src/r_rtc/r_rtc.o
 .rodata.g_rtc_on_rtc
                0x00000000       0x2c ./ra/fsp/src/r_rtc/r_rtc.o
 .text          0x00000000        0x0 ./ra/fsp/src/r_ioport/r_ioport.o
 .data          0x00000000        0x0 ./ra/fsp/src/r_ioport/r_ioport.o
 .bss           0x00000000        0x0 ./ra/fsp/src/r_ioport/r_ioport.o
 .text          0x00000000        0x0 ./ra/fsp/src/r_gpt/r_gpt.o
 .data          0x00000000        0x0 ./ra/fsp/src/r_gpt/r_gpt.o
 .bss           0x00000000        0x0 ./ra/fsp/src/r_gpt/r_gpt.o
 .text.R_GPT_Stop
                0x00000000        0xc ./ra/fsp/src/r_gpt/r_gpt.o
 .text.R_GPT_Reset
                0x00000000        0xc ./ra/fsp/src/r_gpt/r_gpt.o
 .text.R_GPT_Enable
                0x00000000       0x30 ./ra/fsp/src/r_gpt/r_gpt.o
 .text.R_GPT_Disable
                0x00000000       0x18 ./ra/fsp/src/r_gpt/r_gpt.o
 .text.R_GPT_PeriodSet
                0x00000000       0x30 ./ra/fsp/src/r_gpt/r_gpt.o
 .text.R_GPT_InfoGet
                0x00000000       0x44 ./ra/fsp/src/r_gpt/r_gpt.o
 .text.R_GPT_StatusGet
                0x00000000       0x14 ./ra/fsp/src/r_gpt/r_gpt.o
 .text.R_GPT_CallbackSet
                0x00000000       0x10 ./ra/fsp/src/r_gpt/r_gpt.o
 .text.R_GPT_Close
                0x00000000       0xa0 ./ra/fsp/src/r_gpt/r_gpt.o
 .text.R_GPT_CounterSet
                0x00000000        0xc ./ra/fsp/src/r_gpt/r_gpt.o
 .text.R_GPT_OutputEnable
                0x00000000       0x18 ./ra/fsp/src/r_gpt/r_gpt.o
 .text.R_GPT_OutputDisable
                0x00000000       0x18 ./ra/fsp/src/r_gpt/r_gpt.o
 .text.R_GPT_AdcTriggerSet
                0x00000000       0x10 ./ra/fsp/src/r_gpt/r_gpt.o
 .text.R_GPT_PwmOutputDelaySet
                0x00000000        0x4 ./ra/fsp/src/r_gpt/r_gpt.o
 .text.R_GPT_PwmOutputDelayInitialize
                0x00000000        0x4 ./ra/fsp/src/r_gpt/r_gpt.o
 .text.gpt_counter_overflow_isr
                0x00000000       0xb8 ./ra/fsp/src/r_gpt/r_gpt.o
 .text.gpt_capture_a_isr
                0x00000000       0xc8 ./ra/fsp/src/r_gpt/r_gpt.o
 .text.gpt_capture_b_isr
                0x00000000       0xc8 ./ra/fsp/src/r_gpt/r_gpt.o
 .rodata.g_timer_on_gpt
                0x00000000       0x30 ./ra/fsp/src/r_gpt/r_gpt.o
 .text          0x00000000        0x0 ./ra/fsp/src/r_flash_hp/r_flash_hp.o
 .data          0x00000000        0x0 ./ra/fsp/src/r_flash_hp/r_flash_hp.o
 .bss           0x00000000        0x0 ./ra/fsp/src/r_flash_hp/r_flash_hp.o
 .text.R_FLASH_HP_StatusGet
                0x00000000       0x1c ./ra/fsp/src/r_flash_hp/r_flash_hp.o
 .text.R_FLASH_HP_IdCodeSet
                0x00000000        0x4 ./ra/fsp/src/r_flash_hp/r_flash_hp.o
 .text.R_FLASH_HP_AccessWindowSet
                0x00000000        0x4 ./ra/fsp/src/r_flash_hp/r_flash_hp.o
 .text.R_FLASH_HP_AccessWindowClear
                0x00000000        0x4 ./ra/fsp/src/r_flash_hp/r_flash_hp.o
 .text.R_FLASH_HP_StartUpAreaSelect
                0x00000000        0x4 ./ra/fsp/src/r_flash_hp/r_flash_hp.o
 .text.R_FLASH_HP_InfoGet
                0x00000000       0x2c ./ra/fsp/src/r_flash_hp/r_flash_hp.o
 .text.R_FLASH_HP_CallbackSet
                0x00000000       0x10 ./ra/fsp/src/r_flash_hp/r_flash_hp.o
 .text.R_FLASH_HP_BankSwap
                0x00000000        0x4 ./ra/fsp/src/r_flash_hp/r_flash_hp.o
 .text.R_FLASH_HP_BlankCheck
                0x00000000      0x1b0 ./ra/fsp/src/r_flash_hp/r_flash_hp.o
 .text.flash_hp_reset
                0x00000000      0x180 ./ra/fsp/src/r_flash_hp/r_flash_hp.o
 .text.R_FLASH_HP_Reset
                0x00000000        0x4 ./ra/fsp/src/r_flash_hp/r_flash_hp.o
 .text.R_FLASH_HP_UpdateFlashClockFreq
                0x00000000      0x108 ./ra/fsp/src/r_flash_hp/r_flash_hp.o
 .text.fcu_fiferr_isr
                0x00000000       0x94 ./ra/fsp/src/r_flash_hp/r_flash_hp.o
 .text.fcu_frdyi_isr
                0x00000000      0x1ac ./ra/fsp/src/r_flash_hp/r_flash_hp.o
 .rodata.g_flash_on_flash_hp
                0x00000000       0x3c ./ra/fsp/src/r_flash_hp/r_flash_hp.o
 .rodata.g_flash_data_region
                0x00000000        0x8 ./ra/fsp/src/r_flash_hp/r_flash_hp.o
 .rodata.g_data_flash_macro_info
                0x00000000       0x10 ./ra/fsp/src/r_flash_hp/r_flash_hp.o
 .rodata.g_flash_code_region
                0x00000000        0x8 ./ra/fsp/src/r_flash_hp/r_flash_hp.o
 .rodata.g_code_flash_macro_info
                0x00000000       0x20 ./ra/fsp/src/r_flash_hp/r_flash_hp.o
 .text          0x00000000        0x0 ./ra/fsp/src/r_dtc/r_dtc.o
 .data          0x00000000        0x0 ./ra/fsp/src/r_dtc/r_dtc.o
 .bss           0x00000000        0x0 ./ra/fsp/src/r_dtc/r_dtc.o
 .text          0x00000000        0x0 ./ra/fsp/src/r_crc/r_crc.o
 .data          0x00000000        0x0 ./ra/fsp/src/r_crc/r_crc.o
 .bss           0x00000000        0x0 ./ra/fsp/src/r_crc/r_crc.o
 .text.R_CRC_CalculatedValueGet
                0x00000000       0x34 ./ra/fsp/src/r_crc/r_crc.o
 .text.R_CRC_SnoopEnable
                0x00000000        0x4 ./ra/fsp/src/r_crc/r_crc.o
 .text.R_CRC_SnoopDisable
                0x00000000        0x4 ./ra/fsp/src/r_crc/r_crc.o
 .rodata.g_crc_on_crc
                0x00000000       0x18 ./ra/fsp/src/r_crc/r_crc.o
 .text          0x00000000        0x0 ./ra/fsp/src/r_agt/r_agt.o
 .data          0x00000000        0x0 ./ra/fsp/src/r_agt/r_agt.o
 .bss           0x00000000        0x0 ./ra/fsp/src/r_agt/r_agt.o
 .text.R_AGT_Start
                0x00000000       0x60 ./ra/fsp/src/r_agt/r_agt.o
 .text.R_AGT_Stop
                0x00000000       0x24 ./ra/fsp/src/r_agt/r_agt.o
 .text.R_AGT_Disable
                0x00000000       0x1c ./ra/fsp/src/r_agt/r_agt.o
 .text.R_AGT_PeriodSet
                0x00000000       0x4c ./ra/fsp/src/r_agt/r_agt.o
 .text.R_AGT_DutyCycleSet
                0x00000000        0x4 ./ra/fsp/src/r_agt/r_agt.o
 .text.R_AGT_InfoGet
                0x00000000       0xe8 ./ra/fsp/src/r_agt/r_agt.o
 .text.R_AGT_StatusGet
                0x00000000       0x44 ./ra/fsp/src/r_agt/r_agt.o
 .text.R_AGT_CallbackSet
                0x00000000       0x10 ./ra/fsp/src/r_agt/r_agt.o
 .text.R_AGT_Close
                0x00000000       0x74 ./ra/fsp/src/r_agt/r_agt.o
 .text.R_AGT_Reset
                0x00000000       0x3c ./ra/fsp/src/r_agt/r_agt.o
 .rodata.g_timer_on_agt
                0x00000000       0x30 ./ra/fsp/src/r_agt/r_agt.o
 .text          0x00000000        0x0 ./ra/fsp/src/r_adc/r_adc.o
 .data          0x00000000        0x0 ./ra/fsp/src/r_adc/r_adc.o
 .bss           0x00000000        0x0 ./ra/fsp/src/r_adc/r_adc.o
 .text.R_ADC_CallbackSet
                0x00000000       0x10 ./ra/fsp/src/r_adc/r_adc.o
 .text.R_ADC_ScanGroupStart
                0x00000000        0x4 ./ra/fsp/src/r_adc/r_adc.o
 .text.R_ADC_ScanStop
                0x00000000        0xc ./ra/fsp/src/r_adc/r_adc.o
 .text.R_ADC_StatusGet
                0x00000000       0x10 ./ra/fsp/src/r_adc/r_adc.o
 .text.R_ADC_Read32
                0x00000000       0x1c ./ra/fsp/src/r_adc/r_adc.o
 .text.R_ADC_Calibrate
                0x00000000        0x4 ./ra/fsp/src/r_adc/r_adc.o
 .text.R_ADC_OffsetSet
                0x00000000        0x4 ./ra/fsp/src/r_adc/r_adc.o
 .text.r_adc_call_callback
                0x00000000       0x54 ./ra/fsp/src/r_adc/r_adc.o
 .text.R_ADC_InfoGet
                0x00000000       0x6c ./ra/fsp/src/r_adc/r_adc.o
 .text.R_ADC_Close
                0x00000000       0xf4 ./ra/fsp/src/r_adc/r_adc.o
 .text.R_ADC_SampleStateCountSet
                0x00000000       0x14 ./ra/fsp/src/r_adc/r_adc.o
 .text.adc_scan_end_isr
                0x00000000       0x5c ./ra/fsp/src/r_adc/r_adc.o
 .text.adc_scan_end_b_isr
                0x00000000       0x64 ./ra/fsp/src/r_adc/r_adc.o
 .text.adc_window_compare_isr
                0x00000000      0x118 ./ra/fsp/src/r_adc/r_adc.o
 .rodata.g_adc_on_adc
                0x00000000       0x34 ./ra/fsp/src/r_adc/r_adc.o
 .text          0x00000000        0x0 ./ra/fsp/src/bsp/mcu/all/bsp_clocks.o
 .data          0x00000000        0x0 ./ra/fsp/src/bsp/mcu/all/bsp_clocks.o
 .bss           0x00000000        0x0 ./ra/fsp/src/bsp/mcu/all/bsp_clocks.o
 .text.bsp_prv_operating_mode_set
                0x00000000       0x60 ./ra/fsp/src/bsp/mcu/all/bsp_clocks.o
 .text.bsp_prv_prepare_pll
                0x00000000        0xc ./ra/fsp/src/bsp/mcu/all/bsp_clocks.o
 .text.prv_clock_dividers_set
                0x00000000        0xc ./ra/fsp/src/bsp/mcu/all/bsp_clocks.o
 .text.bsp_prv_clock_set
                0x00000000       0xb0 ./ra/fsp/src/bsp/mcu/all/bsp_clocks.o
 .text.R_BSP_SubClockStabilizeWait
                0x00000000        0x8 ./ra/fsp/src/bsp/mcu/all/bsp_clocks.o
 .text.R_BSP_OctaclkUpdate
                0x00000000        0x4 ./ra/fsp/src/bsp/mcu/all/bsp_clocks.o
 .text.R_BSP_SourceClockHzGet
                0x00000000        0xc ./ra/fsp/src/bsp/mcu/all/bsp_clocks.o
 .text          0x00000000        0x0 ./ra/fsp/src/bsp/mcu/all/bsp_common.o
 .data          0x00000000        0x0 ./ra/fsp/src/bsp/mcu/all/bsp_common.o
 .bss           0x00000000        0x0 ./ra/fsp/src/bsp/mcu/all/bsp_common.o
 .text.R_FSP_VersionGet
                0x00000000        0xc ./ra/fsp/src/bsp/mcu/all/bsp_common.o
 .text.__assert_func
                0x00000000        0x4 ./ra/fsp/src/bsp/mcu/all/bsp_common.o
 .text          0x00000000        0x0 ./ra/fsp/src/bsp/mcu/all/bsp_delay.o
 .data          0x00000000        0x0 ./ra/fsp/src/bsp/mcu/all/bsp_delay.o
 .bss           0x00000000        0x0 ./ra/fsp/src/bsp/mcu/all/bsp_delay.o
 .text          0x00000000        0x0 ./ra/fsp/src/bsp/mcu/all/bsp_group_irq.o
 .data          0x00000000        0x0 ./ra/fsp/src/bsp/mcu/all/bsp_group_irq.o
 .bss           0x00000000        0x0 ./ra/fsp/src/bsp/mcu/all/bsp_group_irq.o
 .text.R_BSP_GroupIrqWrite
                0x00000000       0x10 ./ra/fsp/src/bsp/mcu/all/bsp_group_irq.o
 .text          0x00000000        0x0 ./ra/fsp/src/bsp/mcu/all/bsp_guard.o
 .data          0x00000000        0x0 ./ra/fsp/src/bsp/mcu/all/bsp_guard.o
 .bss           0x00000000        0x0 ./ra/fsp/src/bsp/mcu/all/bsp_guard.o
 .debug_info    0x00000000       0x7a ./ra/fsp/src/bsp/mcu/all/bsp_guard.o
 .debug_abbrev  0x00000000       0x26 ./ra/fsp/src/bsp/mcu/all/bsp_guard.o
 .debug_aranges
                0x00000000       0x18 ./ra/fsp/src/bsp/mcu/all/bsp_guard.o
 .debug_line    0x00000000       0x46 ./ra/fsp/src/bsp/mcu/all/bsp_guard.o
 .debug_str     0x00000000      0x1b5 ./ra/fsp/src/bsp/mcu/all/bsp_guard.o
 .comment       0x00000000       0x56 ./ra/fsp/src/bsp/mcu/all/bsp_guard.o
 .ARM.attributes
                0x00000000       0x3a ./ra/fsp/src/bsp/mcu/all/bsp_guard.o
 .text          0x00000000        0x0 ./ra/fsp/src/bsp/mcu/all/bsp_io.o
 .data          0x00000000        0x0 ./ra/fsp/src/bsp/mcu/all/bsp_io.o
 .bss           0x00000000        0x0 ./ra/fsp/src/bsp/mcu/all/bsp_io.o
 .text          0x00000000        0x0 ./ra/fsp/src/bsp/mcu/all/bsp_irq.o
 .data          0x00000000        0x0 ./ra/fsp/src/bsp/mcu/all/bsp_irq.o
 .bss           0x00000000        0x0 ./ra/fsp/src/bsp/mcu/all/bsp_irq.o
 .rodata.g_interrupt_event_link_select
                0x00000000       0xc0 ./ra/fsp/src/bsp/mcu/all/bsp_irq.o
 .text          0x00000000        0x0 ./ra/fsp/src/bsp/mcu/all/bsp_register_protection.o
 .data          0x00000000        0x0 ./ra/fsp/src/bsp/mcu/all/bsp_register_protection.o
 .bss           0x00000000        0x0 ./ra/fsp/src/bsp/mcu/all/bsp_register_protection.o
 .text          0x00000000        0x0 ./ra/fsp/src/bsp/mcu/all/bsp_rom_registers.o
 .data          0x00000000        0x0 ./ra/fsp/src/bsp/mcu/all/bsp_rom_registers.o
 .bss           0x00000000        0x0 ./ra/fsp/src/bsp/mcu/all/bsp_rom_registers.o
 .text          0x00000000        0x0 ./ra/fsp/src/bsp/mcu/all/bsp_sbrk.o
 .data          0x00000000        0x0 ./ra/fsp/src/bsp/mcu/all/bsp_sbrk.o
 .bss           0x00000000        0x0 ./ra/fsp/src/bsp/mcu/all/bsp_sbrk.o
 .text._sbrk    0x00000000       0x40 ./ra/fsp/src/bsp/mcu/all/bsp_sbrk.o
 .bss.current_heap_end.0
                0x00000000        0x4 ./ra/fsp/src/bsp/mcu/all/bsp_sbrk.o
 .debug_info    0x00000000      0x142 ./ra/fsp/src/bsp/mcu/all/bsp_sbrk.o
 .debug_abbrev  0x00000000       0xce ./ra/fsp/src/bsp/mcu/all/bsp_sbrk.o
 .debug_loclists
                0x00000000       0xa5 ./ra/fsp/src/bsp/mcu/all/bsp_sbrk.o
 .debug_aranges
                0x00000000       0x20 ./ra/fsp/src/bsp/mcu/all/bsp_sbrk.o
 .debug_rnglists
                0x00000000       0x13 ./ra/fsp/src/bsp/mcu/all/bsp_sbrk.o
 .debug_line    0x00000000      0x1d3 ./ra/fsp/src/bsp/mcu/all/bsp_sbrk.o
 .debug_str     0x00000000      0x23f ./ra/fsp/src/bsp/mcu/all/bsp_sbrk.o
 .comment       0x00000000       0x56 ./ra/fsp/src/bsp/mcu/all/bsp_sbrk.o
 .debug_frame   0x00000000       0x28 ./ra/fsp/src/bsp/mcu/all/bsp_sbrk.o
 .ARM.attributes
                0x00000000       0x3a ./ra/fsp/src/bsp/mcu/all/bsp_sbrk.o
 .text          0x00000000        0x0 ./ra/fsp/src/bsp/mcu/all/bsp_security.o
 .data          0x00000000        0x0 ./ra/fsp/src/bsp/mcu/all/bsp_security.o
 .bss           0x00000000        0x0 ./ra/fsp/src/bsp/mcu/all/bsp_security.o
 .rodata.gp_start_of_nonsecure_callable_ram
                0x00000000        0x4 ./ra/fsp/src/bsp/mcu/all/bsp_security.o
 .rodata.gp_start_of_nonsecure_ram
                0x00000000        0x4 ./ra/fsp/src/bsp/mcu/all/bsp_security.o
 .rodata.gp_start_of_nonsecure_data_flash
                0x00000000        0x4 ./ra/fsp/src/bsp/mcu/all/bsp_security.o
 .rodata.gp_start_of_nonsecure_callable_flash
                0x00000000        0x4 ./ra/fsp/src/bsp/mcu/all/bsp_security.o
 .rodata.gp_start_of_nonsecure_flash
                0x00000000        0x4 ./ra/fsp/src/bsp/mcu/all/bsp_security.o
 .debug_info    0x00000000      0x12c ./ra/fsp/src/bsp/mcu/all/bsp_security.o
 .debug_abbrev  0x00000000       0x82 ./ra/fsp/src/bsp/mcu/all/bsp_security.o
 .debug_aranges
                0x00000000       0x18 ./ra/fsp/src/bsp/mcu/all/bsp_security.o
 .debug_line    0x00000000      0x142 ./ra/fsp/src/bsp/mcu/all/bsp_security.o
 .debug_str     0x00000000      0x2b5 ./ra/fsp/src/bsp/mcu/all/bsp_security.o
 .comment       0x00000000       0x56 ./ra/fsp/src/bsp/mcu/all/bsp_security.o
 .ARM.attributes
                0x00000000       0x3a ./ra/fsp/src/bsp/mcu/all/bsp_security.o
 .text          0x00000000        0x0 ./ra/fsp/src/bsp/cmsis/Device/RENESAS/Source/startup.o
 .data          0x00000000        0x0 ./ra/fsp/src/bsp/cmsis/Device/RENESAS/Source/startup.o
 .bss           0x00000000        0x0 ./ra/fsp/src/bsp/cmsis/Device/RENESAS/Source/startup.o
 .text          0x00000000        0x0 ./ra/fsp/src/bsp/cmsis/Device/RENESAS/Source/system.o
 .data          0x00000000        0x0 ./ra/fsp/src/bsp/cmsis/Device/RENESAS/Source/system.o
 .bss           0x00000000        0x0 ./ra/fsp/src/bsp/cmsis/Device/RENESAS/Source/system.o
 .text.R_BSP_WarmStart
                0x00000000        0x4 ./ra/fsp/src/bsp/cmsis/Device/RENESAS/Source/system.o
 .text          0x00000000      0x254 c:/renesas/ra/e2studio_v2023-10_fsp_v5.0.0/toolchains/gcc_arm/12.2.mpacbti-rel1/bin/../lib/gcc/arm-none-eabi/12.2.1/thumb/v8-m.main+fp/hard\libgcc.a(_arm_muldf3.o)
 .data          0x00000000        0x0 c:/renesas/ra/e2studio_v2023-10_fsp_v5.0.0/toolchains/gcc_arm/12.2.mpacbti-rel1/bin/../lib/gcc/arm-none-eabi/12.2.1/thumb/v8-m.main+fp/hard\libgcc.a(_arm_muldf3.o)
 .bss           0x00000000        0x0 c:/renesas/ra/e2studio_v2023-10_fsp_v5.0.0/toolchains/gcc_arm/12.2.mpacbti-rel1/bin/../lib/gcc/arm-none-eabi/12.2.1/thumb/v8-m.main+fp/hard\libgcc.a(_arm_muldf3.o)
 .debug_line_str
                0x00000000       0xe2 c:/renesas/ra/e2studio_v2023-10_fsp_v5.0.0/toolchains/gcc_arm/12.2.mpacbti-rel1/bin/../lib/gcc/arm-none-eabi/12.2.1/thumb/v8-m.main+fp/hard\libgcc.a(_arm_muldf3.o)
 .debug_frame   0x00000000       0x30 c:/renesas/ra/e2studio_v2023-10_fsp_v5.0.0/toolchains/gcc_arm/12.2.mpacbti-rel1/bin/../lib/gcc/arm-none-eabi/12.2.1/thumb/v8-m.main+fp/hard\libgcc.a(_arm_muldf3.o)
 .ARM.attributes
                0x00000000       0x26 c:/renesas/ra/e2studio_v2023-10_fsp_v5.0.0/toolchains/gcc_arm/12.2.mpacbti-rel1/bin/../lib/gcc/arm-none-eabi/12.2.1/thumb/v8-m.main+fp/hard\libgcc.a(_arm_muldf3.o)
 .data          0x00000000        0x0 c:/renesas/ra/e2studio_v2023-10_fsp_v5.0.0/toolchains/gcc_arm/12.2.mpacbti-rel1/bin/../lib/gcc/arm-none-eabi/12.2.1/thumb/v8-m.main+fp/hard\libgcc.a(_arm_addsubdf3.o)
 .bss           0x00000000        0x0 c:/renesas/ra/e2studio_v2023-10_fsp_v5.0.0/toolchains/gcc_arm/12.2.mpacbti-rel1/bin/../lib/gcc/arm-none-eabi/12.2.1/thumb/v8-m.main+fp/hard\libgcc.a(_arm_addsubdf3.o)
 .data          0x00000000        0x0 c:/renesas/ra/e2studio_v2023-10_fsp_v5.0.0/toolchains/gcc_arm/12.2.mpacbti-rel1/bin/../lib/gcc/arm-none-eabi/12.2.1/thumb/v8-m.main+fp/hard\libgcc.a(_arm_muldivdf3.o)
 .bss           0x00000000        0x0 c:/renesas/ra/e2studio_v2023-10_fsp_v5.0.0/toolchains/gcc_arm/12.2.mpacbti-rel1/bin/../lib/gcc/arm-none-eabi/12.2.1/thumb/v8-m.main+fp/hard\libgcc.a(_arm_muldivdf3.o)
 .data          0x00000000        0x0 c:/renesas/ra/e2studio_v2023-10_fsp_v5.0.0/toolchains/gcc_arm/12.2.mpacbti-rel1/bin/../lib/gcc/arm-none-eabi/12.2.1/thumb/v8-m.main+fp/hard\libgcc.a(_arm_cmpdf2.o)
 .bss           0x00000000        0x0 c:/renesas/ra/e2studio_v2023-10_fsp_v5.0.0/toolchains/gcc_arm/12.2.mpacbti-rel1/bin/../lib/gcc/arm-none-eabi/12.2.1/thumb/v8-m.main+fp/hard\libgcc.a(_arm_cmpdf2.o)
 .text          0x00000000       0x2c c:/renesas/ra/e2studio_v2023-10_fsp_v5.0.0/toolchains/gcc_arm/12.2.mpacbti-rel1/bin/../lib/gcc/arm-none-eabi/12.2.1/thumb/v8-m.main+fp/hard\libgcc.a(_arm_unorddf2.o)
 .data          0x00000000        0x0 c:/renesas/ra/e2studio_v2023-10_fsp_v5.0.0/toolchains/gcc_arm/12.2.mpacbti-rel1/bin/../lib/gcc/arm-none-eabi/12.2.1/thumb/v8-m.main+fp/hard\libgcc.a(_arm_unorddf2.o)
 .bss           0x00000000        0x0 c:/renesas/ra/e2studio_v2023-10_fsp_v5.0.0/toolchains/gcc_arm/12.2.mpacbti-rel1/bin/../lib/gcc/arm-none-eabi/12.2.1/thumb/v8-m.main+fp/hard\libgcc.a(_arm_unorddf2.o)
 .debug_line_str
                0x00000000       0xe2 c:/renesas/ra/e2studio_v2023-10_fsp_v5.0.0/toolchains/gcc_arm/12.2.mpacbti-rel1/bin/../lib/gcc/arm-none-eabi/12.2.1/thumb/v8-m.main+fp/hard\libgcc.a(_arm_unorddf2.o)
 .debug_frame   0x00000000       0x20 c:/renesas/ra/e2studio_v2023-10_fsp_v5.0.0/toolchains/gcc_arm/12.2.mpacbti-rel1/bin/../lib/gcc/arm-none-eabi/12.2.1/thumb/v8-m.main+fp/hard\libgcc.a(_arm_unorddf2.o)
 .ARM.attributes
                0x00000000       0x26 c:/renesas/ra/e2studio_v2023-10_fsp_v5.0.0/toolchains/gcc_arm/12.2.mpacbti-rel1/bin/../lib/gcc/arm-none-eabi/12.2.1/thumb/v8-m.main+fp/hard\libgcc.a(_arm_unorddf2.o)
 .data          0x00000000        0x0 c:/renesas/ra/e2studio_v2023-10_fsp_v5.0.0/toolchains/gcc_arm/12.2.mpacbti-rel1/bin/../lib/gcc/arm-none-eabi/12.2.1/thumb/v8-m.main+fp/hard\libgcc.a(_arm_fixdfsi.o)
 .bss           0x00000000        0x0 c:/renesas/ra/e2studio_v2023-10_fsp_v5.0.0/toolchains/gcc_arm/12.2.mpacbti-rel1/bin/../lib/gcc/arm-none-eabi/12.2.1/thumb/v8-m.main+fp/hard\libgcc.a(_arm_fixdfsi.o)
 .data          0x00000000        0x0 c:/renesas/ra/e2studio_v2023-10_fsp_v5.0.0/toolchains/gcc_arm/12.2.mpacbti-rel1/bin/../lib/gcc/arm-none-eabi/12.2.1/thumb/v8-m.main+fp/hard\libgcc.a(_arm_fixunsdfsi.o)
 .bss           0x00000000        0x0 c:/renesas/ra/e2studio_v2023-10_fsp_v5.0.0/toolchains/gcc_arm/12.2.mpacbti-rel1/bin/../lib/gcc/arm-none-eabi/12.2.1/thumb/v8-m.main+fp/hard\libgcc.a(_arm_fixunsdfsi.o)
 .data          0x00000000        0x0 c:/renesas/ra/e2studio_v2023-10_fsp_v5.0.0/toolchains/gcc_arm/12.2.mpacbti-rel1/bin/../lib/gcc/arm-none-eabi/12.2.1/thumb/v8-m.main+fp/hard\libgcc.a(_aeabi_ldivmod.o)
 .bss           0x00000000        0x0 c:/renesas/ra/e2studio_v2023-10_fsp_v5.0.0/toolchains/gcc_arm/12.2.mpacbti-rel1/bin/../lib/gcc/arm-none-eabi/12.2.1/thumb/v8-m.main+fp/hard\libgcc.a(_aeabi_ldivmod.o)
 .text          0x00000000        0x0 c:/renesas/ra/e2studio_v2023-10_fsp_v5.0.0/toolchains/gcc_arm/12.2.mpacbti-rel1/bin/../lib/gcc/arm-none-eabi/12.2.1/thumb/v8-m.main+fp/hard\libgcc.a(_udivmoddi4.o)
 .data          0x00000000        0x0 c:/renesas/ra/e2studio_v2023-10_fsp_v5.0.0/toolchains/gcc_arm/12.2.mpacbti-rel1/bin/../lib/gcc/arm-none-eabi/12.2.1/thumb/v8-m.main+fp/hard\libgcc.a(_udivmoddi4.o)
 .bss           0x00000000        0x0 c:/renesas/ra/e2studio_v2023-10_fsp_v5.0.0/toolchains/gcc_arm/12.2.mpacbti-rel1/bin/../lib/gcc/arm-none-eabi/12.2.1/thumb/v8-m.main+fp/hard\libgcc.a(_udivmoddi4.o)
 .ARM.extab.text.__udivmoddi4
                0x00000000        0x0 c:/renesas/ra/e2studio_v2023-10_fsp_v5.0.0/toolchains/gcc_arm/12.2.mpacbti-rel1/bin/../lib/gcc/arm-none-eabi/12.2.1/thumb/v8-m.main+fp/hard\libgcc.a(_udivmoddi4.o)
 .ARM.exidx.text.__udivmoddi4
                0x00000000        0x8 c:/renesas/ra/e2studio_v2023-10_fsp_v5.0.0/toolchains/gcc_arm/12.2.mpacbti-rel1/bin/../lib/gcc/arm-none-eabi/12.2.1/thumb/v8-m.main+fp/hard\libgcc.a(_udivmoddi4.o)
 .data          0x00000000        0x0 c:/renesas/ra/e2studio_v2023-10_fsp_v5.0.0/toolchains/gcc_arm/12.2.mpacbti-rel1/bin/../lib/gcc/arm-none-eabi/12.2.1/thumb/v8-m.main+fp/hard\libgcc.a(_dvmd_tls.o)
 .bss           0x00000000        0x0 c:/renesas/ra/e2studio_v2023-10_fsp_v5.0.0/toolchains/gcc_arm/12.2.mpacbti-rel1/bin/../lib/gcc/arm-none-eabi/12.2.1/thumb/v8-m.main+fp/hard\libgcc.a(_dvmd_tls.o)
 .text          0x00000000        0x0 c:/renesas/ra/e2studio_v2023-10_fsp_v5.0.0/toolchains/gcc_arm/12.2.mpacbti-rel1/bin/../lib/gcc/arm-none-eabi/12.2.1/thumb/v8-m.main+fp/hard\libg_nano.a(libc_a-exit.o)
 .data          0x00000000        0x0 c:/renesas/ra/e2studio_v2023-10_fsp_v5.0.0/toolchains/gcc_arm/12.2.mpacbti-rel1/bin/../lib/gcc/arm-none-eabi/12.2.1/thumb/v8-m.main+fp/hard\libg_nano.a(libc_a-exit.o)
 .bss           0x00000000        0x0 c:/renesas/ra/e2studio_v2023-10_fsp_v5.0.0/toolchains/gcc_arm/12.2.mpacbti-rel1/bin/../lib/gcc/arm-none-eabi/12.2.1/thumb/v8-m.main+fp/hard\libg_nano.a(libc_a-exit.o)
 .text.exit     0x00000000       0x24 c:/renesas/ra/e2studio_v2023-10_fsp_v5.0.0/toolchains/gcc_arm/12.2.mpacbti-rel1/bin/../lib/gcc/arm-none-eabi/12.2.1/thumb/v8-m.main+fp/hard\libg_nano.a(libc_a-exit.o)
 .debug_frame   0x00000000       0x28 c:/renesas/ra/e2studio_v2023-10_fsp_v5.0.0/toolchains/gcc_arm/12.2.mpacbti-rel1/bin/../lib/gcc/arm-none-eabi/12.2.1/thumb/v8-m.main+fp/hard\libg_nano.a(libc_a-exit.o)
 .ARM.attributes
                0x00000000       0x38 c:/renesas/ra/e2studio_v2023-10_fsp_v5.0.0/toolchains/gcc_arm/12.2.mpacbti-rel1/bin/../lib/gcc/arm-none-eabi/12.2.1/thumb/v8-m.main+fp/hard\libg_nano.a(libc_a-exit.o)
 .text          0x00000000        0x0 c:/renesas/ra/e2studio_v2023-10_fsp_v5.0.0/toolchains/gcc_arm/12.2.mpacbti-rel1/bin/../lib/gcc/arm-none-eabi/12.2.1/thumb/v8-m.main+fp/hard\libg_nano.a(libc_a-itoa.o)
 .data          0x00000000        0x0 c:/renesas/ra/e2studio_v2023-10_fsp_v5.0.0/toolchains/gcc_arm/12.2.mpacbti-rel1/bin/../lib/gcc/arm-none-eabi/12.2.1/thumb/v8-m.main+fp/hard\libg_nano.a(libc_a-itoa.o)
 .bss           0x00000000        0x0 c:/renesas/ra/e2studio_v2023-10_fsp_v5.0.0/toolchains/gcc_arm/12.2.mpacbti-rel1/bin/../lib/gcc/arm-none-eabi/12.2.1/thumb/v8-m.main+fp/hard\libg_nano.a(libc_a-itoa.o)
 .text.itoa     0x00000000        0x4 c:/renesas/ra/e2studio_v2023-10_fsp_v5.0.0/toolchains/gcc_arm/12.2.mpacbti-rel1/bin/../lib/gcc/arm-none-eabi/12.2.1/thumb/v8-m.main+fp/hard\libg_nano.a(libc_a-itoa.o)
 .text          0x00000000        0x0 c:/renesas/ra/e2studio_v2023-10_fsp_v5.0.0/toolchains/gcc_arm/12.2.mpacbti-rel1/bin/../lib/gcc/arm-none-eabi/12.2.1/thumb/v8-m.main+fp/hard\libg_nano.a(libc_a-strtol.o)
 .data          0x00000000        0x0 c:/renesas/ra/e2studio_v2023-10_fsp_v5.0.0/toolchains/gcc_arm/12.2.mpacbti-rel1/bin/../lib/gcc/arm-none-eabi/12.2.1/thumb/v8-m.main+fp/hard\libg_nano.a(libc_a-strtol.o)
 .bss           0x00000000        0x0 c:/renesas/ra/e2studio_v2023-10_fsp_v5.0.0/toolchains/gcc_arm/12.2.mpacbti-rel1/bin/../lib/gcc/arm-none-eabi/12.2.1/thumb/v8-m.main+fp/hard\libg_nano.a(libc_a-strtol.o)
 .text._strtol_r
                0x00000000        0x4 c:/renesas/ra/e2studio_v2023-10_fsp_v5.0.0/toolchains/gcc_arm/12.2.mpacbti-rel1/bin/../lib/gcc/arm-none-eabi/12.2.1/thumb/v8-m.main+fp/hard\libg_nano.a(libc_a-strtol.o)
 .text.strtol_l
                0x00000000       0x14 c:/renesas/ra/e2studio_v2023-10_fsp_v5.0.0/toolchains/gcc_arm/12.2.mpacbti-rel1/bin/../lib/gcc/arm-none-eabi/12.2.1/thumb/v8-m.main+fp/hard\libg_nano.a(libc_a-strtol.o)
 .text          0x00000000        0x0 c:/renesas/ra/e2studio_v2023-10_fsp_v5.0.0/toolchains/gcc_arm/12.2.mpacbti-rel1/bin/../lib/gcc/arm-none-eabi/12.2.1/thumb/v8-m.main+fp/hard\libg_nano.a(libc_a-utoa.o)
 .data          0x00000000        0x0 c:/renesas/ra/e2studio_v2023-10_fsp_v5.0.0/toolchains/gcc_arm/12.2.mpacbti-rel1/bin/../lib/gcc/arm-none-eabi/12.2.1/thumb/v8-m.main+fp/hard\libg_nano.a(libc_a-utoa.o)
 .bss           0x00000000        0x0 c:/renesas/ra/e2studio_v2023-10_fsp_v5.0.0/toolchains/gcc_arm/12.2.mpacbti-rel1/bin/../lib/gcc/arm-none-eabi/12.2.1/thumb/v8-m.main+fp/hard\libg_nano.a(libc_a-utoa.o)
 .text.utoa     0x00000000        0x4 c:/renesas/ra/e2studio_v2023-10_fsp_v5.0.0/toolchains/gcc_arm/12.2.mpacbti-rel1/bin/../lib/gcc/arm-none-eabi/12.2.1/thumb/v8-m.main+fp/hard\libg_nano.a(libc_a-utoa.o)
 .text          0x00000000        0x0 c:/renesas/ra/e2studio_v2023-10_fsp_v5.0.0/toolchains/gcc_arm/12.2.mpacbti-rel1/bin/../lib/gcc/arm-none-eabi/12.2.1/thumb/v8-m.main+fp/hard\libg_nano.a(libc_a-ctype_.o)
 .data          0x00000000        0x0 c:/renesas/ra/e2studio_v2023-10_fsp_v5.0.0/toolchains/gcc_arm/12.2.mpacbti-rel1/bin/../lib/gcc/arm-none-eabi/12.2.1/thumb/v8-m.main+fp/hard\libg_nano.a(libc_a-ctype_.o)
 .bss           0x00000000        0x0 c:/renesas/ra/e2studio_v2023-10_fsp_v5.0.0/toolchains/gcc_arm/12.2.mpacbti-rel1/bin/../lib/gcc/arm-none-eabi/12.2.1/thumb/v8-m.main+fp/hard\libg_nano.a(libc_a-ctype_.o)
 .text          0x00000000        0x0 c:/renesas/ra/e2studio_v2023-10_fsp_v5.0.0/toolchains/gcc_arm/12.2.mpacbti-rel1/bin/../lib/gcc/arm-none-eabi/12.2.1/thumb/v8-m.main+fp/hard\libg_nano.a(libc_a-findfp.o)
 .data          0x00000000        0x0 c:/renesas/ra/e2studio_v2023-10_fsp_v5.0.0/toolchains/gcc_arm/12.2.mpacbti-rel1/bin/../lib/gcc/arm-none-eabi/12.2.1/thumb/v8-m.main+fp/hard\libg_nano.a(libc_a-findfp.o)
 .bss           0x00000000        0x0 c:/renesas/ra/e2studio_v2023-10_fsp_v5.0.0/toolchains/gcc_arm/12.2.mpacbti-rel1/bin/../lib/gcc/arm-none-eabi/12.2.1/thumb/v8-m.main+fp/hard\libg_nano.a(libc_a-findfp.o)
 .text.std      0x00000000       0x6c c:/renesas/ra/e2studio_v2023-10_fsp_v5.0.0/toolchains/gcc_arm/12.2.mpacbti-rel1/bin/../lib/gcc/arm-none-eabi/12.2.1/thumb/v8-m.main+fp/hard\libg_nano.a(libc_a-findfp.o)
 .text.stdio_exit_handler
                0x00000000       0x18 c:/renesas/ra/e2studio_v2023-10_fsp_v5.0.0/toolchains/gcc_arm/12.2.mpacbti-rel1/bin/../lib/gcc/arm-none-eabi/12.2.1/thumb/v8-m.main+fp/hard\libg_nano.a(libc_a-findfp.o)
 .text.cleanup_stdio
                0x00000000       0x40 c:/renesas/ra/e2studio_v2023-10_fsp_v5.0.0/toolchains/gcc_arm/12.2.mpacbti-rel1/bin/../lib/gcc/arm-none-eabi/12.2.1/thumb/v8-m.main+fp/hard\libg_nano.a(libc_a-findfp.o)
 .text.__fp_lock
                0x00000000       0x18 c:/renesas/ra/e2studio_v2023-10_fsp_v5.0.0/toolchains/gcc_arm/12.2.mpacbti-rel1/bin/../lib/gcc/arm-none-eabi/12.2.1/thumb/v8-m.main+fp/hard\libg_nano.a(libc_a-findfp.o)
 .text.__fp_unlock
                0x00000000       0x18 c:/renesas/ra/e2studio_v2023-10_fsp_v5.0.0/toolchains/gcc_arm/12.2.mpacbti-rel1/bin/../lib/gcc/arm-none-eabi/12.2.1/thumb/v8-m.main+fp/hard\libg_nano.a(libc_a-findfp.o)
 .text.global_stdio_init.part.0
                0x00000000       0x3c c:/renesas/ra/e2studio_v2023-10_fsp_v5.0.0/toolchains/gcc_arm/12.2.mpacbti-rel1/bin/../lib/gcc/arm-none-eabi/12.2.1/thumb/v8-m.main+fp/hard\libg_nano.a(libc_a-findfp.o)
 .text.__sfp_lock_acquire
                0x00000000        0xc c:/renesas/ra/e2studio_v2023-10_fsp_v5.0.0/toolchains/gcc_arm/12.2.mpacbti-rel1/bin/../lib/gcc/arm-none-eabi/12.2.1/thumb/v8-m.main+fp/hard\libg_nano.a(libc_a-findfp.o)
 .text.__sfp_lock_release
                0x00000000        0xc c:/renesas/ra/e2studio_v2023-10_fsp_v5.0.0/toolchains/gcc_arm/12.2.mpacbti-rel1/bin/../lib/gcc/arm-none-eabi/12.2.1/thumb/v8-m.main+fp/hard\libg_nano.a(libc_a-findfp.o)
 .text.__sfp    0x00000000       0xa4 c:/renesas/ra/e2studio_v2023-10_fsp_v5.0.0/toolchains/gcc_arm/12.2.mpacbti-rel1/bin/../lib/gcc/arm-none-eabi/12.2.1/thumb/v8-m.main+fp/hard\libg_nano.a(libc_a-findfp.o)
 .text.__sinit  0x00000000       0x30 c:/renesas/ra/e2studio_v2023-10_fsp_v5.0.0/toolchains/gcc_arm/12.2.mpacbti-rel1/bin/../lib/gcc/arm-none-eabi/12.2.1/thumb/v8-m.main+fp/hard\libg_nano.a(libc_a-findfp.o)
 .text.__fp_lock_all
                0x00000000       0x1c c:/renesas/ra/e2studio_v2023-10_fsp_v5.0.0/toolchains/gcc_arm/12.2.mpacbti-rel1/bin/../lib/gcc/arm-none-eabi/12.2.1/thumb/v8-m.main+fp/hard\libg_nano.a(libc_a-findfp.o)
 .text.__fp_unlock_all
                0x00000000       0x1c c:/renesas/ra/e2studio_v2023-10_fsp_v5.0.0/toolchains/gcc_arm/12.2.mpacbti-rel1/bin/../lib/gcc/arm-none-eabi/12.2.1/thumb/v8-m.main+fp/hard\libg_nano.a(libc_a-findfp.o)
 .data.__sglue  0x00000000        0xc c:/renesas/ra/e2studio_v2023-10_fsp_v5.0.0/toolchains/gcc_arm/12.2.mpacbti-rel1/bin/../lib/gcc/arm-none-eabi/12.2.1/thumb/v8-m.main+fp/hard\libg_nano.a(libc_a-findfp.o)
 .bss.__stdio_exit_handler
                0x00000000        0x4 c:/renesas/ra/e2studio_v2023-10_fsp_v5.0.0/toolchains/gcc_arm/12.2.mpacbti-rel1/bin/../lib/gcc/arm-none-eabi/12.2.1/thumb/v8-m.main+fp/hard\libg_nano.a(libc_a-findfp.o)
 .text          0x00000000        0x0 c:/renesas/ra/e2studio_v2023-10_fsp_v5.0.0/toolchains/gcc_arm/12.2.mpacbti-rel1/bin/../lib/gcc/arm-none-eabi/12.2.1/thumb/v8-m.main+fp/hard\libg_nano.a(libc_a-fwalk.o)
 .data          0x00000000        0x0 c:/renesas/ra/e2studio_v2023-10_fsp_v5.0.0/toolchains/gcc_arm/12.2.mpacbti-rel1/bin/../lib/gcc/arm-none-eabi/12.2.1/thumb/v8-m.main+fp/hard\libg_nano.a(libc_a-fwalk.o)
 .bss           0x00000000        0x0 c:/renesas/ra/e2studio_v2023-10_fsp_v5.0.0/toolchains/gcc_arm/12.2.mpacbti-rel1/bin/../lib/gcc/arm-none-eabi/12.2.1/thumb/v8-m.main+fp/hard\libg_nano.a(libc_a-fwalk.o)
 .text._fwalk_sglue
                0x00000000       0x3c c:/renesas/ra/e2studio_v2023-10_fsp_v5.0.0/toolchains/gcc_arm/12.2.mpacbti-rel1/bin/../lib/gcc/arm-none-eabi/12.2.1/thumb/v8-m.main+fp/hard\libg_nano.a(libc_a-fwalk.o)
 .debug_frame   0x00000000       0x34 c:/renesas/ra/e2studio_v2023-10_fsp_v5.0.0/toolchains/gcc_arm/12.2.mpacbti-rel1/bin/../lib/gcc/arm-none-eabi/12.2.1/thumb/v8-m.main+fp/hard\libg_nano.a(libc_a-fwalk.o)
 .ARM.attributes
                0x00000000       0x38 c:/renesas/ra/e2studio_v2023-10_fsp_v5.0.0/toolchains/gcc_arm/12.2.mpacbti-rel1/bin/../lib/gcc/arm-none-eabi/12.2.1/thumb/v8-m.main+fp/hard\libg_nano.a(libc_a-fwalk.o)
 .text          0x00000000        0x0 c:/renesas/ra/e2studio_v2023-10_fsp_v5.0.0/toolchains/gcc_arm/12.2.mpacbti-rel1/bin/../lib/gcc/arm-none-eabi/12.2.1/thumb/v8-m.main+fp/hard\libg_nano.a(libc_a-stdio.o)
 .data          0x00000000        0x0 c:/renesas/ra/e2studio_v2023-10_fsp_v5.0.0/toolchains/gcc_arm/12.2.mpacbti-rel1/bin/../lib/gcc/arm-none-eabi/12.2.1/thumb/v8-m.main+fp/hard\libg_nano.a(libc_a-stdio.o)
 .bss           0x00000000        0x0 c:/renesas/ra/e2studio_v2023-10_fsp_v5.0.0/toolchains/gcc_arm/12.2.mpacbti-rel1/bin/../lib/gcc/arm-none-eabi/12.2.1/thumb/v8-m.main+fp/hard\libg_nano.a(libc_a-stdio.o)
 .text.__sread  0x00000000       0x22 c:/renesas/ra/e2studio_v2023-10_fsp_v5.0.0/toolchains/gcc_arm/12.2.mpacbti-rel1/bin/../lib/gcc/arm-none-eabi/12.2.1/thumb/v8-m.main+fp/hard\libg_nano.a(libc_a-stdio.o)
 .text.__seofread
                0x00000000        0x4 c:/renesas/ra/e2studio_v2023-10_fsp_v5.0.0/toolchains/gcc_arm/12.2.mpacbti-rel1/bin/../lib/gcc/arm-none-eabi/12.2.1/thumb/v8-m.main+fp/hard\libg_nano.a(libc_a-stdio.o)
 .text.__swrite
                0x00000000       0x38 c:/renesas/ra/e2studio_v2023-10_fsp_v5.0.0/toolchains/gcc_arm/12.2.mpacbti-rel1/bin/../lib/gcc/arm-none-eabi/12.2.1/thumb/v8-m.main+fp/hard\libg_nano.a(libc_a-stdio.o)
 .text.__sseek  0x00000000       0x24 c:/renesas/ra/e2studio_v2023-10_fsp_v5.0.0/toolchains/gcc_arm/12.2.mpacbti-rel1/bin/../lib/gcc/arm-none-eabi/12.2.1/thumb/v8-m.main+fp/hard\libg_nano.a(libc_a-stdio.o)
 .text.__sclose
                0x00000000        0x8 c:/renesas/ra/e2studio_v2023-10_fsp_v5.0.0/toolchains/gcc_arm/12.2.mpacbti-rel1/bin/../lib/gcc/arm-none-eabi/12.2.1/thumb/v8-m.main+fp/hard\libg_nano.a(libc_a-stdio.o)
 .debug_frame   0x00000000       0x88 c:/renesas/ra/e2studio_v2023-10_fsp_v5.0.0/toolchains/gcc_arm/12.2.mpacbti-rel1/bin/../lib/gcc/arm-none-eabi/12.2.1/thumb/v8-m.main+fp/hard\libg_nano.a(libc_a-stdio.o)
 .ARM.attributes
                0x00000000       0x38 c:/renesas/ra/e2studio_v2023-10_fsp_v5.0.0/toolchains/gcc_arm/12.2.mpacbti-rel1/bin/../lib/gcc/arm-none-eabi/12.2.1/thumb/v8-m.main+fp/hard\libg_nano.a(libc_a-stdio.o)
 .text          0x00000000        0x0 c:/renesas/ra/e2studio_v2023-10_fsp_v5.0.0/toolchains/gcc_arm/12.2.mpacbti-rel1/bin/../lib/gcc/arm-none-eabi/12.2.1/thumb/v8-m.main+fp/hard\libg_nano.a(libc_a-memset.o)
 .data          0x00000000        0x0 c:/renesas/ra/e2studio_v2023-10_fsp_v5.0.0/toolchains/gcc_arm/12.2.mpacbti-rel1/bin/../lib/gcc/arm-none-eabi/12.2.1/thumb/v8-m.main+fp/hard\libg_nano.a(libc_a-memset.o)
 .bss           0x00000000        0x0 c:/renesas/ra/e2studio_v2023-10_fsp_v5.0.0/toolchains/gcc_arm/12.2.mpacbti-rel1/bin/../lib/gcc/arm-none-eabi/12.2.1/thumb/v8-m.main+fp/hard\libg_nano.a(libc_a-memset.o)
 .text          0x00000000        0x0 c:/renesas/ra/e2studio_v2023-10_fsp_v5.0.0/toolchains/gcc_arm/12.2.mpacbti-rel1/bin/../lib/gcc/arm-none-eabi/12.2.1/thumb/v8-m.main+fp/hard\libg_nano.a(libc_a-closer.o)
 .data          0x00000000        0x0 c:/renesas/ra/e2studio_v2023-10_fsp_v5.0.0/toolchains/gcc_arm/12.2.mpacbti-rel1/bin/../lib/gcc/arm-none-eabi/12.2.1/thumb/v8-m.main+fp/hard\libg_nano.a(libc_a-closer.o)
 .bss           0x00000000        0x0 c:/renesas/ra/e2studio_v2023-10_fsp_v5.0.0/toolchains/gcc_arm/12.2.mpacbti-rel1/bin/../lib/gcc/arm-none-eabi/12.2.1/thumb/v8-m.main+fp/hard\libg_nano.a(libc_a-closer.o)
 .text._close_r
                0x00000000       0x20 c:/renesas/ra/e2studio_v2023-10_fsp_v5.0.0/toolchains/gcc_arm/12.2.mpacbti-rel1/bin/../lib/gcc/arm-none-eabi/12.2.1/thumb/v8-m.main+fp/hard\libg_nano.a(libc_a-closer.o)
 .debug_frame   0x00000000       0x2c c:/renesas/ra/e2studio_v2023-10_fsp_v5.0.0/toolchains/gcc_arm/12.2.mpacbti-rel1/bin/../lib/gcc/arm-none-eabi/12.2.1/thumb/v8-m.main+fp/hard\libg_nano.a(libc_a-closer.o)
 .ARM.attributes
                0x00000000       0x38 c:/renesas/ra/e2studio_v2023-10_fsp_v5.0.0/toolchains/gcc_arm/12.2.mpacbti-rel1/bin/../lib/gcc/arm-none-eabi/12.2.1/thumb/v8-m.main+fp/hard\libg_nano.a(libc_a-closer.o)
 .text          0x00000000        0x0 c:/renesas/ra/e2studio_v2023-10_fsp_v5.0.0/toolchains/gcc_arm/12.2.mpacbti-rel1/bin/../lib/gcc/arm-none-eabi/12.2.1/thumb/v8-m.main+fp/hard\libg_nano.a(libc_a-reent.o)
 .data          0x00000000        0x0 c:/renesas/ra/e2studio_v2023-10_fsp_v5.0.0/toolchains/gcc_arm/12.2.mpacbti-rel1/bin/../lib/gcc/arm-none-eabi/12.2.1/thumb/v8-m.main+fp/hard\libg_nano.a(libc_a-reent.o)
 .bss           0x00000000        0x0 c:/renesas/ra/e2studio_v2023-10_fsp_v5.0.0/toolchains/gcc_arm/12.2.mpacbti-rel1/bin/../lib/gcc/arm-none-eabi/12.2.1/thumb/v8-m.main+fp/hard\libg_nano.a(libc_a-reent.o)
 .text._reclaim_reent
                0x00000000       0xac c:/renesas/ra/e2studio_v2023-10_fsp_v5.0.0/toolchains/gcc_arm/12.2.mpacbti-rel1/bin/../lib/gcc/arm-none-eabi/12.2.1/thumb/v8-m.main+fp/hard\libg_nano.a(libc_a-reent.o)
 .bss.errno     0x00000000        0x4 c:/renesas/ra/e2studio_v2023-10_fsp_v5.0.0/toolchains/gcc_arm/12.2.mpacbti-rel1/bin/../lib/gcc/arm-none-eabi/12.2.1/thumb/v8-m.main+fp/hard\libg_nano.a(libc_a-reent.o)
 .debug_frame   0x00000000       0x38 c:/renesas/ra/e2studio_v2023-10_fsp_v5.0.0/toolchains/gcc_arm/12.2.mpacbti-rel1/bin/../lib/gcc/arm-none-eabi/12.2.1/thumb/v8-m.main+fp/hard\libg_nano.a(libc_a-reent.o)
 .ARM.attributes
                0x00000000       0x38 c:/renesas/ra/e2studio_v2023-10_fsp_v5.0.0/toolchains/gcc_arm/12.2.mpacbti-rel1/bin/../lib/gcc/arm-none-eabi/12.2.1/thumb/v8-m.main+fp/hard\libg_nano.a(libc_a-reent.o)
 .text          0x00000000        0x0 c:/renesas/ra/e2studio_v2023-10_fsp_v5.0.0/toolchains/gcc_arm/12.2.mpacbti-rel1/bin/../lib/gcc/arm-none-eabi/12.2.1/thumb/v8-m.main+fp/hard\libg_nano.a(libc_a-impure.o)
 .data          0x00000000        0x0 c:/renesas/ra/e2studio_v2023-10_fsp_v5.0.0/toolchains/gcc_arm/12.2.mpacbti-rel1/bin/../lib/gcc/arm-none-eabi/12.2.1/thumb/v8-m.main+fp/hard\libg_nano.a(libc_a-impure.o)
 .bss           0x00000000        0x0 c:/renesas/ra/e2studio_v2023-10_fsp_v5.0.0/toolchains/gcc_arm/12.2.mpacbti-rel1/bin/../lib/gcc/arm-none-eabi/12.2.1/thumb/v8-m.main+fp/hard\libg_nano.a(libc_a-impure.o)
 .text          0x00000000        0x0 c:/renesas/ra/e2studio_v2023-10_fsp_v5.0.0/toolchains/gcc_arm/12.2.mpacbti-rel1/bin/../lib/gcc/arm-none-eabi/12.2.1/thumb/v8-m.main+fp/hard\libg_nano.a(libc_a-lseekr.o)
 .data          0x00000000        0x0 c:/renesas/ra/e2studio_v2023-10_fsp_v5.0.0/toolchains/gcc_arm/12.2.mpacbti-rel1/bin/../lib/gcc/arm-none-eabi/12.2.1/thumb/v8-m.main+fp/hard\libg_nano.a(libc_a-lseekr.o)
 .bss           0x00000000        0x0 c:/renesas/ra/e2studio_v2023-10_fsp_v5.0.0/toolchains/gcc_arm/12.2.mpacbti-rel1/bin/../lib/gcc/arm-none-eabi/12.2.1/thumb/v8-m.main+fp/hard\libg_nano.a(libc_a-lseekr.o)
 .text._lseek_r
                0x00000000       0x24 c:/renesas/ra/e2studio_v2023-10_fsp_v5.0.0/toolchains/gcc_arm/12.2.mpacbti-rel1/bin/../lib/gcc/arm-none-eabi/12.2.1/thumb/v8-m.main+fp/hard\libg_nano.a(libc_a-lseekr.o)
 .debug_frame   0x00000000       0x2c c:/renesas/ra/e2studio_v2023-10_fsp_v5.0.0/toolchains/gcc_arm/12.2.mpacbti-rel1/bin/../lib/gcc/arm-none-eabi/12.2.1/thumb/v8-m.main+fp/hard\libg_nano.a(libc_a-lseekr.o)
 .ARM.attributes
                0x00000000       0x38 c:/renesas/ra/e2studio_v2023-10_fsp_v5.0.0/toolchains/gcc_arm/12.2.mpacbti-rel1/bin/../lib/gcc/arm-none-eabi/12.2.1/thumb/v8-m.main+fp/hard\libg_nano.a(libc_a-lseekr.o)
 .text          0x00000000        0x0 c:/renesas/ra/e2studio_v2023-10_fsp_v5.0.0/toolchains/gcc_arm/12.2.mpacbti-rel1/bin/../lib/gcc/arm-none-eabi/12.2.1/thumb/v8-m.main+fp/hard\libg_nano.a(libc_a-readr.o)
 .data          0x00000000        0x0 c:/renesas/ra/e2studio_v2023-10_fsp_v5.0.0/toolchains/gcc_arm/12.2.mpacbti-rel1/bin/../lib/gcc/arm-none-eabi/12.2.1/thumb/v8-m.main+fp/hard\libg_nano.a(libc_a-readr.o)
 .bss           0x00000000        0x0 c:/renesas/ra/e2studio_v2023-10_fsp_v5.0.0/toolchains/gcc_arm/12.2.mpacbti-rel1/bin/../lib/gcc/arm-none-eabi/12.2.1/thumb/v8-m.main+fp/hard\libg_nano.a(libc_a-readr.o)
 .text._read_r  0x00000000       0x24 c:/renesas/ra/e2studio_v2023-10_fsp_v5.0.0/toolchains/gcc_arm/12.2.mpacbti-rel1/bin/../lib/gcc/arm-none-eabi/12.2.1/thumb/v8-m.main+fp/hard\libg_nano.a(libc_a-readr.o)
 .debug_frame   0x00000000       0x2c c:/renesas/ra/e2studio_v2023-10_fsp_v5.0.0/toolchains/gcc_arm/12.2.mpacbti-rel1/bin/../lib/gcc/arm-none-eabi/12.2.1/thumb/v8-m.main+fp/hard\libg_nano.a(libc_a-readr.o)
 .ARM.attributes
                0x00000000       0x38 c:/renesas/ra/e2studio_v2023-10_fsp_v5.0.0/toolchains/gcc_arm/12.2.mpacbti-rel1/bin/../lib/gcc/arm-none-eabi/12.2.1/thumb/v8-m.main+fp/hard\libg_nano.a(libc_a-readr.o)
 .text          0x00000000        0x0 c:/renesas/ra/e2studio_v2023-10_fsp_v5.0.0/toolchains/gcc_arm/12.2.mpacbti-rel1/bin/../lib/gcc/arm-none-eabi/12.2.1/thumb/v8-m.main+fp/hard\libg_nano.a(libc_a-writer.o)
 .data          0x00000000        0x0 c:/renesas/ra/e2studio_v2023-10_fsp_v5.0.0/toolchains/gcc_arm/12.2.mpacbti-rel1/bin/../lib/gcc/arm-none-eabi/12.2.1/thumb/v8-m.main+fp/hard\libg_nano.a(libc_a-writer.o)
 .bss           0x00000000        0x0 c:/renesas/ra/e2studio_v2023-10_fsp_v5.0.0/toolchains/gcc_arm/12.2.mpacbti-rel1/bin/../lib/gcc/arm-none-eabi/12.2.1/thumb/v8-m.main+fp/hard\libg_nano.a(libc_a-writer.o)
 .text._write_r
                0x00000000       0x24 c:/renesas/ra/e2studio_v2023-10_fsp_v5.0.0/toolchains/gcc_arm/12.2.mpacbti-rel1/bin/../lib/gcc/arm-none-eabi/12.2.1/thumb/v8-m.main+fp/hard\libg_nano.a(libc_a-writer.o)
 .debug_frame   0x00000000       0x2c c:/renesas/ra/e2studio_v2023-10_fsp_v5.0.0/toolchains/gcc_arm/12.2.mpacbti-rel1/bin/../lib/gcc/arm-none-eabi/12.2.1/thumb/v8-m.main+fp/hard\libg_nano.a(libc_a-writer.o)
 .ARM.attributes
                0x00000000       0x38 c:/renesas/ra/e2studio_v2023-10_fsp_v5.0.0/toolchains/gcc_arm/12.2.mpacbti-rel1/bin/../lib/gcc/arm-none-eabi/12.2.1/thumb/v8-m.main+fp/hard\libg_nano.a(libc_a-writer.o)
 .text          0x00000000        0x0 c:/renesas/ra/e2studio_v2023-10_fsp_v5.0.0/toolchains/gcc_arm/12.2.mpacbti-rel1/bin/../lib/gcc/arm-none-eabi/12.2.1/thumb/v8-m.main+fp/hard\libg_nano.a(libc_a-errno.o)
 .data          0x00000000        0x0 c:/renesas/ra/e2studio_v2023-10_fsp_v5.0.0/toolchains/gcc_arm/12.2.mpacbti-rel1/bin/../lib/gcc/arm-none-eabi/12.2.1/thumb/v8-m.main+fp/hard\libg_nano.a(libc_a-errno.o)
 .bss           0x00000000        0x0 c:/renesas/ra/e2studio_v2023-10_fsp_v5.0.0/toolchains/gcc_arm/12.2.mpacbti-rel1/bin/../lib/gcc/arm-none-eabi/12.2.1/thumb/v8-m.main+fp/hard\libg_nano.a(libc_a-errno.o)
 .text          0x00000000        0x0 c:/renesas/ra/e2studio_v2023-10_fsp_v5.0.0/toolchains/gcc_arm/12.2.mpacbti-rel1/bin/../lib/gcc/arm-none-eabi/12.2.1/thumb/v8-m.main+fp/hard\libg_nano.a(libc_a-init.o)
 .data          0x00000000        0x0 c:/renesas/ra/e2studio_v2023-10_fsp_v5.0.0/toolchains/gcc_arm/12.2.mpacbti-rel1/bin/../lib/gcc/arm-none-eabi/12.2.1/thumb/v8-m.main+fp/hard\libg_nano.a(libc_a-init.o)
 .bss           0x00000000        0x0 c:/renesas/ra/e2studio_v2023-10_fsp_v5.0.0/toolchains/gcc_arm/12.2.mpacbti-rel1/bin/../lib/gcc/arm-none-eabi/12.2.1/thumb/v8-m.main+fp/hard\libg_nano.a(libc_a-init.o)
 .text.__libc_init_array
                0x00000000       0x48 c:/renesas/ra/e2studio_v2023-10_fsp_v5.0.0/toolchains/gcc_arm/12.2.mpacbti-rel1/bin/../lib/gcc/arm-none-eabi/12.2.1/thumb/v8-m.main+fp/hard\libg_nano.a(libc_a-init.o)
 .debug_frame   0x00000000       0x2c c:/renesas/ra/e2studio_v2023-10_fsp_v5.0.0/toolchains/gcc_arm/12.2.mpacbti-rel1/bin/../lib/gcc/arm-none-eabi/12.2.1/thumb/v8-m.main+fp/hard\libg_nano.a(libc_a-init.o)
 .ARM.attributes
                0x00000000       0x38 c:/renesas/ra/e2studio_v2023-10_fsp_v5.0.0/toolchains/gcc_arm/12.2.mpacbti-rel1/bin/../lib/gcc/arm-none-eabi/12.2.1/thumb/v8-m.main+fp/hard\libg_nano.a(libc_a-init.o)
 .text          0x00000000        0x0 c:/renesas/ra/e2studio_v2023-10_fsp_v5.0.0/toolchains/gcc_arm/12.2.mpacbti-rel1/bin/../lib/gcc/arm-none-eabi/12.2.1/thumb/v8-m.main+fp/hard\libg_nano.a(libc_a-lock.o)
 .data          0x00000000        0x0 c:/renesas/ra/e2studio_v2023-10_fsp_v5.0.0/toolchains/gcc_arm/12.2.mpacbti-rel1/bin/../lib/gcc/arm-none-eabi/12.2.1/thumb/v8-m.main+fp/hard\libg_nano.a(libc_a-lock.o)
 .bss           0x00000000        0x0 c:/renesas/ra/e2studio_v2023-10_fsp_v5.0.0/toolchains/gcc_arm/12.2.mpacbti-rel1/bin/../lib/gcc/arm-none-eabi/12.2.1/thumb/v8-m.main+fp/hard\libg_nano.a(libc_a-lock.o)
 .text.__retarget_lock_init
                0x00000000        0x2 c:/renesas/ra/e2studio_v2023-10_fsp_v5.0.0/toolchains/gcc_arm/12.2.mpacbti-rel1/bin/../lib/gcc/arm-none-eabi/12.2.1/thumb/v8-m.main+fp/hard\libg_nano.a(libc_a-lock.o)
 .text.__retarget_lock_init_recursive
                0x00000000        0x2 c:/renesas/ra/e2studio_v2023-10_fsp_v5.0.0/toolchains/gcc_arm/12.2.mpacbti-rel1/bin/../lib/gcc/arm-none-eabi/12.2.1/thumb/v8-m.main+fp/hard\libg_nano.a(libc_a-lock.o)
 .text.__retarget_lock_close
                0x00000000        0x2 c:/renesas/ra/e2studio_v2023-10_fsp_v5.0.0/toolchains/gcc_arm/12.2.mpacbti-rel1/bin/../lib/gcc/arm-none-eabi/12.2.1/thumb/v8-m.main+fp/hard\libg_nano.a(libc_a-lock.o)
 .text.__retarget_lock_close_recursive
                0x00000000        0x2 c:/renesas/ra/e2studio_v2023-10_fsp_v5.0.0/toolchains/gcc_arm/12.2.mpacbti-rel1/bin/../lib/gcc/arm-none-eabi/12.2.1/thumb/v8-m.main+fp/hard\libg_nano.a(libc_a-lock.o)
 .text.__retarget_lock_acquire
                0x00000000        0x2 c:/renesas/ra/e2studio_v2023-10_fsp_v5.0.0/toolchains/gcc_arm/12.2.mpacbti-rel1/bin/../lib/gcc/arm-none-eabi/12.2.1/thumb/v8-m.main+fp/hard\libg_nano.a(libc_a-lock.o)
 .text.__retarget_lock_acquire_recursive
                0x00000000        0x2 c:/renesas/ra/e2studio_v2023-10_fsp_v5.0.0/toolchains/gcc_arm/12.2.mpacbti-rel1/bin/../lib/gcc/arm-none-eabi/12.2.1/thumb/v8-m.main+fp/hard\libg_nano.a(libc_a-lock.o)
 .text.__retarget_lock_try_acquire
                0x00000000        0x4 c:/renesas/ra/e2studio_v2023-10_fsp_v5.0.0/toolchains/gcc_arm/12.2.mpacbti-rel1/bin/../lib/gcc/arm-none-eabi/12.2.1/thumb/v8-m.main+fp/hard\libg_nano.a(libc_a-lock.o)
 .text.__retarget_lock_try_acquire_recursive
                0x00000000        0x4 c:/renesas/ra/e2studio_v2023-10_fsp_v5.0.0/toolchains/gcc_arm/12.2.mpacbti-rel1/bin/../lib/gcc/arm-none-eabi/12.2.1/thumb/v8-m.main+fp/hard\libg_nano.a(libc_a-lock.o)
 .text.__retarget_lock_release
                0x00000000        0x2 c:/renesas/ra/e2studio_v2023-10_fsp_v5.0.0/toolchains/gcc_arm/12.2.mpacbti-rel1/bin/../lib/gcc/arm-none-eabi/12.2.1/thumb/v8-m.main+fp/hard\libg_nano.a(libc_a-lock.o)
 .text.__retarget_lock_release_recursive
                0x00000000        0x2 c:/renesas/ra/e2studio_v2023-10_fsp_v5.0.0/toolchains/gcc_arm/12.2.mpacbti-rel1/bin/../lib/gcc/arm-none-eabi/12.2.1/thumb/v8-m.main+fp/hard\libg_nano.a(libc_a-lock.o)
 .bss.__lock___arc4random_mutex
                0x00000000        0x1 c:/renesas/ra/e2studio_v2023-10_fsp_v5.0.0/toolchains/gcc_arm/12.2.mpacbti-rel1/bin/../lib/gcc/arm-none-eabi/12.2.1/thumb/v8-m.main+fp/hard\libg_nano.a(libc_a-lock.o)
 .bss.__lock___dd_hash_mutex
                0x00000000        0x1 c:/renesas/ra/e2studio_v2023-10_fsp_v5.0.0/toolchains/gcc_arm/12.2.mpacbti-rel1/bin/../lib/gcc/arm-none-eabi/12.2.1/thumb/v8-m.main+fp/hard\libg_nano.a(libc_a-lock.o)
 .bss.__lock___tz_mutex
                0x00000000        0x1 c:/renesas/ra/e2studio_v2023-10_fsp_v5.0.0/toolchains/gcc_arm/12.2.mpacbti-rel1/bin/../lib/gcc/arm-none-eabi/12.2.1/thumb/v8-m.main+fp/hard\libg_nano.a(libc_a-lock.o)
 .bss.__lock___env_recursive_mutex
                0x00000000        0x1 c:/renesas/ra/e2studio_v2023-10_fsp_v5.0.0/toolchains/gcc_arm/12.2.mpacbti-rel1/bin/../lib/gcc/arm-none-eabi/12.2.1/thumb/v8-m.main+fp/hard\libg_nano.a(libc_a-lock.o)
 .bss.__lock___malloc_recursive_mutex
                0x00000000        0x1 c:/renesas/ra/e2studio_v2023-10_fsp_v5.0.0/toolchains/gcc_arm/12.2.mpacbti-rel1/bin/../lib/gcc/arm-none-eabi/12.2.1/thumb/v8-m.main+fp/hard\libg_nano.a(libc_a-lock.o)
 .bss.__lock___at_quick_exit_mutex
                0x00000000        0x1 c:/renesas/ra/e2studio_v2023-10_fsp_v5.0.0/toolchains/gcc_arm/12.2.mpacbti-rel1/bin/../lib/gcc/arm-none-eabi/12.2.1/thumb/v8-m.main+fp/hard\libg_nano.a(libc_a-lock.o)
 .bss.__lock___atexit_recursive_mutex
                0x00000000        0x1 c:/renesas/ra/e2studio_v2023-10_fsp_v5.0.0/toolchains/gcc_arm/12.2.mpacbti-rel1/bin/../lib/gcc/arm-none-eabi/12.2.1/thumb/v8-m.main+fp/hard\libg_nano.a(libc_a-lock.o)
 .bss.__lock___sfp_recursive_mutex
                0x00000000        0x1 c:/renesas/ra/e2studio_v2023-10_fsp_v5.0.0/toolchains/gcc_arm/12.2.mpacbti-rel1/bin/../lib/gcc/arm-none-eabi/12.2.1/thumb/v8-m.main+fp/hard\libg_nano.a(libc_a-lock.o)
 .debug_frame   0x00000000       0xb0 c:/renesas/ra/e2studio_v2023-10_fsp_v5.0.0/toolchains/gcc_arm/12.2.mpacbti-rel1/bin/../lib/gcc/arm-none-eabi/12.2.1/thumb/v8-m.main+fp/hard\libg_nano.a(libc_a-lock.o)
 .ARM.attributes
                0x00000000       0x38 c:/renesas/ra/e2studio_v2023-10_fsp_v5.0.0/toolchains/gcc_arm/12.2.mpacbti-rel1/bin/../lib/gcc/arm-none-eabi/12.2.1/thumb/v8-m.main+fp/hard\libg_nano.a(libc_a-lock.o)
 .text          0x00000000        0x0 c:/renesas/ra/e2studio_v2023-10_fsp_v5.0.0/toolchains/gcc_arm/12.2.mpacbti-rel1/bin/../lib/gcc/arm-none-eabi/12.2.1/thumb/v8-m.main+fp/hard\libg_nano.a(libc_a-strcpy.o)
 .data          0x00000000        0x0 c:/renesas/ra/e2studio_v2023-10_fsp_v5.0.0/toolchains/gcc_arm/12.2.mpacbti-rel1/bin/../lib/gcc/arm-none-eabi/12.2.1/thumb/v8-m.main+fp/hard\libg_nano.a(libc_a-strcpy.o)
 .bss           0x00000000        0x0 c:/renesas/ra/e2studio_v2023-10_fsp_v5.0.0/toolchains/gcc_arm/12.2.mpacbti-rel1/bin/../lib/gcc/arm-none-eabi/12.2.1/thumb/v8-m.main+fp/hard\libg_nano.a(libc_a-strcpy.o)
 .text          0x00000000        0x0 c:/renesas/ra/e2studio_v2023-10_fsp_v5.0.0/toolchains/gcc_arm/12.2.mpacbti-rel1/bin/../lib/gcc/arm-none-eabi/12.2.1/thumb/v8-m.main+fp/hard\libg_nano.a(libc_a-aeabi_memcpy.o)
 .data          0x00000000        0x0 c:/renesas/ra/e2studio_v2023-10_fsp_v5.0.0/toolchains/gcc_arm/12.2.mpacbti-rel1/bin/../lib/gcc/arm-none-eabi/12.2.1/thumb/v8-m.main+fp/hard\libg_nano.a(libc_a-aeabi_memcpy.o)
 .bss           0x00000000        0x0 c:/renesas/ra/e2studio_v2023-10_fsp_v5.0.0/toolchains/gcc_arm/12.2.mpacbti-rel1/bin/../lib/gcc/arm-none-eabi/12.2.1/thumb/v8-m.main+fp/hard\libg_nano.a(libc_a-aeabi_memcpy.o)
 .text          0x00000000        0x0 c:/renesas/ra/e2studio_v2023-10_fsp_v5.0.0/toolchains/gcc_arm/12.2.mpacbti-rel1/bin/../lib/gcc/arm-none-eabi/12.2.1/thumb/v8-m.main+fp/hard\libg_nano.a(libc_a-aeabi_memclr.o)
 .data          0x00000000        0x0 c:/renesas/ra/e2studio_v2023-10_fsp_v5.0.0/toolchains/gcc_arm/12.2.mpacbti-rel1/bin/../lib/gcc/arm-none-eabi/12.2.1/thumb/v8-m.main+fp/hard\libg_nano.a(libc_a-aeabi_memclr.o)
 .bss           0x00000000        0x0 c:/renesas/ra/e2studio_v2023-10_fsp_v5.0.0/toolchains/gcc_arm/12.2.mpacbti-rel1/bin/../lib/gcc/arm-none-eabi/12.2.1/thumb/v8-m.main+fp/hard\libg_nano.a(libc_a-aeabi_memclr.o)
 .text          0x00000000        0x0 c:/renesas/ra/e2studio_v2023-10_fsp_v5.0.0/toolchains/gcc_arm/12.2.mpacbti-rel1/bin/../lib/gcc/arm-none-eabi/12.2.1/thumb/v8-m.main+fp/hard\libg_nano.a(libc_a-memcpy-stub.o)
 .data          0x00000000        0x0 c:/renesas/ra/e2studio_v2023-10_fsp_v5.0.0/toolchains/gcc_arm/12.2.mpacbti-rel1/bin/../lib/gcc/arm-none-eabi/12.2.1/thumb/v8-m.main+fp/hard\libg_nano.a(libc_a-memcpy-stub.o)
 .bss           0x00000000        0x0 c:/renesas/ra/e2studio_v2023-10_fsp_v5.0.0/toolchains/gcc_arm/12.2.mpacbti-rel1/bin/../lib/gcc/arm-none-eabi/12.2.1/thumb/v8-m.main+fp/hard\libg_nano.a(libc_a-memcpy-stub.o)
 .data          0x00000000        0x0 c:/renesas/ra/e2studio_v2023-10_fsp_v5.0.0/toolchains/gcc_arm/12.2.mpacbti-rel1/bin/../lib/gcc/arm-none-eabi/12.2.1/thumb/v8-m.main+fp/hard\libg_nano.a(libc_a-strlen.o)
 .bss           0x00000000        0x0 c:/renesas/ra/e2studio_v2023-10_fsp_v5.0.0/toolchains/gcc_arm/12.2.mpacbti-rel1/bin/../lib/gcc/arm-none-eabi/12.2.1/thumb/v8-m.main+fp/hard\libg_nano.a(libc_a-strlen.o)
 .ARM.extab     0x00000000        0x0 c:/renesas/ra/e2studio_v2023-10_fsp_v5.0.0/toolchains/gcc_arm/12.2.mpacbti-rel1/bin/../lib/gcc/arm-none-eabi/12.2.1/thumb/v8-m.main+fp/hard\libg_nano.a(libc_a-strlen.o)
 .ARM.exidx     0x00000000        0x8 c:/renesas/ra/e2studio_v2023-10_fsp_v5.0.0/toolchains/gcc_arm/12.2.mpacbti-rel1/bin/../lib/gcc/arm-none-eabi/12.2.1/thumb/v8-m.main+fp/hard\libg_nano.a(libc_a-strlen.o)
 .text          0x00000000        0x0 c:/renesas/ra/e2studio_v2023-10_fsp_v5.0.0/toolchains/gcc_arm/12.2.mpacbti-rel1/bin/../lib/gcc/arm-none-eabi/12.2.1/thumb/v8-m.main+fp/hard\libg_nano.a(libc_a-freer.o)
 .data          0x00000000        0x0 c:/renesas/ra/e2studio_v2023-10_fsp_v5.0.0/toolchains/gcc_arm/12.2.mpacbti-rel1/bin/../lib/gcc/arm-none-eabi/12.2.1/thumb/v8-m.main+fp/hard\libg_nano.a(libc_a-freer.o)
 .bss           0x00000000        0x0 c:/renesas/ra/e2studio_v2023-10_fsp_v5.0.0/toolchains/gcc_arm/12.2.mpacbti-rel1/bin/../lib/gcc/arm-none-eabi/12.2.1/thumb/v8-m.main+fp/hard\libg_nano.a(libc_a-freer.o)
 .text._free_r  0x00000000       0x94 c:/renesas/ra/e2studio_v2023-10_fsp_v5.0.0/toolchains/gcc_arm/12.2.mpacbti-rel1/bin/../lib/gcc/arm-none-eabi/12.2.1/thumb/v8-m.main+fp/hard\libg_nano.a(libc_a-freer.o)
 .debug_frame   0x00000000       0x38 c:/renesas/ra/e2studio_v2023-10_fsp_v5.0.0/toolchains/gcc_arm/12.2.mpacbti-rel1/bin/../lib/gcc/arm-none-eabi/12.2.1/thumb/v8-m.main+fp/hard\libg_nano.a(libc_a-freer.o)
 .ARM.attributes
                0x00000000       0x38 c:/renesas/ra/e2studio_v2023-10_fsp_v5.0.0/toolchains/gcc_arm/12.2.mpacbti-rel1/bin/../lib/gcc/arm-none-eabi/12.2.1/thumb/v8-m.main+fp/hard\libg_nano.a(libc_a-freer.o)
 .text          0x00000000        0x0 c:/renesas/ra/e2studio_v2023-10_fsp_v5.0.0/toolchains/gcc_arm/12.2.mpacbti-rel1/bin/../lib/gcc/arm-none-eabi/12.2.1/thumb/v8-m.main+fp/hard\libg_nano.a(libc_a-mallocr.o)
 .data          0x00000000        0x0 c:/renesas/ra/e2studio_v2023-10_fsp_v5.0.0/toolchains/gcc_arm/12.2.mpacbti-rel1/bin/../lib/gcc/arm-none-eabi/12.2.1/thumb/v8-m.main+fp/hard\libg_nano.a(libc_a-mallocr.o)
 .bss           0x00000000        0x0 c:/renesas/ra/e2studio_v2023-10_fsp_v5.0.0/toolchains/gcc_arm/12.2.mpacbti-rel1/bin/../lib/gcc/arm-none-eabi/12.2.1/thumb/v8-m.main+fp/hard\libg_nano.a(libc_a-mallocr.o)
 .text.sbrk_aligned
                0x00000000       0x44 c:/renesas/ra/e2studio_v2023-10_fsp_v5.0.0/toolchains/gcc_arm/12.2.mpacbti-rel1/bin/../lib/gcc/arm-none-eabi/12.2.1/thumb/v8-m.main+fp/hard\libg_nano.a(libc_a-mallocr.o)
 .text._malloc_r
                0x00000000      0x100 c:/renesas/ra/e2studio_v2023-10_fsp_v5.0.0/toolchains/gcc_arm/12.2.mpacbti-rel1/bin/../lib/gcc/arm-none-eabi/12.2.1/thumb/v8-m.main+fp/hard\libg_nano.a(libc_a-mallocr.o)
 .bss.__malloc_sbrk_start
                0x00000000        0x4 c:/renesas/ra/e2studio_v2023-10_fsp_v5.0.0/toolchains/gcc_arm/12.2.mpacbti-rel1/bin/../lib/gcc/arm-none-eabi/12.2.1/thumb/v8-m.main+fp/hard\libg_nano.a(libc_a-mallocr.o)
 .bss.__malloc_free_list
                0x00000000        0x4 c:/renesas/ra/e2studio_v2023-10_fsp_v5.0.0/toolchains/gcc_arm/12.2.mpacbti-rel1/bin/../lib/gcc/arm-none-eabi/12.2.1/thumb/v8-m.main+fp/hard\libg_nano.a(libc_a-mallocr.o)
 .debug_frame   0x00000000       0x50 c:/renesas/ra/e2studio_v2023-10_fsp_v5.0.0/toolchains/gcc_arm/12.2.mpacbti-rel1/bin/../lib/gcc/arm-none-eabi/12.2.1/thumb/v8-m.main+fp/hard\libg_nano.a(libc_a-mallocr.o)
 .ARM.attributes
                0x00000000       0x38 c:/renesas/ra/e2studio_v2023-10_fsp_v5.0.0/toolchains/gcc_arm/12.2.mpacbti-rel1/bin/../lib/gcc/arm-none-eabi/12.2.1/thumb/v8-m.main+fp/hard\libg_nano.a(libc_a-mallocr.o)
 .text          0x00000000        0x0 c:/renesas/ra/e2studio_v2023-10_fsp_v5.0.0/toolchains/gcc_arm/12.2.mpacbti-rel1/bin/../lib/gcc/arm-none-eabi/12.2.1/thumb/v8-m.main+fp/hard\libg_nano.a(libc_a-mlock.o)
 .data          0x00000000        0x0 c:/renesas/ra/e2studio_v2023-10_fsp_v5.0.0/toolchains/gcc_arm/12.2.mpacbti-rel1/bin/../lib/gcc/arm-none-eabi/12.2.1/thumb/v8-m.main+fp/hard\libg_nano.a(libc_a-mlock.o)
 .bss           0x00000000        0x0 c:/renesas/ra/e2studio_v2023-10_fsp_v5.0.0/toolchains/gcc_arm/12.2.mpacbti-rel1/bin/../lib/gcc/arm-none-eabi/12.2.1/thumb/v8-m.main+fp/hard\libg_nano.a(libc_a-mlock.o)
 .text.__malloc_lock
                0x00000000        0xc c:/renesas/ra/e2studio_v2023-10_fsp_v5.0.0/toolchains/gcc_arm/12.2.mpacbti-rel1/bin/../lib/gcc/arm-none-eabi/12.2.1/thumb/v8-m.main+fp/hard\libg_nano.a(libc_a-mlock.o)
 .text.__malloc_unlock
                0x00000000        0xc c:/renesas/ra/e2studio_v2023-10_fsp_v5.0.0/toolchains/gcc_arm/12.2.mpacbti-rel1/bin/../lib/gcc/arm-none-eabi/12.2.1/thumb/v8-m.main+fp/hard\libg_nano.a(libc_a-mlock.o)
 .debug_frame   0x00000000       0x30 c:/renesas/ra/e2studio_v2023-10_fsp_v5.0.0/toolchains/gcc_arm/12.2.mpacbti-rel1/bin/../lib/gcc/arm-none-eabi/12.2.1/thumb/v8-m.main+fp/hard\libg_nano.a(libc_a-mlock.o)
 .ARM.attributes
                0x00000000       0x38 c:/renesas/ra/e2studio_v2023-10_fsp_v5.0.0/toolchains/gcc_arm/12.2.mpacbti-rel1/bin/../lib/gcc/arm-none-eabi/12.2.1/thumb/v8-m.main+fp/hard\libg_nano.a(libc_a-mlock.o)
 .text          0x00000000        0x0 c:/renesas/ra/e2studio_v2023-10_fsp_v5.0.0/toolchains/gcc_arm/12.2.mpacbti-rel1/bin/../lib/gcc/arm-none-eabi/12.2.1/thumb/v8-m.main+fp/hard\libg_nano.a(libc_a-fflush.o)
 .data          0x00000000        0x0 c:/renesas/ra/e2studio_v2023-10_fsp_v5.0.0/toolchains/gcc_arm/12.2.mpacbti-rel1/bin/../lib/gcc/arm-none-eabi/12.2.1/thumb/v8-m.main+fp/hard\libg_nano.a(libc_a-fflush.o)
 .bss           0x00000000        0x0 c:/renesas/ra/e2studio_v2023-10_fsp_v5.0.0/toolchains/gcc_arm/12.2.mpacbti-rel1/bin/../lib/gcc/arm-none-eabi/12.2.1/thumb/v8-m.main+fp/hard\libg_nano.a(libc_a-fflush.o)
 .text.__sflush_r
                0x00000000      0x106 c:/renesas/ra/e2studio_v2023-10_fsp_v5.0.0/toolchains/gcc_arm/12.2.mpacbti-rel1/bin/../lib/gcc/arm-none-eabi/12.2.1/thumb/v8-m.main+fp/hard\libg_nano.a(libc_a-fflush.o)
 .text._fflush_r
                0x00000000       0x50 c:/renesas/ra/e2studio_v2023-10_fsp_v5.0.0/toolchains/gcc_arm/12.2.mpacbti-rel1/bin/../lib/gcc/arm-none-eabi/12.2.1/thumb/v8-m.main+fp/hard\libg_nano.a(libc_a-fflush.o)
 .text.fflush   0x00000000       0x28 c:/renesas/ra/e2studio_v2023-10_fsp_v5.0.0/toolchains/gcc_arm/12.2.mpacbti-rel1/bin/../lib/gcc/arm-none-eabi/12.2.1/thumb/v8-m.main+fp/hard\libg_nano.a(libc_a-fflush.o)
 .debug_frame   0x00000000       0x5c c:/renesas/ra/e2studio_v2023-10_fsp_v5.0.0/toolchains/gcc_arm/12.2.mpacbti-rel1/bin/../lib/gcc/arm-none-eabi/12.2.1/thumb/v8-m.main+fp/hard\libg_nano.a(libc_a-fflush.o)
 .ARM.attributes
                0x00000000       0x38 c:/renesas/ra/e2studio_v2023-10_fsp_v5.0.0/toolchains/gcc_arm/12.2.mpacbti-rel1/bin/../lib/gcc/arm-none-eabi/12.2.1/thumb/v8-m.main+fp/hard\libg_nano.a(libc_a-fflush.o)
 .text          0x00000000        0x0 c:/renesas/ra/e2studio_v2023-10_fsp_v5.0.0/toolchains/gcc_arm/12.2.mpacbti-rel1/bin/../lib/gcc/arm-none-eabi/12.2.1/thumb/v8-m.main+fp/hard\libg_nano.a(libc_a-sbrkr.o)
 .data          0x00000000        0x0 c:/renesas/ra/e2studio_v2023-10_fsp_v5.0.0/toolchains/gcc_arm/12.2.mpacbti-rel1/bin/../lib/gcc/arm-none-eabi/12.2.1/thumb/v8-m.main+fp/hard\libg_nano.a(libc_a-sbrkr.o)
 .bss           0x00000000        0x0 c:/renesas/ra/e2studio_v2023-10_fsp_v5.0.0/toolchains/gcc_arm/12.2.mpacbti-rel1/bin/../lib/gcc/arm-none-eabi/12.2.1/thumb/v8-m.main+fp/hard\libg_nano.a(libc_a-sbrkr.o)
 .text._sbrk_r  0x00000000       0x20 c:/renesas/ra/e2studio_v2023-10_fsp_v5.0.0/toolchains/gcc_arm/12.2.mpacbti-rel1/bin/../lib/gcc/arm-none-eabi/12.2.1/thumb/v8-m.main+fp/hard\libg_nano.a(libc_a-sbrkr.o)
 .debug_frame   0x00000000       0x2c c:/renesas/ra/e2studio_v2023-10_fsp_v5.0.0/toolchains/gcc_arm/12.2.mpacbti-rel1/bin/../lib/gcc/arm-none-eabi/12.2.1/thumb/v8-m.main+fp/hard\libg_nano.a(libc_a-sbrkr.o)
 .ARM.attributes
                0x00000000       0x38 c:/renesas/ra/e2studio_v2023-10_fsp_v5.0.0/toolchains/gcc_arm/12.2.mpacbti-rel1/bin/../lib/gcc/arm-none-eabi/12.2.1/thumb/v8-m.main+fp/hard\libg_nano.a(libc_a-sbrkr.o)
 .data          0x00000000        0x0 c:/renesas/ra/e2studio_v2023-10_fsp_v5.0.0/toolchains/gcc_arm/12.2.mpacbti-rel1/bin/../lib/gcc/arm-none-eabi/12.2.1/thumb/v8-m.main+fp/hard\libg_nano.a(libc_a-aeabi_memset-soft.o)
 .bss           0x00000000        0x0 c:/renesas/ra/e2studio_v2023-10_fsp_v5.0.0/toolchains/gcc_arm/12.2.mpacbti-rel1/bin/../lib/gcc/arm-none-eabi/12.2.1/thumb/v8-m.main+fp/hard\libg_nano.a(libc_a-aeabi_memset-soft.o)
 .ARM.extab     0x00000000        0x0 c:/renesas/ra/e2studio_v2023-10_fsp_v5.0.0/toolchains/gcc_arm/12.2.mpacbti-rel1/bin/../lib/gcc/arm-none-eabi/12.2.1/thumb/v8-m.main+fp/hard\libg_nano.a(libc_a-aeabi_memset-soft.o)
 .ARM.exidx     0x00000000        0x8 c:/renesas/ra/e2studio_v2023-10_fsp_v5.0.0/toolchains/gcc_arm/12.2.mpacbti-rel1/bin/../lib/gcc/arm-none-eabi/12.2.1/thumb/v8-m.main+fp/hard\libg_nano.a(libc_a-aeabi_memset-soft.o)
 .text          0x00000000        0x0 c:/renesas/ra/e2studio_v2023-10_fsp_v5.0.0/toolchains/gcc_arm/12.2.mpacbti-rel1/bin/../lib/gcc/arm-none-eabi/12.2.1/thumb/v8-m.main+fp/hard\librdimon_nano.a(arm_librdimon_a-_exit.o)
 .data          0x00000000        0x0 c:/renesas/ra/e2studio_v2023-10_fsp_v5.0.0/toolchains/gcc_arm/12.2.mpacbti-rel1/bin/../lib/gcc/arm-none-eabi/12.2.1/thumb/v8-m.main+fp/hard\librdimon_nano.a(arm_librdimon_a-_exit.o)
 .bss           0x00000000        0x0 c:/renesas/ra/e2studio_v2023-10_fsp_v5.0.0/toolchains/gcc_arm/12.2.mpacbti-rel1/bin/../lib/gcc/arm-none-eabi/12.2.1/thumb/v8-m.main+fp/hard\librdimon_nano.a(arm_librdimon_a-_exit.o)
 .text._exit    0x00000000       0x14 c:/renesas/ra/e2studio_v2023-10_fsp_v5.0.0/toolchains/gcc_arm/12.2.mpacbti-rel1/bin/../lib/gcc/arm-none-eabi/12.2.1/thumb/v8-m.main+fp/hard\librdimon_nano.a(arm_librdimon_a-_exit.o)
 .debug_frame   0x00000000       0x28 c:/renesas/ra/e2studio_v2023-10_fsp_v5.0.0/toolchains/gcc_arm/12.2.mpacbti-rel1/bin/../lib/gcc/arm-none-eabi/12.2.1/thumb/v8-m.main+fp/hard\librdimon_nano.a(arm_librdimon_a-_exit.o)
 .ARM.attributes
                0x00000000       0x38 c:/renesas/ra/e2studio_v2023-10_fsp_v5.0.0/toolchains/gcc_arm/12.2.mpacbti-rel1/bin/../lib/gcc/arm-none-eabi/12.2.1/thumb/v8-m.main+fp/hard\librdimon_nano.a(arm_librdimon_a-_exit.o)
 .text          0x00000000        0x0 c:/renesas/ra/e2studio_v2023-10_fsp_v5.0.0/toolchains/gcc_arm/12.2.mpacbti-rel1/bin/../lib/gcc/arm-none-eabi/12.2.1/thumb/v8-m.main+fp/hard\librdimon_nano.a(arm_librdimon_a-_kill.o)
 .data          0x00000000        0x0 c:/renesas/ra/e2studio_v2023-10_fsp_v5.0.0/toolchains/gcc_arm/12.2.mpacbti-rel1/bin/../lib/gcc/arm-none-eabi/12.2.1/thumb/v8-m.main+fp/hard\librdimon_nano.a(arm_librdimon_a-_kill.o)
 .bss           0x00000000        0x0 c:/renesas/ra/e2studio_v2023-10_fsp_v5.0.0/toolchains/gcc_arm/12.2.mpacbti-rel1/bin/../lib/gcc/arm-none-eabi/12.2.1/thumb/v8-m.main+fp/hard\librdimon_nano.a(arm_librdimon_a-_kill.o)
 .text._kill_shared
                0x00000000       0x26 c:/renesas/ra/e2studio_v2023-10_fsp_v5.0.0/toolchains/gcc_arm/12.2.mpacbti-rel1/bin/../lib/gcc/arm-none-eabi/12.2.1/thumb/v8-m.main+fp/hard\librdimon_nano.a(arm_librdimon_a-_kill.o)
 .text._kill    0x00000000       0x18 c:/renesas/ra/e2studio_v2023-10_fsp_v5.0.0/toolchains/gcc_arm/12.2.mpacbti-rel1/bin/../lib/gcc/arm-none-eabi/12.2.1/thumb/v8-m.main+fp/hard\librdimon_nano.a(arm_librdimon_a-_kill.o)
 .debug_frame   0x00000000       0x40 c:/renesas/ra/e2studio_v2023-10_fsp_v5.0.0/toolchains/gcc_arm/12.2.mpacbti-rel1/bin/../lib/gcc/arm-none-eabi/12.2.1/thumb/v8-m.main+fp/hard\librdimon_nano.a(arm_librdimon_a-_kill.o)
 .ARM.attributes
                0x00000000       0x38 c:/renesas/ra/e2studio_v2023-10_fsp_v5.0.0/toolchains/gcc_arm/12.2.mpacbti-rel1/bin/../lib/gcc/arm-none-eabi/12.2.1/thumb/v8-m.main+fp/hard\librdimon_nano.a(arm_librdimon_a-_kill.o)
 .text          0x00000000        0x0 c:/renesas/ra/e2studio_v2023-10_fsp_v5.0.0/toolchains/gcc_arm/12.2.mpacbti-rel1/bin/../lib/gcc/arm-none-eabi/12.2.1/thumb/v8-m.main+fp/hard\librdimon_nano.a(arm_librdimon_a-syscalls.o)
 .data          0x00000000        0x0 c:/renesas/ra/e2studio_v2023-10_fsp_v5.0.0/toolchains/gcc_arm/12.2.mpacbti-rel1/bin/../lib/gcc/arm-none-eabi/12.2.1/thumb/v8-m.main+fp/hard\librdimon_nano.a(arm_librdimon_a-syscalls.o)
 .bss           0x00000000        0x0 c:/renesas/ra/e2studio_v2023-10_fsp_v5.0.0/toolchains/gcc_arm/12.2.mpacbti-rel1/bin/../lib/gcc/arm-none-eabi/12.2.1/thumb/v8-m.main+fp/hard\librdimon_nano.a(arm_librdimon_a-syscalls.o)
 .text.findslot
                0x00000000       0x34 c:/renesas/ra/e2studio_v2023-10_fsp_v5.0.0/toolchains/gcc_arm/12.2.mpacbti-rel1/bin/../lib/gcc/arm-none-eabi/12.2.1/thumb/v8-m.main+fp/hard\librdimon_nano.a(arm_librdimon_a-syscalls.o)
 .text.error    0x00000000       0x1c c:/renesas/ra/e2studio_v2023-10_fsp_v5.0.0/toolchains/gcc_arm/12.2.mpacbti-rel1/bin/../lib/gcc/arm-none-eabi/12.2.1/thumb/v8-m.main+fp/hard\librdimon_nano.a(arm_librdimon_a-syscalls.o)
 .text.checkerror
                0x00000000        0xa c:/renesas/ra/e2studio_v2023-10_fsp_v5.0.0/toolchains/gcc_arm/12.2.mpacbti-rel1/bin/../lib/gcc/arm-none-eabi/12.2.1/thumb/v8-m.main+fp/hard\librdimon_nano.a(arm_librdimon_a-syscalls.o)
 .text._swiread
                0x00000000       0x20 c:/renesas/ra/e2studio_v2023-10_fsp_v5.0.0/toolchains/gcc_arm/12.2.mpacbti-rel1/bin/../lib/gcc/arm-none-eabi/12.2.1/thumb/v8-m.main+fp/hard\librdimon_nano.a(arm_librdimon_a-syscalls.o)
 .text._read    0x00000000       0x34 c:/renesas/ra/e2studio_v2023-10_fsp_v5.0.0/toolchains/gcc_arm/12.2.mpacbti-rel1/bin/../lib/gcc/arm-none-eabi/12.2.1/thumb/v8-m.main+fp/hard\librdimon_nano.a(arm_librdimon_a-syscalls.o)
 .text._swilseek
                0x00000000       0x78 c:/renesas/ra/e2studio_v2023-10_fsp_v5.0.0/toolchains/gcc_arm/12.2.mpacbti-rel1/bin/../lib/gcc/arm-none-eabi/12.2.1/thumb/v8-m.main+fp/hard\librdimon_nano.a(arm_librdimon_a-syscalls.o)
 .text._lseek   0x00000000        0x4 c:/renesas/ra/e2studio_v2023-10_fsp_v5.0.0/toolchains/gcc_arm/12.2.mpacbti-rel1/bin/../lib/gcc/arm-none-eabi/12.2.1/thumb/v8-m.main+fp/hard\librdimon_nano.a(arm_librdimon_a-syscalls.o)
 .text._swiwrite
                0x00000000       0x20 c:/renesas/ra/e2studio_v2023-10_fsp_v5.0.0/toolchains/gcc_arm/12.2.mpacbti-rel1/bin/../lib/gcc/arm-none-eabi/12.2.1/thumb/v8-m.main+fp/hard\librdimon_nano.a(arm_librdimon_a-syscalls.o)
 .text._write   0x00000000       0x40 c:/renesas/ra/e2studio_v2023-10_fsp_v5.0.0/toolchains/gcc_arm/12.2.mpacbti-rel1/bin/../lib/gcc/arm-none-eabi/12.2.1/thumb/v8-m.main+fp/hard\librdimon_nano.a(arm_librdimon_a-syscalls.o)
 .text._swiclose
                0x00000000       0x1a c:/renesas/ra/e2studio_v2023-10_fsp_v5.0.0/toolchains/gcc_arm/12.2.mpacbti-rel1/bin/../lib/gcc/arm-none-eabi/12.2.1/thumb/v8-m.main+fp/hard\librdimon_nano.a(arm_librdimon_a-syscalls.o)
 .text._close   0x00000000       0x44 c:/renesas/ra/e2studio_v2023-10_fsp_v5.0.0/toolchains/gcc_arm/12.2.mpacbti-rel1/bin/../lib/gcc/arm-none-eabi/12.2.1/thumb/v8-m.main+fp/hard\librdimon_nano.a(arm_librdimon_a-syscalls.o)
 .text._getpid  0x00000000        0x4 c:/renesas/ra/e2studio_v2023-10_fsp_v5.0.0/toolchains/gcc_arm/12.2.mpacbti-rel1/bin/../lib/gcc/arm-none-eabi/12.2.1/thumb/v8-m.main+fp/hard\librdimon_nano.a(arm_librdimon_a-syscalls.o)
 .text._sbrk    0x00000000       0x48 c:/renesas/ra/e2studio_v2023-10_fsp_v5.0.0/toolchains/gcc_arm/12.2.mpacbti-rel1/bin/../lib/gcc/arm-none-eabi/12.2.1/thumb/v8-m.main+fp/hard\librdimon_nano.a(arm_librdimon_a-syscalls.o)
 .text._swistat
                0x00000000       0x42 c:/renesas/ra/e2studio_v2023-10_fsp_v5.0.0/toolchains/gcc_arm/12.2.mpacbti-rel1/bin/../lib/gcc/arm-none-eabi/12.2.1/thumb/v8-m.main+fp/hard\librdimon_nano.a(arm_librdimon_a-syscalls.o)
 .text._fstat   0x00000000       0x1c c:/renesas/ra/e2studio_v2023-10_fsp_v5.0.0/toolchains/gcc_arm/12.2.mpacbti-rel1/bin/../lib/gcc/arm-none-eabi/12.2.1/thumb/v8-m.main+fp/hard\librdimon_nano.a(arm_librdimon_a-syscalls.o)
 .text._stat    0x00000000       0x3a c:/renesas/ra/e2studio_v2023-10_fsp_v5.0.0/toolchains/gcc_arm/12.2.mpacbti-rel1/bin/../lib/gcc/arm-none-eabi/12.2.1/thumb/v8-m.main+fp/hard\librdimon_nano.a(arm_librdimon_a-syscalls.o)
 .text._swiopen
                0x00000000       0xb0 c:/renesas/ra/e2studio_v2023-10_fsp_v5.0.0/toolchains/gcc_arm/12.2.mpacbti-rel1/bin/../lib/gcc/arm-none-eabi/12.2.1/thumb/v8-m.main+fp/hard\librdimon_nano.a(arm_librdimon_a-syscalls.o)
 .text._open    0x00000000       0x12 c:/renesas/ra/e2studio_v2023-10_fsp_v5.0.0/toolchains/gcc_arm/12.2.mpacbti-rel1/bin/../lib/gcc/arm-none-eabi/12.2.1/thumb/v8-m.main+fp/hard\librdimon_nano.a(arm_librdimon_a-syscalls.o)
 .rodata._get_semihosting_exts.str1.1
                0x00000000       0x16 c:/renesas/ra/e2studio_v2023-10_fsp_v5.0.0/toolchains/gcc_arm/12.2.mpacbti-rel1/bin/../lib/gcc/arm-none-eabi/12.2.1/thumb/v8-m.main+fp/hard\librdimon_nano.a(arm_librdimon_a-syscalls.o)
 .text._get_semihosting_exts
                0x00000000       0xb4 c:/renesas/ra/e2studio_v2023-10_fsp_v5.0.0/toolchains/gcc_arm/12.2.mpacbti-rel1/bin/../lib/gcc/arm-none-eabi/12.2.1/thumb/v8-m.main+fp/hard\librdimon_nano.a(arm_librdimon_a-syscalls.o)
 .text.initialise_semihosting_exts
                0x00000000       0x34 c:/renesas/ra/e2studio_v2023-10_fsp_v5.0.0/toolchains/gcc_arm/12.2.mpacbti-rel1/bin/../lib/gcc/arm-none-eabi/12.2.1/thumb/v8-m.main+fp/hard\librdimon_nano.a(arm_librdimon_a-syscalls.o)
 .text._has_ext_exit_extended
                0x00000000       0x18 c:/renesas/ra/e2studio_v2023-10_fsp_v5.0.0/toolchains/gcc_arm/12.2.mpacbti-rel1/bin/../lib/gcc/arm-none-eabi/12.2.1/thumb/v8-m.main+fp/hard\librdimon_nano.a(arm_librdimon_a-syscalls.o)
 .text._has_ext_stdout_stderr
                0x00000000       0x18 c:/renesas/ra/e2studio_v2023-10_fsp_v5.0.0/toolchains/gcc_arm/12.2.mpacbti-rel1/bin/../lib/gcc/arm-none-eabi/12.2.1/thumb/v8-m.main+fp/hard\librdimon_nano.a(arm_librdimon_a-syscalls.o)
 .rodata.initialise_monitor_handles.str1.1
                0x00000000        0x4 c:/renesas/ra/e2studio_v2023-10_fsp_v5.0.0/toolchains/gcc_arm/12.2.mpacbti-rel1/bin/../lib/gcc/arm-none-eabi/12.2.1/thumb/v8-m.main+fp/hard\librdimon_nano.a(arm_librdimon_a-syscalls.o)
 .text.initialise_monitor_handles
                0x00000000       0xc0 c:/renesas/ra/e2studio_v2023-10_fsp_v5.0.0/toolchains/gcc_arm/12.2.mpacbti-rel1/bin/../lib/gcc/arm-none-eabi/12.2.1/thumb/v8-m.main+fp/hard\librdimon_nano.a(arm_librdimon_a-syscalls.o)
 .text._link    0x00000000       0x10 c:/renesas/ra/e2studio_v2023-10_fsp_v5.0.0/toolchains/gcc_arm/12.2.mpacbti-rel1/bin/../lib/gcc/arm-none-eabi/12.2.1/thumb/v8-m.main+fp/hard\librdimon_nano.a(arm_librdimon_a-syscalls.o)
 .text._unlink  0x00000000       0x28 c:/renesas/ra/e2studio_v2023-10_fsp_v5.0.0/toolchains/gcc_arm/12.2.mpacbti-rel1/bin/../lib/gcc/arm-none-eabi/12.2.1/thumb/v8-m.main+fp/hard\librdimon_nano.a(arm_librdimon_a-syscalls.o)
 .text._gettimeofday
                0x00000000       0x28 c:/renesas/ra/e2studio_v2023-10_fsp_v5.0.0/toolchains/gcc_arm/12.2.mpacbti-rel1/bin/../lib/gcc/arm-none-eabi/12.2.1/thumb/v8-m.main+fp/hard\librdimon_nano.a(arm_librdimon_a-syscalls.o)
 .text._clock   0x00000000       0x12 c:/renesas/ra/e2studio_v2023-10_fsp_v5.0.0/toolchains/gcc_arm/12.2.mpacbti-rel1/bin/../lib/gcc/arm-none-eabi/12.2.1/thumb/v8-m.main+fp/hard\librdimon_nano.a(arm_librdimon_a-syscalls.o)
 .text._times   0x00000000       0x16 c:/renesas/ra/e2studio_v2023-10_fsp_v5.0.0/toolchains/gcc_arm/12.2.mpacbti-rel1/bin/../lib/gcc/arm-none-eabi/12.2.1/thumb/v8-m.main+fp/hard\librdimon_nano.a(arm_librdimon_a-syscalls.o)
 .text._isatty  0x00000000       0x3a c:/renesas/ra/e2studio_v2023-10_fsp_v5.0.0/toolchains/gcc_arm/12.2.mpacbti-rel1/bin/../lib/gcc/arm-none-eabi/12.2.1/thumb/v8-m.main+fp/hard\librdimon_nano.a(arm_librdimon_a-syscalls.o)
 .text._system  0x00000000       0x3c c:/renesas/ra/e2studio_v2023-10_fsp_v5.0.0/toolchains/gcc_arm/12.2.mpacbti-rel1/bin/../lib/gcc/arm-none-eabi/12.2.1/thumb/v8-m.main+fp/hard\librdimon_nano.a(arm_librdimon_a-syscalls.o)
 .text._rename  0x00000000       0x36 c:/renesas/ra/e2studio_v2023-10_fsp_v5.0.0/toolchains/gcc_arm/12.2.mpacbti-rel1/bin/../lib/gcc/arm-none-eabi/12.2.1/thumb/v8-m.main+fp/hard\librdimon_nano.a(arm_librdimon_a-syscalls.o)
 .bss.heap_end.0
                0x00000000        0x4 c:/renesas/ra/e2studio_v2023-10_fsp_v5.0.0/toolchains/gcc_arm/12.2.mpacbti-rel1/bin/../lib/gcc/arm-none-eabi/12.2.1/thumb/v8-m.main+fp/hard\librdimon_nano.a(arm_librdimon_a-syscalls.o)
 .data.__heap_limit
                0x00000000        0x4 c:/renesas/ra/e2studio_v2023-10_fsp_v5.0.0/toolchains/gcc_arm/12.2.mpacbti-rel1/bin/../lib/gcc/arm-none-eabi/12.2.1/thumb/v8-m.main+fp/hard\librdimon_nano.a(arm_librdimon_a-syscalls.o)
 .data.supports_ext_stdout_stderr
                0x00000000        0x4 c:/renesas/ra/e2studio_v2023-10_fsp_v5.0.0/toolchains/gcc_arm/12.2.mpacbti-rel1/bin/../lib/gcc/arm-none-eabi/12.2.1/thumb/v8-m.main+fp/hard\librdimon_nano.a(arm_librdimon_a-syscalls.o)
 .data.supports_ext_exit_extended
                0x00000000        0x4 c:/renesas/ra/e2studio_v2023-10_fsp_v5.0.0/toolchains/gcc_arm/12.2.mpacbti-rel1/bin/../lib/gcc/arm-none-eabi/12.2.1/thumb/v8-m.main+fp/hard\librdimon_nano.a(arm_librdimon_a-syscalls.o)
 .bss.monitor_stderr
                0x00000000        0x4 c:/renesas/ra/e2studio_v2023-10_fsp_v5.0.0/toolchains/gcc_arm/12.2.mpacbti-rel1/bin/../lib/gcc/arm-none-eabi/12.2.1/thumb/v8-m.main+fp/hard\librdimon_nano.a(arm_librdimon_a-syscalls.o)
 .bss.monitor_stdout
                0x00000000        0x4 c:/renesas/ra/e2studio_v2023-10_fsp_v5.0.0/toolchains/gcc_arm/12.2.mpacbti-rel1/bin/../lib/gcc/arm-none-eabi/12.2.1/thumb/v8-m.main+fp/hard\librdimon_nano.a(arm_librdimon_a-syscalls.o)
 .bss.monitor_stdin
                0x00000000        0x4 c:/renesas/ra/e2studio_v2023-10_fsp_v5.0.0/toolchains/gcc_arm/12.2.mpacbti-rel1/bin/../lib/gcc/arm-none-eabi/12.2.1/thumb/v8-m.main+fp/hard\librdimon_nano.a(arm_librdimon_a-syscalls.o)
 .bss.openfiles
                0x00000000       0xa0 c:/renesas/ra/e2studio_v2023-10_fsp_v5.0.0/toolchains/gcc_arm/12.2.mpacbti-rel1/bin/../lib/gcc/arm-none-eabi/12.2.1/thumb/v8-m.main+fp/hard\librdimon_nano.a(arm_librdimon_a-syscalls.o)
 .debug_frame   0x00000000      0x39c c:/renesas/ra/e2studio_v2023-10_fsp_v5.0.0/toolchains/gcc_arm/12.2.mpacbti-rel1/bin/../lib/gcc/arm-none-eabi/12.2.1/thumb/v8-m.main+fp/hard\librdimon_nano.a(arm_librdimon_a-syscalls.o)
 .ARM.attributes
                0x00000000       0x38 c:/renesas/ra/e2studio_v2023-10_fsp_v5.0.0/toolchains/gcc_arm/12.2.mpacbti-rel1/bin/../lib/gcc/arm-none-eabi/12.2.1/thumb/v8-m.main+fp/hard\librdimon_nano.a(arm_librdimon_a-syscalls.o)
 .text          0x00000000        0x0 c:/renesas/ra/e2studio_v2023-10_fsp_v5.0.0/toolchains/gcc_arm/12.2.mpacbti-rel1/bin/../lib/gcc/arm-none-eabi/12.2.1/thumb/v8-m.main+fp/hard/crtend.o
 .data          0x00000000        0x0 c:/renesas/ra/e2studio_v2023-10_fsp_v5.0.0/toolchains/gcc_arm/12.2.mpacbti-rel1/bin/../lib/gcc/arm-none-eabi/12.2.1/thumb/v8-m.main+fp/hard/crtend.o
 .bss           0x00000000        0x0 c:/renesas/ra/e2studio_v2023-10_fsp_v5.0.0/toolchains/gcc_arm/12.2.mpacbti-rel1/bin/../lib/gcc/arm-none-eabi/12.2.1/thumb/v8-m.main+fp/hard/crtend.o
 .rodata.all_implied_fbits
                0x00000000       0x24 c:/renesas/ra/e2studio_v2023-10_fsp_v5.0.0/toolchains/gcc_arm/12.2.mpacbti-rel1/bin/../lib/gcc/arm-none-eabi/12.2.1/thumb/v8-m.main+fp/hard/crtend.o
 .text          0x00000000        0x0 c:/renesas/ra/e2studio_v2023-10_fsp_v5.0.0/toolchains/gcc_arm/12.2.mpacbti-rel1/bin/../lib/gcc/arm-none-eabi/12.2.1/thumb/v8-m.main+fp/hard/crtn.o
 .data          0x00000000        0x0 c:/renesas/ra/e2studio_v2023-10_fsp_v5.0.0/toolchains/gcc_arm/12.2.mpacbti-rel1/bin/../lib/gcc/arm-none-eabi/12.2.1/thumb/v8-m.main+fp/hard/crtn.o
 .bss           0x00000000        0x0 c:/renesas/ra/e2studio_v2023-10_fsp_v5.0.0/toolchains/gcc_arm/12.2.mpacbti-rel1/bin/../lib/gcc/arm-none-eabi/12.2.1/thumb/v8-m.main+fp/hard/crtn.o

Memory Configuration

Name             Origin             Length             Attributes
ITCM             0x00000000         0x00000000         xr
DTCM             0x00000000         0x00000000         xrw
FLASH            0x00010000         0x00050000         xr
RAM              0x20000000         0x00020000         xrw
DATA_FLASH       0x08000000         0x00002000         xr
QSPI_FLASH       0x60000000         0x04000000         xr
OSPI_DEVICE_0    0x80020000         0x00000000         xr
OSPI_DEVICE_1    0x80030000         0x00000000         xr
OSPI_DEVICE_0_RAM 0x80020000         0x00000000         xrw
OSPI_DEVICE_1_RAM 0x80030000         0x00000000         xrw
SDRAM            0x80010000         0x00000000         xrw
OPTION_SETTING   0x0100a100         0x00000100         r
OPTION_SETTING_OFS 0x0100a100         0x00000018         r
OPTION_SETTING_SAS 0x0100a134         0x000000cc         r
OPTION_SETTING_S 0x0100a200         0x00000100         r
ID_CODE          0x00000000         0x00000000         xr
*default*        0x00000000         0xffffffff

Linker script and memory map

LOAD c:/renesas/ra/e2studio_v2023-10_fsp_v5.0.0/toolchains/gcc_arm/12.2.mpacbti-rel1/bin/../lib/gcc/arm-none-eabi/12.2.1/thumb/v8-m.main+fp/hard/crti.o
LOAD c:/renesas/ra/e2studio_v2023-10_fsp_v5.0.0/toolchains/gcc_arm/12.2.mpacbti-rel1/bin/../lib/gcc/arm-none-eabi/12.2.1/thumb/v8-m.main+fp/hard/crtbegin.o
LOAD c:/renesas/ra/e2studio_v2023-10_fsp_v5.0.0/toolchains/gcc_arm/12.2.mpacbti-rel1/bin/../lib/gcc/arm-none-eabi/12.2.1/thumb/v8-m.main+fp/hard/rdimon-crt0.o
                0x00010000                        FLASH_IMAGE_START = 0x10000
                0x00050000                        FLASH_IMAGE_LENGTH = 0x50000
START GROUP
LOAD ./src/adc_temp.o
LOAD ./src/angle.o
LOAD ./src/control_table.o
LOAD ./src/crc8.o
LOAD ./src/global_variables.o
LOAD ./src/hal_entry.o
LOAD ./src/interpolation.o
LOAD ./src/monitor.o
LOAD ./src/packet.o
LOAD ./src/pid.o
LOAD ./src/power_monitor.o
LOAD ./src/sintable.o
LOAD ./src/usart.o
LOAD ./ra_gen/common_data.o
LOAD ./ra_gen/hal_data.o
LOAD ./ra_gen/main.o
LOAD ./ra_gen/pin_data.o
LOAD ./ra_gen/vector_data.o
LOAD ./ra/fsp/src/r_sci_uart/r_sci_uart.o
LOAD ./ra/fsp/src/r_sci_spi/r_sci_spi.o
LOAD ./ra/fsp/src/r_sci_i2c/r_sci_i2c.o
LOAD ./ra/fsp/src/r_rtc/r_rtc.o
LOAD ./ra/fsp/src/r_ioport/r_ioport.o
LOAD ./ra/fsp/src/r_gpt/r_gpt.o
LOAD ./ra/fsp/src/r_flash_hp/r_flash_hp.o
LOAD ./ra/fsp/src/r_dtc/r_dtc.o
LOAD ./ra/fsp/src/r_crc/r_crc.o
LOAD ./ra/fsp/src/r_agt/r_agt.o
LOAD ./ra/fsp/src/r_adc/r_adc.o
LOAD ./ra/fsp/src/bsp/mcu/all/bsp_clocks.o
LOAD ./ra/fsp/src/bsp/mcu/all/bsp_common.o
LOAD ./ra/fsp/src/bsp/mcu/all/bsp_delay.o
LOAD ./ra/fsp/src/bsp/mcu/all/bsp_group_irq.o
LOAD ./ra/fsp/src/bsp/mcu/all/bsp_guard.o
LOAD ./ra/fsp/src/bsp/mcu/all/bsp_io.o
LOAD ./ra/fsp/src/bsp/mcu/all/bsp_irq.o
LOAD ./ra/fsp/src/bsp/mcu/all/bsp_register_protection.o
LOAD ./ra/fsp/src/bsp/mcu/all/bsp_rom_registers.o
LOAD ./ra/fsp/src/bsp/mcu/all/bsp_sbrk.o
LOAD ./ra/fsp/src/bsp/mcu/all/bsp_security.o
LOAD ./ra/fsp/src/bsp/cmsis/Device/RENESAS/Source/startup.o
LOAD ./ra/fsp/src/bsp/cmsis/Device/RENESAS/Source/system.o
END GROUP
START GROUP
LOAD c:/renesas/ra/e2studio_v2023-10_fsp_v5.0.0/toolchains/gcc_arm/12.2.mpacbti-rel1/bin/../lib/gcc/arm-none-eabi/12.2.1/thumb/v8-m.main+fp/hard\libgcc.a
LOAD c:/renesas/ra/e2studio_v2023-10_fsp_v5.0.0/toolchains/gcc_arm/12.2.mpacbti-rel1/bin/../lib/gcc/arm-none-eabi/12.2.1/thumb/v8-m.main+fp/hard\libg_nano.a
LOAD c:/renesas/ra/e2studio_v2023-10_fsp_v5.0.0/toolchains/gcc_arm/12.2.mpacbti-rel1/bin/../lib/gcc/arm-none-eabi/12.2.1/thumb/v8-m.main+fp/hard\libc_nano.a
END GROUP
START GROUP
LOAD c:/renesas/ra/e2studio_v2023-10_fsp_v5.0.0/toolchains/gcc_arm/12.2.mpacbti-rel1/bin/../lib/gcc/arm-none-eabi/12.2.1/thumb/v8-m.main+fp/hard\libgcc.a
LOAD c:/renesas/ra/e2studio_v2023-10_fsp_v5.0.0/toolchains/gcc_arm/12.2.mpacbti-rel1/bin/../lib/gcc/arm-none-eabi/12.2.1/thumb/v8-m.main+fp/hard\libc_nano.a
LOAD c:/renesas/ra/e2studio_v2023-10_fsp_v5.0.0/toolchains/gcc_arm/12.2.mpacbti-rel1/bin/../lib/gcc/arm-none-eabi/12.2.1/thumb/v8-m.main+fp/hard\librdimon_nano.a
END GROUP
START GROUP
LOAD c:/renesas/ra/e2studio_v2023-10_fsp_v5.0.0/toolchains/gcc_arm/12.2.mpacbti-rel1/bin/../lib/gcc/arm-none-eabi/12.2.1/thumb/v8-m.main+fp/hard\libgcc.a
LOAD c:/renesas/ra/e2studio_v2023-10_fsp_v5.0.0/toolchains/gcc_arm/12.2.mpacbti-rel1/bin/../lib/gcc/arm-none-eabi/12.2.1/thumb/v8-m.main+fp/hard\libc_nano.a
LOAD c:/renesas/ra/e2studio_v2023-10_fsp_v5.0.0/toolchains/gcc_arm/12.2.mpacbti-rel1/bin/../lib/gcc/arm-none-eabi/12.2.1/thumb/v8-m.main+fp/hard\librdimon_nano.a
END GROUP
LOAD c:/renesas/ra/e2studio_v2023-10_fsp_v5.0.0/toolchains/gcc_arm/12.2.mpacbti-rel1/bin/../lib/gcc/arm-none-eabi/12.2.1/thumb/v8-m.main+fp/hard/crtend.o
LOAD c:/renesas/ra/e2studio_v2023-10_fsp_v5.0.0/toolchains/gcc_arm/12.2.mpacbti-rel1/bin/../lib/gcc/arm-none-eabi/12.2.1/thumb/v8-m.main+fp/hard/crtn.o
                0x20000000                        RAM_START = 0x20000000
                0x00020000                        RAM_LENGTH = 0x20000
                0x00000000                        FLASH_START = 0x0
                0x00060000                        FLASH_LENGTH = 0x60000
                0x08000000                        DATA_FLASH_START = 0x8000000
                0x00002000                        DATA_FLASH_LENGTH = 0x2000
                0x0100a100                        OPTION_SETTING_START = 0x100a100
                0x00000100                        OPTION_SETTING_LENGTH = 0x100
                0x0100a200                        OPTION_SETTING_S_START = 0x100a200
                0x00000100                        OPTION_SETTING_S_LENGTH = 0x100
                0x00000000                        ID_CODE_START = 0x0
                0x00000000                        ID_CODE_LENGTH = 0x0
                0x80010000                        SDRAM_START = 0x80010000
                0x00000000                        SDRAM_LENGTH = 0x0
                0x60000000                        QSPI_FLASH_START = 0x60000000
                0x04000000                        QSPI_FLASH_LENGTH = 0x4000000
                0x80020000                        OSPI_DEVICE_0_START = 0x80020000
                0x00000000                        OSPI_DEVICE_0_LENGTH = 0x0
                0x80030000                        OSPI_DEVICE_1_START = 0x80030000
                0x00000000                        OSPI_DEVICE_1_LENGTH = 0x0
                0x04000000                        QSPI_FLASH_PRV_LENGTH = DEFINED (QSPI_FLASH_SIZE)?ABSOLUTE (QSPI_FLASH_SIZE):ABSOLUTE (QSPI_FLASH_LENGTH)
                0x00000000                        OSPI_DEVICE_0_PRV_LENGTH = DEFINED (OSPI_DEVICE_0_SIZE)?ABSOLUTE (OSPI_DEVICE_0_SIZE):ABSOLUTE (OSPI_DEVICE_0_LENGTH)
                0x00000000                        OSPI_DEVICE_1_PRV_LENGTH = DEFINED (OSPI_DEVICE_1_SIZE)?ABSOLUTE (OSPI_DEVICE_1_SIZE):ABSOLUTE (OSPI_DEVICE_1_LENGTH)
                0x00000000                        __RESERVE_NS_RAM = ((! (DEFINED (PROJECT_NONSECURE)) && DEFINED (RAM_NS_BUFFER_LENGTH)) && (OPTION_SETTING_S_LENGTH != 0x0))
                0x00000000                        ITCM_START = DEFINED (ITCM_START)?ITCM_START:0x0
                0x00000000                        ITCM_LENGTH = DEFINED (ITCM_LENGTH)?ITCM_LENGTH:0x0
                0x00000000                        DTCM_START = DEFINED (DTCM_START)?DTCM_START:0x0
                0x00000000                        DTCM_LENGTH = DEFINED (DTCM_LENGTH)?DTCM_LENGTH:0x0
                0x00000000                        RAM_NS_BUFFER_BLOCK_LENGTH = DEFINED (RAM_NS_BUFFER_LENGTH)?ALIGN (RAM_NS_BUFFER_LENGTH, 0x2000):0x0
                0x00000000                        RAM_NS_BUFFER_LENGTH = DEFINED (RAM_NS_BUFFER_LENGTH)?RAM_NS_BUFFER_LENGTH:0x0
                0x20020000                        RAM_NS_BUFFER_START = ((RAM_START + RAM_LENGTH) - RAM_NS_BUFFER_LENGTH)
                0x20020000                        RAM_NS_BUFFER_BLOCK_START = ((RAM_START + RAM_LENGTH) - RAM_NS_BUFFER_BLOCK_LENGTH)
                0x0100a180                        OPTION_SETTING_START_NS = DEFINED (PROJECT_NONSECURE)?OPTION_SETTING_START:(OPTION_SETTING_START + 0x80)
                0x00000001                        __bl_FSP_BOOTABLE_IMAGE = 0x1
                0x00000001                        __bln_FSP_BOOTABLE_IMAGE = 0x1
                0x00000001                        PROJECT_SECURE_OR_FLAT = (((! (DEFINED (PROJECT_NONSECURE)) || DEFINED (PROJECT_SECURE)) && OPTION_SETTING_LENGTH) && ! (DEFINED (FSP_BOOTABLE_IMAGE)))
                0x00000000                        USE_OPTION_SETTING_NS = (DEFINED (PROJECT_NONSECURE) && ! (DEFINED (FSP_BOOTABLE_IMAGE)))
                0x00000000                        __bl_FLASH_IMAGE_START = ! (DEFINED (FLASH_BOOTLOADER_LENGTH))?0x0:(FLASH_APPLICATION_IMAGE_NUMBER == 0x1)?((FLASH_START + FLASH_BOOTLOADER_LENGTH) + FLASH_BOOTLOADER_HEADER_LENGTH):((((FLASH_START + FLASH_BOOTLOADER_LENGTH) + FLASH_BOOTLOADER_SCRATCH_LENGTH) + FLASH_APPLICATION_S_LENGTH) + FLASH_BOOTLOADER_HEADER_LENGTH)
                0x00000000                        __bl_FLASH_IMAGE_LENGTH = ! (DEFINED (FLASH_BOOTLOADER_LENGTH))?0x0:(FLASH_APPLICATION_S_LENGTH - FLASH_BOOTLOADER_HEADER_LENGTH)
                0x00000000                        __bl_FLASH_IMAGE_END = (__bl_FLASH_IMAGE_START + __bl_FLASH_IMAGE_LENGTH)
                0x00000000                        __bl_XIP_SECONDARY_FLASH_IMAGE_START = ! (DEFINED (FLASH_BOOTLOADER_LENGTH))?0x0:((FLASH_BOOTLOADER_LENGTH + FLASH_APPLICATION_S_LENGTH) + FLASH_BOOTLOADER_HEADER_LENGTH)
                0x00000000                        __bl_XIP_SECONDARY_FLASH_IMAGE_END = (__bl_XIP_SECONDARY_FLASH_IMAGE_START + __bl_FLASH_IMAGE_LENGTH)
                0x00000000                        __bl_FLASH_NS_START = ! (DEFINED (FLASH_BOOTLOADER_LENGTH))?0x0:(FLASH_APPLICATION_NS_LENGTH == 0x0)?__bl_FLASH_IMAGE_END:((__bl_FLASH_IMAGE_START - FLASH_BOOTLOADER_HEADER_LENGTH) + FLASH_APPLICATION_S_LENGTH)
                0x00000000                        __bl_FLASH_NSC_START = ! (DEFINED (FLASH_BOOTLOADER_LENGTH))?0x0:(FLASH_APPLICATION_NS_LENGTH == 0x0)?__bl_FLASH_IMAGE_END:(__bl_FLASH_IMAGE_END - FLASH_APPLICATION_NSC_LENGTH)
                0x00000000                        __bl_RAM_NS_START = ! (DEFINED (FLASH_BOOTLOADER_LENGTH))?0x0:(FLASH_APPLICATION_NS_LENGTH == 0x0)?(RAM_START + RAM_LENGTH):((RAM_START + RAM_LENGTH) - RAM_APPLICATION_NS_LENGTH)
                0x00000000                        __bl_RAM_NSC_START = ! (DEFINED (FLASH_BOOTLOADER_LENGTH))?0x0:(FLASH_APPLICATION_NS_LENGTH == 0x0)?(RAM_START + RAM_LENGTH):(__bl_RAM_NS_START - RAM_APPLICATION_NSC_LENGTH)
                0x00000000                        __bl_FLASH_NS_IMAGE_START = ! (DEFINED (FLASH_BOOTLOADER_LENGTH))?0x0:(FLASH_APPLICATION_NS_LENGTH == 0x0)?__bl_FLASH_IMAGE_END:(__bl_FLASH_NS_START + FLASH_BOOTLOADER_HEADER_LENGTH_2)
                0x00000000                        __bln_FLASH_IMAGE_START = (__bl_FLASH_NS_IMAGE_START | ! (DEFINED (NS_OFFSET_START))?0x0:NS_OFFSET_START)
                0x00000000                        __bln_FLASH_IMAGE_LENGTH = ! (DEFINED (FLASH_BOOTLOADER_LENGTH))?0x0:(FLASH_APPLICATION_NS_LENGTH == 0x0)?__bl_FLASH_IMAGE_END:(FLASH_APPLICATION_NS_LENGTH - FLASH_BOOTLOADER_HEADER_LENGTH_2)
                0x00000000                        XIP_SECONDARY_SLOT_IMAGE = DEFINED (XIP_SECONDARY_SLOT_IMAGE)?XIP_SECONDARY_SLOT_IMAGE:0x0
                0x00010000                        FLASH_ORIGIN = ! (DEFINED (FLASH_IMAGE_START))?FLASH_START:(XIP_SECONDARY_SLOT_IMAGE == 0x1)?XIP_SECONDARY_FLASH_IMAGE_START:FLASH_IMAGE_START
                0x00050000                        LIMITED_FLASH_LENGTH = DEFINED (FLASH_IMAGE_LENGTH)?FLASH_IMAGE_LENGTH:DEFINED (FLASH_BOOTLOADER_LENGTH)?FLASH_BOOTLOADER_LENGTH:FLASH_LENGTH
                0x00000034                        OPTION_SETTING_SAS_SIZE = 0x34
                0x000000cc                        OPTION_SETTING_SAS_LENGTH = ! (DEFINED (OPTION_SETTING_LENGTH))?0x0:(OPTION_SETTING_LENGTH == 0x0)?0x0:(OPTION_SETTING_LENGTH - OPTION_SETTING_SAS_SIZE)
START GROUP
LOAD c:/renesas/ra/e2studio_v2023-10_fsp_v5.0.0/toolchains/gcc_arm/12.2.mpacbti-rel1/bin/../lib/gcc/arm-none-eabi/12.2.1/thumb/v8-m.main+fp/hard\libgcc.a
LOAD c:/renesas/ra/e2studio_v2023-10_fsp_v5.0.0/toolchains/gcc_arm/12.2.mpacbti-rel1/bin/../lib/gcc/arm-none-eabi/12.2.1/thumb/v8-m.main+fp/hard\libc.a
LOAD c:/renesas/ra/e2studio_v2023-10_fsp_v5.0.0/toolchains/gcc_arm/12.2.mpacbti-rel1/bin/../lib/gcc/arm-none-eabi/12.2.1/thumb/v8-m.main+fp/hard\libm.a
END GROUP

.text           0x00010000     0xa668
                0x00000000                        __tz_FLASH_S = ABSOLUTE (FLASH_START)
                0x00010000                        __ROM_Start = .
 *(.fixed_vectors*)
 .fixed_vectors
                0x00010000       0x40 ./ra/fsp/src/bsp/cmsis/Device/RENESAS/Source/startup.o
                0x00010000                __Vectors
 *(.application_vectors*)
 .application_vectors
                0x00010040      0x180 ./ra_gen/vector_data.o
                0x00010040                g_vector_table
                0x000101c0                        __Vectors_End = .
                0x000101c0                        . = (OPTION_SETTING_LENGTH > 0x0)?.:(__ROM_Start + 0x400)
 *(.rom_registers*)
                0x000101c0                        . = (OPTION_SETTING_LENGTH > 0x0)?.:(__ROM_Start + 0x500)
                0x00010200                        . = ALIGN (0x80)
 *fill*         0x000101c0       0x40 ff
 *(.mcuboot_sce9_key*)
 *(.text*)
 .text.deregister_tm_clones
                0x00010200       0x1c c:/renesas/ra/e2studio_v2023-10_fsp_v5.0.0/toolchains/gcc_arm/12.2.mpacbti-rel1/bin/../lib/gcc/arm-none-eabi/12.2.1/thumb/v8-m.main+fp/hard/crtbegin.o
 .text.register_tm_clones
                0x0001021c       0x28 c:/renesas/ra/e2studio_v2023-10_fsp_v5.0.0/toolchains/gcc_arm/12.2.mpacbti-rel1/bin/../lib/gcc/arm-none-eabi/12.2.1/thumb/v8-m.main+fp/hard/crtbegin.o
 .text.__do_global_dtors_aux
                0x00010244       0x28 c:/renesas/ra/e2studio_v2023-10_fsp_v5.0.0/toolchains/gcc_arm/12.2.mpacbti-rel1/bin/../lib/gcc/arm-none-eabi/12.2.1/thumb/v8-m.main+fp/hard/crtbegin.o
 .text.frame_dummy
                0x0001026c       0x24 c:/renesas/ra/e2studio_v2023-10_fsp_v5.0.0/toolchains/gcc_arm/12.2.mpacbti-rel1/bin/../lib/gcc/arm-none-eabi/12.2.1/thumb/v8-m.main+fp/hard/crtbegin.o
 .text.movingmean
                0x00010290       0x80 ./src/adc_temp.o
 .text.get_motor_temp
                0x00010310       0x38 ./src/adc_temp.o
                0x00010310                get_motor_temp
 .text.get_hvamp_temp
                0x00010348       0x3c ./src/adc_temp.o
                0x00010348                get_hvamp_temp
 *fill*         0x00010384        0x4 ff
 .text.get_cpu_temp
                0x00010388       0x68 ./src/adc_temp.o
                0x00010388                get_cpu_temp
 .text.update_adcvalue
                0x000103f0       0x90 ./src/adc_temp.o
                0x000103f0                update_adcvalue
 .text.sci_spi_callback
                0x00010480       0x18 ./src/angle.o
                0x00010480                sci_spi_callback
 .text.tad2141_readstream
                0x00010498       0xa8 ./src/angle.o
                0x00010498                tad2141_readstream
 .text.tad2141_init
                0x00010540       0xdc ./src/angle.o
                0x00010540                tad2141_init
 .text.RestoreControlTable2FactoryDefaults
                0x0001061c       0xd4 ./src/control_table.o
                0x0001061c                RestoreControlTable2FactoryDefaults
 .text.write_item
                0x000106f0       0xd4 ./src/control_table.o
                0x000106f0                write_item
 .text.read_item
                0x000107c4       0x70 ./src/control_table.o
                0x000107c4                read_item
 .text.SaveCcontroltableToNVM
                0x00010834       0xc0 ./src/control_table.o
                0x00010834                SaveCcontroltableToNVM
 *fill*         0x000108f4        0x4 ff
 .text.LoadCcontroltableFromNVM
                0x000108f8       0xb4 ./src/control_table.o
                0x000108f8                LoadCcontroltableFromNVM
 .text.CalcCRC8
                0x000109ac       0x28 ./src/crc8.o
                0x000109ac                CalcCRC8
 .text.GetCRC8  0x000109d4       0x14 ./src/crc8.o
                0x000109d4                GetCRC8
 .text.__NVIC_SystemReset
                0x000109e8       0x24 ./src/hal_entry.o
 .text.CurveInterpolation
                0x00010a0c      0x2e4 ./src/hal_entry.o
 .text.ReqNumConversionItems
                0x00010cf0      0x104 ./src/hal_entry.o
 .text.led_on   0x00010df4       0x18 ./src/hal_entry.o
                0x00010df4                led_on
 .text.led_off  0x00010e0c       0x18 ./src/hal_entry.o
                0x00010e0c                led_off
 *fill*         0x00010e24        0x4 ff
 .text.rgt0_callback
                0x00010e28     0x14b4 ./src/hal_entry.o
                0x00010e28                rgt0_callback
 .text.hal_entry
                0x000122dc      0x1a0 ./src/hal_entry.o
                0x000122dc                hal_entry
 .text.R_BSP_WarmStart
                0x0001247c       0x18 ./src/hal_entry.o
                0x0001247c                R_BSP_WarmStart
 .text.interp1dim
                0x00012494       0x8c ./src/interpolation.o
                0x00012494                interp1dim
 .text.MonConditions
                0x00012520      0x134 ./src/monitor.o
                0x00012520                MonConditions
 *fill*         0x00012654        0x4 ff
 .text.write_item_callback
                0x00012658      0x274 ./src/packet.o
                0x00012658                write_item_callback
 .text.concack.part.0
                0x000128cc       0x94 ./src/packet.o
 .text.cmd_rb   0x00012960       0x58 ./src/packet.o
 .text.read_item_callback
                0x000129b8       0x38 ./src/packet.o
                0x000129b8                read_item_callback
 .text.concdec.part.0
                0x000129f0       0xac ./src/packet.o
 .text.cmd_cb   0x00012a9c       0x44 ./src/packet.o
 .text.cmd_cp   0x00012ae0       0x44 ./src/packet.o
 .text.cmd_cc   0x00012b24       0x44 ./src/packet.o
 .text.cmd_cv   0x00012b68       0x44 ./src/packet.o
 .text.cmd_ca   0x00012bac       0x44 ./src/packet.o
 .text.cmd_vr   0x00012bf0      0x1d4 ./src/packet.o
 .text.cmd_st   0x00012dc4       0xd8 ./src/packet.o
 .text.cmd_wd   0x00012e9c       0x48 ./src/packet.o
 .text.cmd_sg   0x00012ee4       0xe4 ./src/packet.o
 .text.cmd_ex   0x00012fc8       0x74 ./src/packet.o
 .text.cmd_tp   0x0001303c       0x74 ./src/packet.o
 .text.cmd_tc   0x000130b0       0x9c ./src/packet.o
 .text.cmd_tv   0x0001314c       0x9c ./src/packet.o
 .text.cmd_ta   0x000131e8       0x9c ./src/packet.o
 .text.cmd_wr   0x00013284       0xd4 ./src/packet.o
 .text.cmd_ct   0x00013358       0xec ./src/packet.o
 .text.cmd_crc  0x00013444       0xe0 ./src/packet.o
 .text.cmd_id   0x00013524       0xe8 ./src/packet.o
 .text.cmd_ini  0x0001360c       0xc4 ./src/packet.o
 .text.cmd_rr   0x000136d0      0x448 ./src/packet.o
 .text.packet_receive
                0x00013b18      0x1c4 ./src/packet.o
                0x00013b18                packet_receive
 .text.packet_handling
                0x00013cdc      0x374 ./src/packet.o
                0x00013cdc                packet_handling
 .text.PIDReset_real
                0x00014050       0x14 ./src/pid.o
                0x00014050                PIDReset_real
 .text.PIDUpdate_real
                0x00014064      0x110 ./src/pid.o
                0x00014064                PIDUpdate_real
 .text.sci_i2c_master_callback
                0x00014174       0xe8 ./src/power_monitor.o
                0x00014174                sci_i2c_master_callback
 .text.isl28022_write
                0x0001425c       0xcc ./src/power_monitor.o
                0x0001425c                isl28022_write
 .text.isl28022_read
                0x00014328       0x58 ./src/power_monitor.o
                0x00014328                isl28022_read
 .text.isl28022_read_ex
                0x00014380       0x80 ./src/power_monitor.o
                0x00014380                isl28022_read_ex
 .text.isl28022_comp_stat
                0x00014400       0x18 ./src/power_monitor.o
                0x00014400                isl28022_comp_stat
 .text.isl28022_force_reset_stat
                0x00014418       0x24 ./src/power_monitor.o
                0x00014418                isl28022_force_reset_stat
 .text.isl28022_init
                0x0001443c      0x11c ./src/power_monitor.o
                0x0001443c                isl28022_init
 .text.my_cos1000
                0x00014558       0xa8 ./src/sintable.o
                0x00014558                my_cos1000
 .text.user_uart_callback
                0x00014600       0x94 ./src/usart.o
                0x00014600                user_uart_callback
 .text.us_tx_buff
                0x00014694       0x10 ./src/usart.o
                0x00014694                us_tx_buff
 .text.us_rx_buff
                0x000146a4       0x1c ./src/usart.o
                0x000146a4                us_rx_buff
 .text.us_putsb
                0x000146c0       0x9c ./src/usart.o
                0x000146c0                us_putsb
 .text.us_getc  0x0001475c       0x30 ./src/usart.o
                0x0001475c                us_getc
 .text.us_setbaudrate
                0x0001478c       0x30 ./src/usart.o
                0x0001478c                us_setbaudrate
 .text.us_init  0x000147bc       0x78 ./src/usart.o
                0x000147bc                us_init
 .text.startup.main
                0x00014834        0xc ./ra_gen/main.o
                0x00014834                main
 .text.R_SCI_UART_Write
                0x00014840       0xac ./ra/fsp/src/r_sci_uart/r_sci_uart.o
                0x00014840                R_SCI_UART_Write
 .text.R_SCI_UART_BaudSet
                0x000148ec       0x4c ./ra/fsp/src/r_sci_uart/r_sci_uart.o
                0x000148ec                R_SCI_UART_BaudSet
 .text.R_SCI_UART_Abort
                0x00014938       0x84 ./ra/fsp/src/r_sci_uart/r_sci_uart.o
                0x00014938                R_SCI_UART_Abort
 .text.R_SCI_UART_Open
                0x000149bc      0x42c ./ra/fsp/src/r_sci_uart/r_sci_uart.o
                0x000149bc                R_SCI_UART_Open
 .text.R_SCI_UART_BaudCalculate
                0x00014de8      0x1d0 ./ra/fsp/src/r_sci_uart/r_sci_uart.o
                0x00014de8                R_SCI_UART_BaudCalculate
 .text.sci_uart_txi_isr
                0x00014fb8      0x160 ./ra/fsp/src/r_sci_uart/r_sci_uart.o
                0x00014fb8                sci_uart_txi_isr
 .text.sci_uart_rxi_isr
                0x00015118      0x16c ./ra/fsp/src/r_sci_uart/r_sci_uart.o
                0x00015118                sci_uart_rxi_isr
 .text.sci_uart_tei_isr
                0x00015284       0x80 ./ra/fsp/src/r_sci_uart/r_sci_uart.o
                0x00015284                sci_uart_tei_isr
 .text.sci_uart_eri_isr
                0x00015304       0xb8 ./ra/fsp/src/r_sci_uart/r_sci_uart.o
                0x00015304                sci_uart_eri_isr
 .text.R_SCI_SPI_WriteRead
                0x000153bc      0x124 ./ra/fsp/src/r_sci_spi/r_sci_spi.o
                0x000153bc                R_SCI_SPI_WriteRead
 .text.R_SCI_SPI_Open
                0x000154e0      0x2d4 ./ra/fsp/src/r_sci_spi/r_sci_spi.o
                0x000154e0                R_SCI_SPI_Open
 .text.sci_spi_txi_isr
                0x000157b4       0x6c ./ra/fsp/src/r_sci_spi/r_sci_spi.o
                0x000157b4                sci_spi_txi_isr
 .text.sci_spi_rxi_isr
                0x00015820       0x78 ./ra/fsp/src/r_sci_spi/r_sci_spi.o
                0x00015820                sci_spi_rxi_isr
 .text.sci_spi_tei_isr
                0x00015898       0x70 ./ra/fsp/src/r_sci_spi/r_sci_spi.o
                0x00015898                sci_spi_tei_isr
 .text.sci_spi_eri_isr
                0x00015908       0x78 ./ra/fsp/src/r_sci_spi/r_sci_spi.o
                0x00015908                sci_spi_eri_isr
 .text.R_SCI_I2C_SlaveAddressSet
                0x00015980        0xc ./ra/fsp/src/r_sci_i2c/r_sci_i2c.o
                0x00015980                R_SCI_I2C_SlaveAddressSet
 .text.R_SCI_I2C_Read
                0x0001598c       0x94 ./ra/fsp/src/r_sci_i2c/r_sci_i2c.o
                0x0001598c                R_SCI_I2C_Read
 .text.R_SCI_I2C_Write
                0x00015a20       0x90 ./ra/fsp/src/r_sci_i2c/r_sci_i2c.o
                0x00015a20                R_SCI_I2C_Write
 .text.R_SCI_I2C_Open
                0x00015ab0      0x170 ./ra/fsp/src/r_sci_i2c/r_sci_i2c.o
                0x00015ab0                R_SCI_I2C_Open
 .text.sci_i2c_txi_isr
                0x00015c20      0x144 ./ra/fsp/src/r_sci_i2c/r_sci_i2c.o
                0x00015c20                sci_i2c_txi_isr
 .text.sci_i2c_tei_isr
                0x00015d64      0x120 ./ra/fsp/src/r_sci_i2c/r_sci_i2c.o
                0x00015d64                sci_i2c_tei_isr
 .text.rtc_carry_isr
                0x00015e84       0x30 ./ra/fsp/src/r_rtc/r_rtc.o
                0x00015e84                rtc_carry_isr
 .text.R_IOPORT_Close
                0x00015eb4        0xc ./ra/fsp/src/r_ioport/r_ioport.o
                0x00015eb4                R_IOPORT_Close
 .text.R_IOPORT_PinRead
                0x00015ec0       0x24 ./ra/fsp/src/r_ioport/r_ioport.o
                0x00015ec0                R_IOPORT_PinRead
 .text.R_IOPORT_PortRead
                0x00015ee4       0x14 ./ra/fsp/src/r_ioport/r_ioport.o
                0x00015ee4                R_IOPORT_PortRead
 .text.R_IOPORT_PortWrite
                0x00015ef8       0x1c ./ra/fsp/src/r_ioport/r_ioport.o
                0x00015ef8                R_IOPORT_PortWrite
 .text.R_IOPORT_PinWrite
                0x00015f14       0x20 ./ra/fsp/src/r_ioport/r_ioport.o
                0x00015f14                R_IOPORT_PinWrite
 .text.R_IOPORT_PortDirectionSet
                0x00015f34       0x2c ./ra/fsp/src/r_ioport/r_ioport.o
                0x00015f34                R_IOPORT_PortDirectionSet
 .text.R_IOPORT_PortEventInputRead
                0x00015f60       0x18 ./ra/fsp/src/r_ioport/r_ioport.o
                0x00015f60                R_IOPORT_PortEventInputRead
 .text.R_IOPORT_PinEventInputRead
                0x00015f78       0x34 ./ra/fsp/src/r_ioport/r_ioport.o
                0x00015f78                R_IOPORT_PinEventInputRead
 .text.R_IOPORT_PortEventOutputWrite
                0x00015fac       0x1c ./ra/fsp/src/r_ioport/r_ioport.o
                0x00015fac                R_IOPORT_PortEventOutputWrite
 .text.R_IOPORT_PinEventOutputWrite
                0x00015fc8       0x34 ./ra/fsp/src/r_ioport/r_ioport.o
                0x00015fc8                R_IOPORT_PinEventOutputWrite
 .text.bsp_vbatt_init
                0x00015ffc      0x128 ./ra/fsp/src/r_ioport/r_ioport.o
 .text.r_ioport_pins_config
                0x00016124       0xa8 ./ra/fsp/src/r_ioport/r_ioport.o
 .text.R_IOPORT_Open
                0x000161cc       0x14 ./ra/fsp/src/r_ioport/r_ioport.o
                0x000161cc                R_IOPORT_Open
 .text.R_IOPORT_PinsCfg
                0x000161e0        0xc ./ra/fsp/src/r_ioport/r_ioport.o
                0x000161e0                R_IOPORT_PinsCfg
 .text.R_IOPORT_PinCfg
                0x000161ec       0xa8 ./ra/fsp/src/r_ioport/r_ioport.o
                0x000161ec                R_IOPORT_PinCfg
 .text.R_GPT_Start
                0x00016294        0xc ./ra/fsp/src/r_gpt/r_gpt.o
                0x00016294                R_GPT_Start
 .text.r_gpt_enable_irq
                0x000162a0       0x60 ./ra/fsp/src/r_gpt/r_gpt.o
 .text.R_GPT_DutyCycleSet
                0x00016300      0x188 ./ra/fsp/src/r_gpt/r_gpt.o
                0x00016300                R_GPT_DutyCycleSet
 .text.R_GPT_Open
                0x00016488      0x298 ./ra/fsp/src/r_gpt/r_gpt.o
                0x00016488                R_GPT_Open
 .text.R_FLASH_HP_Close
                0x00016720       0x6c ./ra/fsp/src/r_flash_hp/r_flash_hp.o
                0x00016720                R_FLASH_HP_Close
 .text.flash_hp_enter_pe_df_mode
                0x0001678c       0xd0 ./ra/fsp/src/r_flash_hp/r_flash_hp.o
 .text.R_FLASH_HP_Open
                0x0001685c      0x1e0 ./ra/fsp/src/r_flash_hp/r_flash_hp.o
                0x0001685c                R_FLASH_HP_Open
 .text.R_FLASH_HP_Erase
                0x00016a3c      0x18c ./ra/fsp/src/r_flash_hp/r_flash_hp.o
                0x00016a3c                R_FLASH_HP_Erase
 .text.R_FLASH_HP_Write
                0x00016bc8      0x224 ./ra/fsp/src/r_flash_hp/r_flash_hp.o
                0x00016bc8                R_FLASH_HP_Write
 .text.R_DTC_Reset
                0x00016dec       0x8c ./ra/fsp/src/r_dtc/r_dtc.o
                0x00016dec                R_DTC_Reset
 .text.R_DTC_SoftwareStart
                0x00016e78        0x4 ./ra/fsp/src/r_dtc/r_dtc.o
                0x00016e78                R_DTC_SoftwareStart
 .text.R_DTC_SoftwareStop
                0x00016e7c        0x4 ./ra/fsp/src/r_dtc/r_dtc.o
                0x00016e7c                R_DTC_SoftwareStop
 .text.R_DTC_Enable
                0x00016e80       0x20 ./ra/fsp/src/r_dtc/r_dtc.o
                0x00016e80                R_DTC_Enable
 .text.R_DTC_Disable
                0x00016ea0       0x20 ./ra/fsp/src/r_dtc/r_dtc.o
                0x00016ea0                R_DTC_Disable
 .text.R_DTC_InfoGet
                0x00016ec0       0x5c ./ra/fsp/src/r_dtc/r_dtc.o
                0x00016ec0                R_DTC_InfoGet
 .text.R_DTC_Reload
                0x00016f1c        0x4 ./ra/fsp/src/r_dtc/r_dtc.o
                0x00016f1c                R_DTC_Reload
 .text.R_DTC_Close
                0x00016f20       0x34 ./ra/fsp/src/r_dtc/r_dtc.o
                0x00016f20                R_DTC_Close
 .text.R_DTC_Open
                0x00016f54       0xbc ./ra/fsp/src/r_dtc/r_dtc.o
                0x00016f54                R_DTC_Open
 .text.R_DTC_Reconfigure
                0x00017010       0x7c ./ra/fsp/src/r_dtc/r_dtc.o
                0x00017010                R_DTC_Reconfigure
 .text.R_CRC_Open
                0x0001708c       0x44 ./ra/fsp/src/r_crc/r_crc.o
                0x0001708c                R_CRC_Open
 .text.R_CRC_Close
                0x000170d0       0x28 ./ra/fsp/src/r_crc/r_crc.o
                0x000170d0                R_CRC_Close
 .text.R_CRC_Calculate
                0x000170f8       0x88 ./ra/fsp/src/r_crc/r_crc.o
                0x000170f8                R_CRC_Calculate
 .text.R_AGT_Enable
                0x00017180       0x24 ./ra/fsp/src/r_agt/r_agt.o
                0x00017180                R_AGT_Enable
 .text.R_AGT_Open
                0x000171a4      0x150 ./ra/fsp/src/r_agt/r_agt.o
                0x000171a4                R_AGT_Open
 .text.agt_int_isr
                0x000172f4       0x9c ./ra/fsp/src/r_agt/r_agt.o
                0x000172f4                agt_int_isr
 .text.R_ADC_ScanStart
                0x00017390        0xc ./ra/fsp/src/r_adc/r_adc.o
                0x00017390                R_ADC_ScanStart
 .text.R_ADC_Read
                0x0001739c       0x10 ./ra/fsp/src/r_adc/r_adc.o
                0x0001739c                R_ADC_Read
 .text.R_ADC_ScanCfg
                0x000173ac      0x1e8 ./ra/fsp/src/r_adc/r_adc.o
                0x000173ac                R_ADC_ScanCfg
 .text.R_ADC_Open
                0x00017594      0x23c ./ra/fsp/src/r_adc/r_adc.o
                0x00017594                R_ADC_Open
 .text.SystemCoreClockUpdate
                0x000177d0       0x28 ./ra/fsp/src/bsp/mcu/all/bsp_clocks.o
                0x000177d0                SystemCoreClockUpdate
 .text.R_BSP_SubClockStabilizeWaitAfterReset
                0x000177f8        0x4 ./ra/fsp/src/bsp/mcu/all/bsp_clocks.o
                0x000177f8                R_BSP_SubClockStabilizeWaitAfterReset
 .text.bsp_clock_init
                0x000177fc      0x174 ./ra/fsp/src/bsp/mcu/all/bsp_clocks.o
                0x000177fc                bsp_clock_init
 .text.R_BSP_Init_RTC
                0x00017970       0x28 ./ra/fsp/src/bsp/mcu/all/bsp_clocks.o
                0x00017970                R_BSP_Init_RTC
 .text.bsp_init_internal
                0x00017998        0x4 ./ra/fsp/src/bsp/mcu/all/bsp_common.o
                0x00017998                bsp_init_internal
                0x00017998                bsp_init
 .text.bsp_prv_software_delay_loop
                0x0001799c        0xc ./ra/fsp/src/bsp/mcu/all/bsp_delay.o
                0x0001799c                bsp_prv_software_delay_loop
 .text.R_BSP_SoftwareDelay
                0x000179a8       0x58 ./ra/fsp/src/bsp/mcu/all/bsp_delay.o
                0x000179a8                R_BSP_SoftwareDelay
 .text.NMI_Handler
                0x00017a00       0x3c ./ra/fsp/src/bsp/mcu/all/bsp_group_irq.o
                0x00017a00                NMI_Handler
 .text.bsp_irq_cfg
                0x00017a3c       0xa4 ./ra/fsp/src/bsp/mcu/all/bsp_irq.o
                0x00017a3c                bsp_irq_cfg
 .text.R_BSP_RegisterProtectEnable
                0x00017ae0       0x60 ./ra/fsp/src/bsp/mcu/all/bsp_register_protection.o
                0x00017ae0                R_BSP_RegisterProtectEnable
 .text.R_BSP_RegisterProtectDisable
                0x00017b40       0x54 ./ra/fsp/src/bsp/mcu/all/bsp_register_protection.o
                0x00017b40                R_BSP_RegisterProtectDisable
 .text.Default_Handler
                0x00017b94        0x4 ./ra/fsp/src/bsp/cmsis/Device/RENESAS/Source/startup.o
                0x00017b94                DebugMon_Handler
                0x00017b94                HardFault_Handler
                0x00017b94                SysTick_Handler
                0x00017b94                PendSV_Handler
                0x00017b94                UsageFault_Handler
                0x00017b94                SecureFault_Handler
                0x00017b94                Default_Handler
                0x00017b94                MemManage_Handler
                0x00017b94                SVC_Handler
                0x00017b94                BusFault_Handler
 .text.Reset_Handler
                0x00017b98        0xc ./ra/fsp/src/bsp/cmsis/Device/RENESAS/Source/startup.o
                0x00017b98                Reset_Handler
 .text.SystemInit
                0x00017ba4       0xc4 ./ra/fsp/src/bsp/cmsis/Device/RENESAS/Source/system.o
                0x00017ba4                SystemInit
 .text          0x00017c68      0x378 c:/renesas/ra/e2studio_v2023-10_fsp_v5.0.0/toolchains/gcc_arm/12.2.mpacbti-rel1/bin/../lib/gcc/arm-none-eabi/12.2.1/thumb/v8-m.main+fp/hard\libgcc.a(_arm_addsubdf3.o)
                0x00017c68                __aeabi_drsub
                0x00017c70                __aeabi_dsub
                0x00017c70                __subdf3
                0x00017c74                __aeabi_dadd
                0x00017c74                __adddf3
                0x00017eec                __floatunsidf
                0x00017eec                __aeabi_ui2d
                0x00017f0c                __floatsidf
                0x00017f0c                __aeabi_i2d
                0x00017f30                __aeabi_f2d
                0x00017f30                __extendsfdf2
                0x00017f74                __floatundidf
                0x00017f74                __aeabi_ul2d
                0x00017f84                __floatdidf
                0x00017f84                __aeabi_l2d
 .text          0x00017fe0      0x424 c:/renesas/ra/e2studio_v2023-10_fsp_v5.0.0/toolchains/gcc_arm/12.2.mpacbti-rel1/bin/../lib/gcc/arm-none-eabi/12.2.1/thumb/v8-m.main+fp/hard\libgcc.a(_arm_muldivdf3.o)
                0x00017fe0                __aeabi_dmul
                0x00017fe0                __muldf3
                0x00018234                __divdf3
                0x00018234                __aeabi_ddiv
 .text          0x00018404      0x110 c:/renesas/ra/e2studio_v2023-10_fsp_v5.0.0/toolchains/gcc_arm/12.2.mpacbti-rel1/bin/../lib/gcc/arm-none-eabi/12.2.1/thumb/v8-m.main+fp/hard\libgcc.a(_arm_cmpdf2.o)
                0x00018404                __gtdf2
                0x00018404                __gedf2
                0x0001840c                __ltdf2
                0x0001840c                __ledf2
                0x00018414                __nedf2
                0x00018414                __eqdf2
                0x00018414                __cmpdf2
                0x00018490                __aeabi_cdrcmple
                0x000184a0                __aeabi_cdcmpeq
                0x000184a0                __aeabi_cdcmple
                0x000184b0                __aeabi_dcmpeq
                0x000184c4                __aeabi_dcmplt
                0x000184d8                __aeabi_dcmple
                0x000184ec                __aeabi_dcmpge
                0x00018500                __aeabi_dcmpgt
 .text          0x00018514       0x50 c:/renesas/ra/e2studio_v2023-10_fsp_v5.0.0/toolchains/gcc_arm/12.2.mpacbti-rel1/bin/../lib/gcc/arm-none-eabi/12.2.1/thumb/v8-m.main+fp/hard\libgcc.a(_arm_fixdfsi.o)
                0x00018514                __aeabi_d2iz
                0x00018514                __fixdfsi
 .text          0x00018564       0x40 c:/renesas/ra/e2studio_v2023-10_fsp_v5.0.0/toolchains/gcc_arm/12.2.mpacbti-rel1/bin/../lib/gcc/arm-none-eabi/12.2.1/thumb/v8-m.main+fp/hard\libgcc.a(_arm_fixunsdfsi.o)
                0x00018564                __aeabi_d2uiz
                0x00018564                __fixunsdfsi
 .text          0x000185a4       0xa0 c:/renesas/ra/e2studio_v2023-10_fsp_v5.0.0/toolchains/gcc_arm/12.2.mpacbti-rel1/bin/../lib/gcc/arm-none-eabi/12.2.1/thumb/v8-m.main+fp/hard\libgcc.a(_aeabi_ldivmod.o)
                0x000185a4                __aeabi_ldivmod
 .text.__udivmoddi4
                0x00018644      0x2e4 c:/renesas/ra/e2studio_v2023-10_fsp_v5.0.0/toolchains/gcc_arm/12.2.mpacbti-rel1/bin/../lib/gcc/arm-none-eabi/12.2.1/thumb/v8-m.main+fp/hard\libgcc.a(_udivmoddi4.o)
                0x00018644                __udivmoddi4
 .text          0x00018928        0x4 c:/renesas/ra/e2studio_v2023-10_fsp_v5.0.0/toolchains/gcc_arm/12.2.mpacbti-rel1/bin/../lib/gcc/arm-none-eabi/12.2.1/thumb/v8-m.main+fp/hard\libgcc.a(_dvmd_tls.o)
                0x00018928                __aeabi_idiv0
                0x00018928                __aeabi_ldiv0
 .text.__itoa   0x0001892c       0x30 c:/renesas/ra/e2studio_v2023-10_fsp_v5.0.0/toolchains/gcc_arm/12.2.mpacbti-rel1/bin/../lib/gcc/arm-none-eabi/12.2.1/thumb/v8-m.main+fp/hard\libg_nano.a(libc_a-itoa.o)
                0x0001892c                __itoa
 .text._strtol_l.constprop.0
                0x0001895c       0xfc c:/renesas/ra/e2studio_v2023-10_fsp_v5.0.0/toolchains/gcc_arm/12.2.mpacbti-rel1/bin/../lib/gcc/arm-none-eabi/12.2.1/thumb/v8-m.main+fp/hard\libg_nano.a(libc_a-strtol.o)
 .text.strtol   0x00018a58       0x14 c:/renesas/ra/e2studio_v2023-10_fsp_v5.0.0/toolchains/gcc_arm/12.2.mpacbti-rel1/bin/../lib/gcc/arm-none-eabi/12.2.1/thumb/v8-m.main+fp/hard\libg_nano.a(libc_a-strtol.o)
                0x00018a58                strtol
 .text.__utoa   0x00018a6c       0x84 c:/renesas/ra/e2studio_v2023-10_fsp_v5.0.0/toolchains/gcc_arm/12.2.mpacbti-rel1/bin/../lib/gcc/arm-none-eabi/12.2.1/thumb/v8-m.main+fp/hard\libg_nano.a(libc_a-utoa.o)
                0x00018a6c                __utoa
 .text.memset   0x00018af0       0x10 c:/renesas/ra/e2studio_v2023-10_fsp_v5.0.0/toolchains/gcc_arm/12.2.mpacbti-rel1/bin/../lib/gcc/arm-none-eabi/12.2.1/thumb/v8-m.main+fp/hard\libg_nano.a(libc_a-memset.o)
                0x00018af0                memset
 .text.__errno  0x00018b00        0xc c:/renesas/ra/e2studio_v2023-10_fsp_v5.0.0/toolchains/gcc_arm/12.2.mpacbti-rel1/bin/../lib/gcc/arm-none-eabi/12.2.1/thumb/v8-m.main+fp/hard\libg_nano.a(libc_a-errno.o)
                0x00018b00                __errno
 .text.strcpy   0x00018b0c       0x10 c:/renesas/ra/e2studio_v2023-10_fsp_v5.0.0/toolchains/gcc_arm/12.2.mpacbti-rel1/bin/../lib/gcc/arm-none-eabi/12.2.1/thumb/v8-m.main+fp/hard\libg_nano.a(libc_a-strcpy.o)
                0x00018b0c                strcpy
 .text.__aeabi_memcpy
                0x00018b1c        0x4 c:/renesas/ra/e2studio_v2023-10_fsp_v5.0.0/toolchains/gcc_arm/12.2.mpacbti-rel1/bin/../lib/gcc/arm-none-eabi/12.2.1/thumb/v8-m.main+fp/hard\libg_nano.a(libc_a-aeabi_memcpy.o)
                0x00018b1c                __aeabi_memcpy4
                0x00018b1c                __aeabi_memcpy8
                0x00018b1c                __aeabi_memcpy
 .text.__aeabi_memclr
                0x00018b20        0x6 c:/renesas/ra/e2studio_v2023-10_fsp_v5.0.0/toolchains/gcc_arm/12.2.mpacbti-rel1/bin/../lib/gcc/arm-none-eabi/12.2.1/thumb/v8-m.main+fp/hard\libg_nano.a(libc_a-aeabi_memclr.o)
                0x00018b20                __aeabi_memclr
                0x00018b20                __aeabi_memclr4
                0x00018b20                __aeabi_memclr8
 .text.memcpy   0x00018b26       0x1a c:/renesas/ra/e2studio_v2023-10_fsp_v5.0.0/toolchains/gcc_arm/12.2.mpacbti-rel1/bin/../lib/gcc/arm-none-eabi/12.2.1/thumb/v8-m.main+fp/hard\libg_nano.a(libc_a-memcpy-stub.o)
                0x00018b26                memcpy
 .text          0x00018b40       0x10 c:/renesas/ra/e2studio_v2023-10_fsp_v5.0.0/toolchains/gcc_arm/12.2.mpacbti-rel1/bin/../lib/gcc/arm-none-eabi/12.2.1/thumb/v8-m.main+fp/hard\libg_nano.a(libc_a-strlen.o)
                0x00018b40                strlen
 .text          0x00018b50       0x9a c:/renesas/ra/e2studio_v2023-10_fsp_v5.0.0/toolchains/gcc_arm/12.2.mpacbti-rel1/bin/../lib/gcc/arm-none-eabi/12.2.1/thumb/v8-m.main+fp/hard\libg_nano.a(libc_a-aeabi_memset-soft.o)
                0x00018b50                __aeabi_memset8
                0x00018b50                __aeabi_memset4
                0x00018b50                __aeabi_memset
 *(.version)
 *fill*         0x00018bea        0x2 ff
 .version       0x00018bec       0x50 ./ra/fsp/src/bsp/mcu/all/bsp_common.o
 *(.init)
 .init          0x00018c3c        0x4 c:/renesas/ra/e2studio_v2023-10_fsp_v5.0.0/toolchains/gcc_arm/12.2.mpacbti-rel1/bin/../lib/gcc/arm-none-eabi/12.2.1/thumb/v8-m.main+fp/hard/crti.o
                0x00018c3c                _init
 .init          0x00018c40        0x8 c:/renesas/ra/e2studio_v2023-10_fsp_v5.0.0/toolchains/gcc_arm/12.2.mpacbti-rel1/bin/../lib/gcc/arm-none-eabi/12.2.1/thumb/v8-m.main+fp/hard/crtn.o
 *(.fini)
 .fini          0x00018c48        0x4 c:/renesas/ra/e2studio_v2023-10_fsp_v5.0.0/toolchains/gcc_arm/12.2.mpacbti-rel1/bin/../lib/gcc/arm-none-eabi/12.2.1/thumb/v8-m.main+fp/hard/crti.o
                0x00018c48                _fini
 .fini          0x00018c4c        0x8 c:/renesas/ra/e2studio_v2023-10_fsp_v5.0.0/toolchains/gcc_arm/12.2.mpacbti-rel1/bin/../lib/gcc/arm-none-eabi/12.2.1/thumb/v8-m.main+fp/hard/crtn.o
 *crtbegin.o(.ctors)
 *crtbegin?.o(.ctors)
 *(EXCLUDE_FILE(*crtend.o *crtend?.o) .ctors)
 *(SORT_BY_NAME(.ctors.*))
 *(.ctors)
 *crtbegin.o(.dtors)
 *crtbegin?.o(.dtors)
 *(EXCLUDE_FILE(*crtend.o *crtend?.o) .dtors)
 *(SORT_BY_NAME(.dtors.*))
 *(.dtors)
 *(.rodata*)
 .rodata.interp_hvamp_1d
                0x00018c54       0x90 ./src/adc_temp.o
 .rodata.interp_ntc_1d
                0x00018ce4       0x58 ./src/adc_temp.o
 .rodata        0x00018d3c        0x5 ./src/angle.o
 *fill*         0x00018d41        0x3 ff
 .rodata.ItemInfo
                0x00018d44      0x840 ./src/control_table.o
                0x00018d44                ItemInfo
 .rodata.Default_ControlTable
                0x00019584      0x1a0 ./src/control_table.o
                0x00019584                Default_ControlTable
 .rodata.CRC8_SAE_J1850
                0x00019724      0x100 ./src/crc8.o
 .rodata.interp_current_compliance_ar_w
                0x00019824        0x4 ./src/global_variables.o
                0x00019824                interp_current_compliance_ar_w
 .rodata.interp_angle_compliance_ar_w
                0x00019828        0x4 ./src/global_variables.o
                0x00019828                interp_angle_compliance_ar_w
 .rodata.interp_tad2141_ar_w
                0x0001982c        0x4 ./src/global_variables.o
                0x0001982c                interp_tad2141_ar_w
 .rodata.pwm_gain.2
                0x00019830       0x14 ./src/hal_entry.o
 .rodata.baudrate_list
                0x00019844       0x3c ./src/hal_entry.o
                0x00019844                baudrate_list
 .rodata.concack.part.0.str1.4
                0x00019880       0x10 ./src/packet.o
 .rodata.concdec.part.0.str1.4
                0x00019890        0x2 ./src/packet.o
 *fill*         0x00019892        0x2 ff
 .rodata.cmd_vr.str1.4
                0x00019894        0x2 ./src/packet.o
 *fill*         0x00019896        0x2 ff
 .rodata.cmd_ct.str1.4
                0x00019898        0xc ./src/packet.o
 .rodata.packet_handling.str1.4
                0x000198a4        0x2 ./src/packet.o
 *fill*         0x000198a6        0x2 ff
 .rodata.ofs.1  0x000198a8        0x6 ./src/packet.o
 *fill*         0x000198ae        0x2 ff
 .rodata.ofs.2  0x000198b0        0x6 ./src/packet.o
 *fill*         0x000198b6        0x2 ff
 .rodata.ofs.3  0x000198b8        0x6 ./src/packet.o
 *fill*         0x000198be        0x2 ff
 .rodata.str1.4
                0x000198c0       0x10 ./src/packet.o
 .rodata.ak.4   0x000198d0       0x10 ./src/packet.o
 .rodata.gain.5
                0x000198e0        0x6 ./src/packet.o
 *fill*         0x000198e6        0x2 ff
 .rodata.CmdInfo
                0x000198e8      0x150 ./src/packet.o
 .rodata.SindegTable
                0x00019a38      0x70a ./src/sintable.o
 *fill*         0x0001a142        0x2 ff
 .rodata.g_ioport
                0x0001a144        0xc ./ra_gen/common_data.o
                0x0001a144                g_ioport
 .rodata.g_uart4_cfg
                0x0001a150       0x20 ./ra_gen/hal_data.o
                0x0001a150                g_uart4_cfg
 .rodata.g_uart4_cfg_extend
                0x0001a170       0x14 ./ra_gen/hal_data.o
                0x0001a170                g_uart4_cfg_extend
 .rodata.g_i2c3_cfg
                0x0001a184       0x28 ./ra_gen/hal_data.o
                0x0001a184                g_i2c3_cfg
 .rodata.g_i2c3_cfg_extend
                0x0001a1ac        0x6 ./ra_gen/hal_data.o
                0x0001a1ac                g_i2c3_cfg_extend
 *fill*         0x0001a1b2        0x2 ff
 .rodata.g_spi2_cfg
                0x0001a1b4       0x24 ./ra_gen/hal_data.o
                0x0001a1b4                g_spi2_cfg
 .rodata.g_spi2_cfg_extend
                0x0001a1d8        0x3 ./ra_gen/hal_data.o
                0x0001a1d8                g_spi2_cfg_extend
 *fill*         0x0001a1db        0x1 ff
 .rodata.g_transfer0
                0x0001a1dc        0xc ./ra_gen/hal_data.o
                0x0001a1dc                g_transfer0
 .rodata.g_transfer0_cfg
                0x0001a1e8        0x8 ./ra_gen/hal_data.o
                0x0001a1e8                g_transfer0_cfg
 .rodata.g_transfer0_cfg_extend
                0x0001a1f0        0x1 ./ra_gen/hal_data.o
                0x0001a1f0                g_transfer0_cfg_extend
 *fill*         0x0001a1f1        0x3 ff
 .rodata.g_transfer1
                0x0001a1f4        0xc ./ra_gen/hal_data.o
                0x0001a1f4                g_transfer1
 .rodata.g_transfer1_cfg
                0x0001a200        0x8 ./ra_gen/hal_data.o
                0x0001a200                g_transfer1_cfg
 .rodata.g_transfer1_cfg_extend
                0x0001a208        0x1 ./ra_gen/hal_data.o
                0x0001a208                g_transfer1_cfg_extend
 *fill*         0x0001a209        0x3 ff
 .rodata.g_timer5_cfg
                0x0001a20c       0x20 ./ra_gen/hal_data.o
                0x0001a20c                g_timer5_cfg
 .rodata.g_timer5_extend
                0x0001a22c       0x30 ./ra_gen/hal_data.o
                0x0001a22c                g_timer5_extend
 .rodata.g_timer0_cfg
                0x0001a25c       0x20 ./ra_gen/hal_data.o
                0x0001a25c                g_timer0_cfg
 .rodata.g_timer0_extend
                0x0001a27c        0x8 ./ra_gen/hal_data.o
                0x0001a27c                g_timer0_extend
 .rodata.g_adc0_channel_cfg
                0x0001a284       0x14 ./ra_gen/hal_data.o
                0x0001a284                g_adc0_channel_cfg
 .rodata.g_adc0_cfg
                0x0001a298       0x18 ./ra_gen/hal_data.o
                0x0001a298                g_adc0_cfg
 .rodata.g_adc0_cfg_extend
                0x0001a2b0        0xa ./ra_gen/hal_data.o
                0x0001a2b0                g_adc0_cfg_extend
 *fill*         0x0001a2ba        0x2 ff
 .rodata.g_flash0_cfg
                0x0001a2bc       0x14 ./ra_gen/hal_data.o
                0x0001a2bc                g_flash0_cfg
 .rodata.g_crc0_cfg
                0x0001a2d0        0xc ./ra_gen/hal_data.o
                0x0001a2d0                g_crc0_cfg
 .rodata.g_bsp_pin_cfg
                0x0001a2dc        0xc ./ra_gen/pin_data.o
                0x0001a2dc                g_bsp_pin_cfg
 .rodata.g_bsp_pin_cfg_data
                0x0001a2e8       0x98 ./ra_gen/pin_data.o
                0x0001a2e8                g_bsp_pin_cfg_data
 .rodata.g_interrupt_event_link_select
                0x0001a380       0xc0 ./ra_gen/vector_data.o
                0x0001a380                g_interrupt_event_link_select
 .rodata.g_div_coefficient
                0x0001a440       0x1a ./ra/fsp/src/r_sci_uart/r_sci_uart.o
 *fill*         0x0001a45a        0x2 ff
 .rodata.g_async_baud
                0x0001a45c        0xd ./ra/fsp/src/r_sci_uart/r_sci_uart.o
 *fill*         0x0001a469        0x3 ff
 .rodata.g_ioport_on_ioport
                0x0001a46c       0x34 ./ra/fsp/src/r_ioport/r_ioport.o
                0x0001a46c                g_ioport_on_ioport
 .rodata.g_transfer_on_dtc
                0x0001a4a0       0x28 ./ra/fsp/src/r_dtc/r_dtc.o
                0x0001a4a0                g_transfer_on_dtc
 .rodata.adc_elc_trigger_lut
                0x0001a4c8        0xc ./ra/fsp/src/r_adc/r_adc.o
 .rodata.g_prcr_masks
                0x0001a4d4        0x8 ./ra/fsp/src/bsp/mcu/all/bsp_register_protection.o
 .rodata.__utoa.str1.1
                0x0001a4dc       0x25 c:/renesas/ra/e2studio_v2023-10_fsp_v5.0.0/toolchains/gcc_arm/12.2.mpacbti-rel1/bin/../lib/gcc/arm-none-eabi/12.2.1/thumb/v8-m.main+fp/hard\libg_nano.a(libc_a-utoa.o)
 .rodata._ctype_
                0x0001a501      0x101 c:/renesas/ra/e2studio_v2023-10_fsp_v5.0.0/toolchains/gcc_arm/12.2.mpacbti-rel1/bin/../lib/gcc/arm-none-eabi/12.2.1/thumb/v8-m.main+fp/hard\libg_nano.a(libc_a-ctype_.o)
                0x0001a501                _ctype_
                0x0001a602                        __usb_dev_descriptor_start_fs = .
 *(.usb_device_desc_fs*)
                0x0001a602                        __usb_cfg_descriptor_start_fs = .
 *(.usb_config_desc_fs*)
                0x0001a602                        __usb_interface_descriptor_start_fs = .
 *(.usb_interface_desc_fs*)
                0x0001a602                        __usb_descriptor_end_fs = .
                0x0001a602                        __usb_dev_descriptor_start_hs = .
 *(.usb_device_desc_hs*)
                0x0001a602                        __usb_cfg_descriptor_start_hs = .
 *(.usb_config_desc_hs*)
                0x0001a602                        __usb_interface_descriptor_start_hs = .
 *(.usb_interface_desc_hs*)
                0x0001a602                        __usb_descriptor_end_hs = .
 *(.eh_frame*)
 *fill*         0x0001a602        0x2 ff
 .eh_frame      0x0001a604        0x0 c:/renesas/ra/e2studio_v2023-10_fsp_v5.0.0/toolchains/gcc_arm/12.2.mpacbti-rel1/bin/../lib/gcc/arm-none-eabi/12.2.1/thumb/v8-m.main+fp/hard/crtbegin.o
 .eh_frame      0x0001a604       0x28 c:/renesas/ra/e2studio_v2023-10_fsp_v5.0.0/toolchains/gcc_arm/12.2.mpacbti-rel1/bin/../lib/gcc/arm-none-eabi/12.2.1/thumb/v8-m.main+fp/hard\libg_nano.a(libc_a-strlen.o)
 .eh_frame      0x0001a62c       0x38 c:/renesas/ra/e2studio_v2023-10_fsp_v5.0.0/toolchains/gcc_arm/12.2.mpacbti-rel1/bin/../lib/gcc/arm-none-eabi/12.2.1/thumb/v8-m.main+fp/hard\libg_nano.a(libc_a-aeabi_memset-soft.o)
 .eh_frame      0x0001a664        0x4 c:/renesas/ra/e2studio_v2023-10_fsp_v5.0.0/toolchains/gcc_arm/12.2.mpacbti-rel1/bin/../lib/gcc/arm-none-eabi/12.2.1/thumb/v8-m.main+fp/hard/crtend.o
                0x0001a668                        __ROM_End = .
                0x000001c0                        __Vectors_Size = (__Vectors_End - __Vectors)

.glue_7         0x0001a668        0x0
 .glue_7        0x0001a668        0x0 linker stubs

.glue_7t        0x0001a668        0x0
 .glue_7t       0x0001a668        0x0 linker stubs

.vfp11_veneer   0x0001a668        0x0
 .vfp11_veneer  0x0001a668        0x0 linker stubs

.v4_bx          0x0001a668        0x0
 .v4_bx         0x0001a668        0x0 linker stubs

.iplt           0x0001a668        0x0
 .iplt          0x0001a668        0x0 c:/renesas/ra/e2studio_v2023-10_fsp_v5.0.0/toolchains/gcc_arm/12.2.mpacbti-rel1/bin/../lib/gcc/arm-none-eabi/12.2.1/thumb/v8-m.main+fp/hard/crtbegin.o
                0x0001a668                        . = .
                0x0001a668                        __itcm_data_pre_location = .

.itcm_data      0x00000000        0x0 load address 0x0001a670
                0x00000000                        __tz_ITCM_S = ABSOLUTE (ITCM_START)
                0x00000000                        __itcm_data_start = .
 *(.itcm_data*)
                0x00000000                        . = ALIGN (0x8)
                0x00000000                        __itcm_data_end = .
                0x00000000                        __tz_ITCM_N = DEFINED (ITCM_NS_START)?ABSOLUTE (ITCM_NS_START):ALIGN (__itcm_data_end, 0x2000)
                0x0001a670                        __itcm_data_init_start = LOADADDR (.itcm_data)
                0x0001a670                        __itcm_data_init_end = (LOADADDR (.itcm_data) + SIZEOF (.itcm_data))
                0x00000001                        ASSERT (((ORIGIN (ITCM) % 0x8) == 0x0), ITCM memory region origin must be aligned to 8 bytes.)
                0x00000001                        ASSERT (((LENGTH (ITCM) % 0x8) == 0x0), ITCM memory region length must be a multiple of 8 bytes.)
                0x00000001                        ASSERT (((LOADADDR (.itcm_data) % 0x10) == 0x0), .itcm_data section must be aligned to 16 bytes.)
                0x00000001                        ASSERT (((SIZEOF (.itcm_data) % 0x8) == 0x0), .itcm_data section size must be a multiple of 8 bytes.)
                0x0001a668                        . = (SIZEOF (.itcm_data) > 0x0)?__itcm_data_init_end:__itcm_data_pre_location
                0x0001a668                        __exidx_start = .

/DISCARD/
 *(.ARM.extab* .gnu.linkonce.armextab.*)
 *(.ARM.exidx* .gnu.linkonce.armexidx.*)
                0x0001a668                        __exidx_end = .
                0x0001a668                        __etext = .
                0x20000000                        __tz_RAM_S = ORIGIN (RAM)

.fsp_dtc_vector_table
                0x20000000      0x180
                0x20000000                        . = ORIGIN (RAM)
 *(.fsp_dtc_vector_table)
 .fsp_dtc_vector_table
                0x20000000      0x180 ./ra/fsp/src/r_dtc/r_dtc.o

.data           0x20000180      0x2e8 load address 0x0001a668
                0x20000180                        __data_start__ = .
                0x20000180                        . = ALIGN (0x4)
                0x20000180                        __Code_In_RAM_Start = .
 *(.code_in_ram*)
                0x20000180                        __Code_In_RAM_End = .
 *(vtable)
 *(.data.*)
 .data.g_wait_count
                0x20000180        0x4 ./src/angle.o
 *fill*         0x20000184        0x4 
 .data.pidparam_cur
                0x20000188       0x50 ./src/global_variables.o
                0x20000188                pidparam_cur
 .data.pidparam_velo
                0x200001d8       0x50 ./src/global_variables.o
                0x200001d8                pidparam_velo
 .data.pidparam_ang
                0x20000228       0x50 ./src/global_variables.o
                0x20000228                pidparam_ang
 .data.interp_current_compliance_1d
                0x20000278       0x20 ./src/global_variables.o
                0x20000278                interp_current_compliance_1d
 .data.interp_angle_compliance_1d
                0x20000298       0x20 ./src/global_variables.o
                0x20000298                interp_angle_compliance_1d
 .data.interp_tad2141_1d
                0x200002b8      0x128 ./src/global_variables.o
                0x200002b8                interp_tad2141_1d
 .data.prev_moncon.1
                0x200003e0        0x1 ./src/hal_entry.o
 .data.isl28022_targetreg.23
                0x200003e1        0x1 ./src/hal_entry.o
 *fill*         0x200003e2        0x2 
 .data.PreviousID
                0x200003e4        0x4 ./src/packet.o
 .data.txcomp   0x200003e8        0x1 ./src/usart.o
 *fill*         0x200003e9        0x3 
 .data.g_uart4_baud_setting
                0x200003ec        0x4 ./ra_gen/hal_data.o
                0x200003ec                g_uart4_baud_setting
 .data.g_transfer0_info
                0x200003f0       0x10 ./ra_gen/hal_data.o
                0x200003f0                g_transfer0_info
 .data.g_transfer1_info
                0x20000400       0x10 ./ra_gen/hal_data.o
                0x20000400                g_transfer1_info
 .data._impure_ptr
                0x20000410        0x4 c:/renesas/ra/e2studio_v2023-10_fsp_v5.0.0/toolchains/gcc_arm/12.2.mpacbti-rel1/bin/../lib/gcc/arm-none-eabi/12.2.1/thumb/v8-m.main+fp/hard\libg_nano.a(libc_a-impure.o)
                0x20000410                _impure_ptr
 .data._impure_data
                0x20000414       0x4c c:/renesas/ra/e2studio_v2023-10_fsp_v5.0.0/toolchains/gcc_arm/12.2.mpacbti-rel1/bin/../lib/gcc/arm-none-eabi/12.2.1/thumb/v8-m.main+fp/hard\libg_nano.a(libc_a-impure.o)
                0x20000414                _impure_data
 *(.data)
                0x20000460                        . = ALIGN (0x4)
                0x20000460                        PROVIDE (__preinit_array_start = .)
 *(.preinit_array)
                0x20000460                        PROVIDE (__preinit_array_end = .)
                0x20000460                        . = ALIGN (0x4)
                0x20000460                        PROVIDE (__init_array_start = .)
 *(SORT_BY_NAME(.init_array.*))
 *(.init_array)
 .init_array    0x20000460        0x4 c:/renesas/ra/e2studio_v2023-10_fsp_v5.0.0/toolchains/gcc_arm/12.2.mpacbti-rel1/bin/../lib/gcc/arm-none-eabi/12.2.1/thumb/v8-m.main+fp/hard/crtbegin.o
                0x20000464                        PROVIDE (__init_array_end = .)
                0x20000464                        . = ALIGN (0x4)
                [!provide]                        PROVIDE (__fini_array_start = .)
 *(SORT_BY_NAME(.fini_array.*))
 *(.fini_array)
 .fini_array    0x20000464        0x4 c:/renesas/ra/e2studio_v2023-10_fsp_v5.0.0/toolchains/gcc_arm/12.2.mpacbti-rel1/bin/../lib/gcc/arm-none-eabi/12.2.1/thumb/v8-m.main+fp/hard/crtbegin.o
                [!provide]                        PROVIDE (__fini_array_end = .)
 *(.jcr*)
                0x20000468                        . = ALIGN (0x4)
                0x20000468                        __data_end__ = .

.tm_clone_table
                0x20000468        0x0 load address 0x0001a950
 .tm_clone_table
                0x20000468        0x0 c:/renesas/ra/e2studio_v2023-10_fsp_v5.0.0/toolchains/gcc_arm/12.2.mpacbti-rel1/bin/../lib/gcc/arm-none-eabi/12.2.1/thumb/v8-m.main+fp/hard/crtbegin.o
 .tm_clone_table
                0x20000468        0x0 c:/renesas/ra/e2studio_v2023-10_fsp_v5.0.0/toolchains/gcc_arm/12.2.mpacbti-rel1/bin/../lib/gcc/arm-none-eabi/12.2.1/thumb/v8-m.main+fp/hard/crtend.o

.igot.plt       0x20000468        0x0 load address 0x0001a950
 .igot.plt      0x20000468        0x0 c:/renesas/ra/e2studio_v2023-10_fsp_v5.0.0/toolchains/gcc_arm/12.2.mpacbti-rel1/bin/../lib/gcc/arm-none-eabi/12.2.1/thumb/v8-m.main+fp/hard/crtbegin.o
                0x20000468                        . = .
                0x0001a950                        __dtcm_data_pre_location = (LOADADDR (.data) + SIZEOF (.data))

.dtcm_data      0x00000000        0x0 load address 0x0001a950
                0x00000000                        __tz_DTCM_S = ABSOLUTE (DTCM_START)
                0x00000000                        __dtcm_data_start = .
 *(.dtcm_data*)
                0x00000000                        . = ALIGN (0x8)
                0x00000000                        __dtcm_data_end = .
                0x00000000                        . = __dtcm_data_end

.dtcm_bss       0x00000000        0x0
                0x00000000                        __dtcm_bss_start = .
 *(.dtcm_bss*)
                0x00000000                        . = ALIGN (0x8)
                0x00000000                        __dtcm_bss_end = .
                0x00000000                        __tz_DTCM_N = DEFINED (DTCM_NS_START)?ABSOLUTE (DTCM_NS_START):ALIGN (__dtcm_bss_end, 0x2000)
                0x0001a950                        __dtcm_data_init_start = LOADADDR (.dtcm_data)
                0x0001a950                        __dtcm_data_init_end = (LOADADDR (.dtcm_data) + SIZEOF (.dtcm_data))
                0x00000001                        ASSERT (((ORIGIN (DTCM) % 0x8) == 0x0), DTCM memory region origin must be aligned to 8 bytes.)
                0x00000001                        ASSERT (((LENGTH (DTCM) % 0x8) == 0x0), DTCM memory region length must be a multiple of 8 bytes.)
                0x00000001                        ASSERT ((LOADADDR (.dtcm_bss) == ADDR (.dtcm_bss)), .dtcm_bss has (VMA != LMA) but should be NOLOAD (VMA == LMA).)
                0x00000001                        ASSERT (((LOADADDR (.dtcm_data) % 0x10) == 0x0), .dtcm_data section must be aligned to 16 bytes.)
                0x00000001                        ASSERT (((SIZEOF (.dtcm_data) % 0x8) == 0x0), .dtcm_data section size must be a multiple of 8 bytes.)
                0x00000001                        ASSERT (((LOADADDR (.dtcm_bss) % 0x8) == 0x0), .dtcm_bss section must be aligned to 8 bytes.)
                0x00000001                        ASSERT (((SIZEOF (.dtcm_bss) % 0x8) == 0x0), .dtcm_bss section size must be a multiple of 8 bytes.)
                0x00000001                        ASSERT ((__dtcm_bss_start == __dtcm_data_end), .dtcm_bss section is not adjacent to .dtcm_data section.)
                0x0001a950                        . = (SIZEOF (.dtcm_data) > 0x0)?__dtcm_data_init_end:__dtcm_data_pre_location
                0x0001a950                        sgstubs_pre_location = .
                0x0001ac00                        SGSTUBS_LOC = (DEFINED (PROJECT_SECURE) && DEFINED (FLASH_NSC_START))?ABSOLUTE (FLASH_NSC_START):ALIGN (0x400)

.gnu.sgstubs    0x0001ac00        0x0
                0x0001ac00                        __tz_FLASH_C = DEFINED (FLASH_NSC_START)?ABSOLUTE (FLASH_NSC_START):__RESERVE_NS_RAM?ABSOLUTE ((FLASH_START + FLASH_LENGTH)):ALIGN (0x400)
                0x0001ac00                        _start_sg = .
 *(.gnu.sgstubs*)
                0x0001ac00                        . = ALIGN (0x20)
                0x0001ac00                        _end_sg = .
                0x00020000                        __tz_FLASH_N = DEFINED (FLASH_NS_START)?ABSOLUTE (FLASH_NS_START):__RESERVE_NS_RAM?ABSOLUTE ((FLASH_START + FLASH_LENGTH)):(FLASH_LENGTH < 0x8000)?FLASH_LENGTH:ALIGN (0x8000)
                0x00020000                        FLASH_NS_IMAGE_START = DEFINED (FLASH_NS_IMAGE_START)?FLASH_NS_IMAGE_START:__tz_FLASH_N
                0x60000000                        __tz_QSPI_FLASH_S = ORIGIN (QSPI_FLASH)

.qspi_flash     0x60000000        0x0
                0x60000000                        __qspi_flash_start__ = .
 *(.qspi_flash*)
 *(.code_in_qspi*)
                0x60000000                        __qspi_flash_end__ = .
                0x00000000                        __qspi_flash_code_size__ = (__qspi_flash_end__ - __qspi_flash_start__)
                0x0001a950                        __qspi_flash_code_addr__ = sgstubs_pre_location

.qspi_non_retentive
                0x60000000        0x0 load address 0x0001a950
                0x60000000                        __qspi_non_retentive_start__ = .
 *(.qspi_non_retentive*)
                0x60000000                        __qspi_non_retentive_end__ = .
                0x00000000                        __qspi_non_retentive_size__ = (__qspi_non_retentive_end__ - __qspi_non_retentive_start__)
                0x04000000                        __qspi_region_max_size__ = 0x4000000
                0x60000000                        __qspi_region_start_address__ = __qspi_flash_start__
                0x64000000                        __qspi_region_end_address__ = (__qspi_flash_start__ + __qspi_region_max_size__)
                0x60000000                        __tz_QSPI_FLASH_N = __qspi_non_retentive_end__

.OSPI_DEVICE_0_NO_LOAD
                0x80020000        0x0
                0x80020000                        . = ALIGN (0x4)
                0x80020000                        __ospi_device_0_start__ = .
 *(.ospi_device_0_no_load*)
                0x80020000                        . = ALIGN (0x4)
                0x80020000                        __ospi_device_0_end__ = .

.OSPI_DEVICE_1_NO_LOAD
                0x80030000        0x0
                0x80030000                        . = ALIGN (0x4)
                0x80030000                        __ospi_device_1_start__ = .
 *(.ospi_device_1_no_load*)
                0x80030000                        . = ALIGN (0x4)
                0x80030000                        __ospi_device_1_end__ = .
                0x80020000                        __tz_OSPI_DEVICE_0_S = ORIGIN (OSPI_DEVICE_0)

.OSPI_DEVICE_0  0x80020000        0x0
                0x80020000                        __ospi_device_0_start__ = .
 *(.ospi_device_0*)
 *(.code_in_ospi_device_0*)
                0x80020000                        __ospi_device_0_end__ = .
                0x00000000                        __ospi_device_0_code_size__ = (__ospi_device_0_end__ - __ospi_device_0_start__)
                0x0001a950                        __ospi_device_0_code_addr__ = (sgstubs_pre_location + SIZEOF (.qspi_non_retentive))

.ospi_device_0_non_retentive
                0x80020000        0x0 load address 0x0001a950
                0x80020000                        __ospi_device_0_non_retentive_start__ = .
 *(.ospi_device_0_non_retentive*)
                0x80020000                        __ospi_device_0_non_retentive_end__ = .
                0x00000000                        __ospi_device_0_non_retentive_size__ = (__ospi_device_0_non_retentive_end__ - __ospi_device_0_non_retentive_start__)
                0x08000000                        __ospi_device_0_region_max_size__ = 0x8000000
                0x80020000                        __ospi_device_0_region_start_address__ = __ospi_device_0_start__
                0x88020000                        __ospi_device_0_region_end_address__ = (__ospi_device_0_start__ + __ospi_device_0_region_max_size__)
                0x80020000                        __tz_OSPI_DEVICE_0_N = __ospi_device_0_non_retentive_end__
                0x80030000                        __tz_OSPI_DEVICE_1_S = ORIGIN (OSPI_DEVICE_1)

.OSPI_DEVICE_1  0x80030000        0x0
                0x80030000                        __ospi_device_1_start__ = .
 *(.ospi_device_1*)
 *(.code_in_ospi_device_1*)
                0x80030000                        __ospi_device_1_end__ = .
                0x00000000                        __ospi_device_1_code_size__ = (__ospi_device_1_end__ - __ospi_device_1_start__)
                0x0001a950                        __ospi_device_1_code_addr__ = (sgstubs_pre_location + (SIZEOF (.qspi_non_retentive) + SIZEOF (.ospi_device_0_non_retentive)))

.ospi_device_1_non_retentive
                0x80030000        0x0 load address 0x0001a950
                0x80030000                        __ospi_device_1_non_retentive_start__ = .
 *(.ospi_device_1_non_retentive*)
                0x80030000                        __ospi_device_1_non_retentive_end__ = .
                0x00000000                        __ospi_device_1_non_retentive_size__ = (__ospi_device_1_non_retentive_end__ - __ospi_device_1_non_retentive_start__)
                0x10000000                        __ospi_device_1_region_max_size__ = 0x10000000
                0x80030000                        __ospi_device_1_region_start_address__ = __ospi_device_1_start__
                0x90030000                        __ospi_device_1_region_end_address__ = (__ospi_device_1_start__ + __ospi_device_1_region_max_size__)
                0x80030000                        __tz_OSPI_DEVICE_1_N = __ospi_device_1_non_retentive_end__

.noinit         0x20000468       0x20
                0x20000468                        . = ALIGN (0x4)
                0x20000468                        __noinit_start = .
 *(.noinit*)
 .noinit        0x20000468       0x1c ./ra/fsp/src/bsp/mcu/all/bsp_clocks.o
                0x20000488                        . = ALIGN (0x8)
 *fill*         0x20000484        0x4 
 *(.heap.*)
                0x20000488                        __noinit_end = .

.bss            0x20000488     0x3b4c
                0x20000488                        . = ALIGN (0x4)
                0x20000488                        __bss_start__ = .
 *(.bss*)
 .bss.completed.1
                0x20000488        0x1 c:/renesas/ra/e2studio_v2023-10_fsp_v5.0.0/toolchains/gcc_arm/12.2.mpacbti-rel1/bin/../lib/gcc/arm-none-eabi/12.2.1/thumb/v8-m.main+fp/hard/crtbegin.o
 *fill*         0x20000489        0x3 
 .bss.object.0  0x2000048c       0x18 c:/renesas/ra/e2studio_v2023-10_fsp_v5.0.0/toolchains/gcc_arm/12.2.mpacbti-rel1/bin/../lib/gcc/arm-none-eabi/12.2.1/thumb/v8-m.main+fp/hard/crtbegin.o
 *fill*         0x200004a4        0x4 
 .bss.adc_value
                0x200004a8       0x18 ./src/adc_temp.o
 .bss.spi_master_event
                0x200004c0        0x1 ./src/angle.o
 *fill*         0x200004c1        0x3 
 .bss.ControlTable
                0x200004c4      0x1a0 ./src/control_table.o
                0x200004c4                ControlTable
 .bss.UpdateTargetValue
                0x20000664        0x1 ./src/global_variables.o
                0x20000664                UpdateTargetValue
 *fill*         0x20000665        0x3 
 .bss.packet.0  0x20000668      0x7d0 ./src/hal_entry.o
 .bss.MonCount.3
                0x20000e38        0x2 ./src/hal_entry.o
 *fill*         0x20000e3a        0x2 
 .bss.StartCurrent.4
                0x20000e3c        0x4 ./src/hal_entry.o
 .bss.prev_targetcurrent.5
                0x20000e40        0x4 ./src/hal_entry.o
 .bss.StartVelocity.6
                0x20000e44        0x4 ./src/hal_entry.o
 .bss.prev_targetvelocity.7
                0x20000e48        0x4 ./src/hal_entry.o
 .bss.LimitedTargetAngle.8
                0x20000e4c        0x4 ./src/hal_entry.o
 .bss.StartAngle.9
                0x20000e50        0x4 ./src/hal_entry.o
 .bss.TransitionTime.10
                0x20000e54        0x4 ./src/hal_entry.o
 .bss.prev_set_transition_mode.11
                0x20000e58        0x1 ./src/hal_entry.o
 *fill*         0x20000e59        0x3 
 .bss.prev_set_transition_time.12
                0x20000e5c        0x4 ./src/hal_entry.o
 .bss.prev_targetangle.13
                0x20000e60        0x4 ./src/hal_entry.o
 .bss.ex14_targetangle.14
                0x20000e64        0x4 ./src/hal_entry.o
 .bss.TargetCurrent.15
                0x20000e68        0x4 ./src/hal_entry.o
 .bss.TargetVelocity.16
                0x20000e6c        0x4 ./src/hal_entry.o
 .bss.stall.17  0x20000e70        0x1 ./src/hal_entry.o
 *fill*         0x20000e71        0x3 
 .bss.TargetAngle.18
                0x20000e74        0x4 ./src/hal_entry.o
 .bss.prevmode.19
                0x20000e78        0x1 ./src/hal_entry.o
 *fill*         0x20000e79        0x7 
 .bss.current.20
                0x20000e80        0x8 ./src/hal_entry.o
 .bss.stat_cur.21
                0x20000e88        0x8 ./src/hal_entry.o
 .bss.isl28022_read_data.22
                0x20000e90        0x2 ./src/hal_entry.o
 .bss.angle_depth.24
                0x20000e92        0x1 ./src/hal_entry.o
 .bss.led_stat  0x20000e93        0x1 ./src/hal_entry.o
 .bss.ang_history
                0x20000e94       0x80 ./src/hal_entry.o
 .bss.ang_ex    0x20000f14        0x4 ./src/hal_entry.o
 .bss.now_ang   0x20000f18        0x4 ./src/hal_entry.o
 .bss.prev_ang  0x20000f1c        0x4 ./src/hal_entry.o
 .bss.rxb       0x20000f20      0xfa0 ./src/hal_entry.o
 .bss.txb       0x20001ec0      0xfa0 ./src/hal_entry.o
 .bss.cmd_r.0   0x20002e60      0x3e8 ./src/packet.o
 .bss.hostcrc   0x20003248        0x1 ./src/packet.o
 .bss.MakeAck   0x20003249        0x1 ./src/packet.o
 .bss.AckSend   0x2000324a        0x1 ./src/packet.o
 *fill*         0x2000324b        0x1 
 .bss.Ack       0x2000324c      0x7d0 ./src/packet.o
 .bss.MachedID  0x20003a1c        0x1 ./src/packet.o
 *fill*         0x20003a1d        0x3 
 .bss.FlagOfIDs
                0x20003a20      0x100 ./src/packet.o
 .bss.packet_req_init_id_baud
                0x20003b20        0x1 ./src/packet.o
                0x20003b20                packet_req_init_id_baud
 .bss.packet_req_initalize
                0x20003b21        0x1 ./src/packet.o
                0x20003b21                packet_req_initalize
 *fill*         0x20003b22        0x2 
 .bss.rreg.1    0x20003b24        0x4 ./src/power_monitor.o
 .bss.dat.0     0x20003b28        0x3 ./src/power_monitor.o
 .bss.i2c_stat  0x20003b2b        0x1 ./src/power_monitor.o
 .bss.iic_pstat
                0x20003b2c        0x1 ./src/power_monitor.o
 *fill*         0x20003b2d        0x3 
 .bss.isl28022_destreaddata
                0x20003b30        0x4 ./src/power_monitor.o
 .bss.FIFO      0x20003b34       0x18 ./src/usart.o
 .bss.g_ioport_ctrl
                0x20003b4c        0x8 ./ra_gen/common_data.o
                0x20003b4c                g_ioport_ctrl
 .bss.g_uart4_ctrl
                0x20003b54       0x30 ./ra_gen/hal_data.o
                0x20003b54                g_uart4_ctrl
 .bss.g_i2c3_ctrl
                0x20003b84       0x40 ./ra_gen/hal_data.o
                0x20003b84                g_i2c3_ctrl
 .bss.g_spi2_ctrl
                0x20003bc4       0x2c ./ra_gen/hal_data.o
                0x20003bc4                g_spi2_ctrl
 .bss.g_transfer0_ctrl
                0x20003bf0        0x8 ./ra_gen/hal_data.o
                0x20003bf0                g_transfer0_ctrl
 .bss.g_transfer1_ctrl
                0x20003bf8        0x8 ./ra_gen/hal_data.o
                0x20003bf8                g_transfer1_ctrl
 .bss.g_timer5_ctrl
                0x20003c00       0x20 ./ra_gen/hal_data.o
                0x20003c00                g_timer5_ctrl
 .bss.g_timer0_ctrl
                0x20003c20       0x20 ./ra_gen/hal_data.o
                0x20003c20                g_timer0_ctrl
 .bss.g_adc0_ctrl
                0x20003c40       0x24 ./ra_gen/hal_data.o
                0x20003c40                g_adc0_ctrl
 .bss.g_flash0_ctrl
                0x20003c64       0x44 ./ra_gen/hal_data.o
                0x20003c64                g_flash0_ctrl
 .bss.g_crc0_ctrl
                0x20003ca8        0x8 ./ra_gen/hal_data.o
                0x20003ca8                g_crc0_ctrl
 .bss.tx_dummy.0
                0x20003cb0        0x1 ./ra/fsp/src/r_sci_spi/r_sci_spi.o
 .bss.g_dtc_state_initialized.0
                0x20003cb1        0x1 ./ra/fsp/src/r_dtc/r_dtc.o
 *fill*         0x20003cb2        0x2 
 .bss.gp_prv_agt_periods
                0x20003cb4       0x18 ./ra/fsp/src/r_agt/r_agt.o
 .bss.g_bsp_group_irq_sources
                0x20003ccc       0x40 ./ra/fsp/src/bsp/mcu/all/bsp_group_irq.o
                0x20003ccc                g_bsp_group_irq_sources
 .bss.g_protect_pfswe_counter
                0x20003d0c        0x4 ./ra/fsp/src/bsp/mcu/all/bsp_io.o
                0x20003d0c                g_protect_pfswe_counter
 .bss.gp_renesas_isr_context
                0x20003d10      0x180 ./ra/fsp/src/bsp/mcu/all/bsp_irq.o
                0x20003d10                gp_renesas_isr_context
 .bss.g_protect_counters
                0x20003e90        0x8 ./ra/fsp/src/bsp/mcu/all/bsp_register_protection.o
                0x20003e90                g_protect_counters
 .bss.SystemCoreClock
                0x20003e98        0x4 ./ra/fsp/src/bsp/cmsis/Device/RENESAS/Source/system.o
                0x20003e98                SystemCoreClock
 .bss.__sf      0x20003e9c      0x138 c:/renesas/ra/e2studio_v2023-10_fsp_v5.0.0/toolchains/gcc_arm/12.2.mpacbti-rel1/bin/../lib/gcc/arm-none-eabi/12.2.1/thumb/v8-m.main+fp/hard\libg_nano.a(libc_a-findfp.o)
                0x20003e9c                __sf
 *(COMMON)
                0x20003fd4                        . = ALIGN (0x4)
                0x20003fd4                        __bss_end__ = .

.heap           0x20003fd4        0x4
                0x20003fd8                        . = ALIGN (0x8)
 *fill*         0x20003fd4        0x4 
                0x20003fd8                        __HeapBase = .
 *(.heap)
                0x20003fd8                        __HeapLimit = .

.stack_dummy    0x20003fd8     0x1000
                0x20003fd8                        . = ALIGN (0x8)
                0x20003fd8                        __StackLimit = .
 *(.stack)
 .stack         0x20003fd8     0x1000 ./ra/fsp/src/bsp/cmsis/Device/RENESAS/Source/startup.o
                0x20004fd8                        __StackTop = .
 *(.stack*)
                0x20004fd8                        __StackTopAll = .
                0x20004fd8                        PROVIDE (__stack = __StackTopAll)
                0x20004fd8                        __RAM_segment_used_end__ = ALIGN (__StackTopAll, 0x4)
                0x20005000                        __tz_RAM_C = DEFINED (RAM_NSC_START)?ABSOLUTE ((RAM_NSC_START - RAM_NS_BUFFER_BLOCK_LENGTH)):__RESERVE_NS_RAM?ABSOLUTE (RAM_NS_BUFFER_BLOCK_START):ALIGN (__RAM_segment_used_end__, 0x400)
                0x20006000                        __tz_RAM_N = DEFINED (RAM_NS_START)?ABSOLUTE ((RAM_NS_START - RAM_NS_BUFFER_BLOCK_LENGTH)):__RESERVE_NS_RAM?ABSOLUTE (RAM_NS_BUFFER_BLOCK_START):ALIGN (__tz_RAM_C, 0x2000)

.ns_buffer      0x20004fd8        0x0
                0x20004fd8                        . = __RESERVE_NS_RAM?ABSOLUTE ((RAM_NS_BUFFER_START & 0xffffffe0)):.
 *(.ns_buffer*)

.data_flash     0x08000000        0x0
                0x08000000                        . = ORIGIN (DATA_FLASH)
                0x08000000                        __tz_DATA_FLASH_S = .
                0x08000000                        __Data_Flash_Start = .
 *(.data_flash*)
                0x08000000                        __Data_Flash_End = .
                0x08000000                        __tz_DATA_FLASH_N = DEFINED (DATA_FLASH_NS_START)?ABSOLUTE (DATA_FLASH_NS_START):__RESERVE_NS_RAM?ABSOLUTE ((DATA_FLASH_START + DATA_FLASH_LENGTH)):ALIGN (0x400)
                0x80010000                        __tz_SDRAM_S = ORIGIN (SDRAM)

.sdram          0x80010000        0x0
                0x80010000                        __SDRAM_Start = .
 *(.sdram*)
 *(.frame*)
                0x80010000                        __SDRAM_End = .
                0x80010000                        __tz_SDRAM_N = __SDRAM_End
                0x00000000                        __tz_ID_CODE_S = ORIGIN (ID_CODE)
                0x00000000                        __tz_ID_CODE_N = __tz_ID_CODE_S

.id_code        0x00000000        0x0
                0x00000000                        __ID_Code_Start = .
 *(.id_code*)
                0x00000000                        __ID_Code_End = .
                0x0100a100                        __tz_OPTION_SETTING_S = ORIGIN (OPTION_SETTING_OFS)

.option_setting_ofs
                0x0100a100       0x10
                0x0100a100                        __OPTION_SETTING_OFS_Start = .
 *(.option_setting_ofs0)
 .option_setting_ofs0
                0x0100a100        0x4 ./ra/fsp/src/bsp/mcu/all/bsp_rom_registers.o
                0x0100a104                        . = PROJECT_SECURE_OR_FLAT?(__OPTION_SETTING_OFS_Start + 0x4):__OPTION_SETTING_OFS_Start
 *(.option_setting_ofs2)
                0x0100a110                        . = PROJECT_SECURE_OR_FLAT?(__OPTION_SETTING_OFS_Start + 0x10):__OPTION_SETTING_OFS_Start
 *fill*         0x0100a104        0xc ff
 *(.option_setting_dualsel)
                0x0100a110                        __OPTION_SETTING_OFS_End = .

.option_setting_sas
                0x0100a134        0x4
                0x0100a134                        __OPTION_SETTING_SAS_Start = .
 *(.option_setting_sas)
 .option_setting_sas
                0x0100a134        0x4 ./ra/fsp/src/bsp/mcu/all/bsp_rom_registers.o
                0x0100a138                        __OPTION_SETTING_SAS_End = .
                0x0100a180                        __tz_OPTION_SETTING_N = ABSOLUTE (OPTION_SETTING_START_NS)

.option_setting_ns
                0x0100a100        0x0
                0x0100a100                        __OPTION_SETTING_NS_Start = .
 *(.option_setting_ofs1)
                0x0100a100                        . = USE_OPTION_SETTING_NS?(__OPTION_SETTING_NS_Start + 0x4):__OPTION_SETTING_NS_Start
 *(.option_setting_ofs3)
                0x0100a100                        . = USE_OPTION_SETTING_NS?(__OPTION_SETTING_NS_Start + 0x10):__OPTION_SETTING_NS_Start
 *(.option_setting_banksel)
                0x0100a100                        . = USE_OPTION_SETTING_NS?(__OPTION_SETTING_NS_Start + 0x40):__OPTION_SETTING_NS_Start
 *(.option_setting_bps0)
                0x0100a100                        . = USE_OPTION_SETTING_NS?(__OPTION_SETTING_NS_Start + 0x44):__OPTION_SETTING_NS_Start
 *(.option_setting_bps1)
                0x0100a100                        . = USE_OPTION_SETTING_NS?(__OPTION_SETTING_NS_Start + 0x48):__OPTION_SETTING_NS_Start
 *(.option_setting_bps2)
                0x0100a100                        . = USE_OPTION_SETTING_NS?(__OPTION_SETTING_NS_Start + 0x4c):__OPTION_SETTING_NS_Start
 *(.option_setting_bps3)
                0x0100a100                        . = USE_OPTION_SETTING_NS?(__OPTION_SETTING_NS_Start + 0x60):__OPTION_SETTING_NS_Start
 *(.option_setting_pbps0)
                0x0100a100                        . = USE_OPTION_SETTING_NS?(__OPTION_SETTING_NS_Start + 0x64):__OPTION_SETTING_NS_Start
 *(.option_setting_pbps1)
                0x0100a100                        . = USE_OPTION_SETTING_NS?(__OPTION_SETTING_NS_Start + 0x68):__OPTION_SETTING_NS_Start
 *(.option_setting_pbps2)
                0x0100a100                        . = USE_OPTION_SETTING_NS?(__OPTION_SETTING_NS_Start + 0x6c):__OPTION_SETTING_NS_Start
 *(.option_setting_pbps3)
                0x0100a100                        __OPTION_SETTING_NS_End = .
                0x0100a200                        __tz_OPTION_SETTING_S_S = ORIGIN (OPTION_SETTING_S)

.option_setting_s
                0x0100a200       0xd0
                0x0100a200                        __OPTION_SETTING_S_Start = .
 *(.option_setting_ofs1_sec)
 .option_setting_ofs1_sec
                0x0100a200        0x4 ./ra/fsp/src/bsp/mcu/all/bsp_rom_registers.o
                0x0100a204                        . = PROJECT_SECURE_OR_FLAT?(__OPTION_SETTING_S_Start + 0x4):__OPTION_SETTING_S_Start
 *(.option_setting_ofs3_sec)
                0x0100a210                        . = PROJECT_SECURE_OR_FLAT?(__OPTION_SETTING_S_Start + 0x10):__OPTION_SETTING_S_Start
 *fill*         0x0100a204        0xc ff
 *(.option_setting_banksel_sec)
 .option_setting_banksel_sec
                0x0100a210        0x4 ./ra/fsp/src/bsp/mcu/all/bsp_rom_registers.o
                0x0100a240                        . = PROJECT_SECURE_OR_FLAT?(__OPTION_SETTING_S_Start + 0x40):__OPTION_SETTING_S_Start
 *fill*         0x0100a214       0x2c ff
 *(.option_setting_bps_sec0)
 .option_setting_bps_sec0
                0x0100a240        0x4 ./ra/fsp/src/bsp/mcu/all/bsp_rom_registers.o
                0x0100a244                        . = PROJECT_SECURE_OR_FLAT?(__OPTION_SETTING_S_Start + 0x44):__OPTION_SETTING_S_Start
 *(.option_setting_bps_sec1)
 .option_setting_bps_sec1
                0x0100a244        0x4 ./ra/fsp/src/bsp/mcu/all/bsp_rom_registers.o
                0x0100a248                        . = PROJECT_SECURE_OR_FLAT?(__OPTION_SETTING_S_Start + 0x48):__OPTION_SETTING_S_Start
 *(.option_setting_bps_sec2)
 .option_setting_bps_sec2
                0x0100a248        0x4 ./ra/fsp/src/bsp/mcu/all/bsp_rom_registers.o
                0x0100a24c                        . = PROJECT_SECURE_OR_FLAT?(__OPTION_SETTING_S_Start + 0x4c):__OPTION_SETTING_S_Start
 *(.option_setting_bps_sec3)
 .option_setting_bps_sec3
                0x0100a24c        0x4 ./ra/fsp/src/bsp/mcu/all/bsp_rom_registers.o
                0x0100a260                        . = PROJECT_SECURE_OR_FLAT?(__OPTION_SETTING_S_Start + 0x60):__OPTION_SETTING_S_Start
 *fill*         0x0100a250       0x10 ff
 *(.option_setting_pbps_sec0)
 .option_setting_pbps_sec0
                0x0100a260        0x4 ./ra/fsp/src/bsp/mcu/all/bsp_rom_registers.o
                0x0100a264                        . = PROJECT_SECURE_OR_FLAT?(__OPTION_SETTING_S_Start + 0x64):__OPTION_SETTING_S_Start
 *(.option_setting_pbps_sec1)
 .option_setting_pbps_sec1
                0x0100a264        0x4 ./ra/fsp/src/bsp/mcu/all/bsp_rom_registers.o
                0x0100a268                        . = PROJECT_SECURE_OR_FLAT?(__OPTION_SETTING_S_Start + 0x68):__OPTION_SETTING_S_Start
 *(.option_setting_pbps_sec2)
 .option_setting_pbps_sec2
                0x0100a268        0x4 ./ra/fsp/src/bsp/mcu/all/bsp_rom_registers.o
                0x0100a26c                        . = PROJECT_SECURE_OR_FLAT?(__OPTION_SETTING_S_Start + 0x6c):__OPTION_SETTING_S_Start
 *(.option_setting_pbps_sec3)
 .option_setting_pbps_sec3
                0x0100a26c        0x4 ./ra/fsp/src/bsp/mcu/all/bsp_rom_registers.o
                0x0100a280                        . = PROJECT_SECURE_OR_FLAT?(__OPTION_SETTING_S_Start + 0x80):__OPTION_SETTING_S_Start
 *fill*         0x0100a270       0x10 ff
 *(.option_setting_ofs1_sel)
 .option_setting_ofs1_sel
                0x0100a280        0x4 ./ra/fsp/src/bsp/mcu/all/bsp_rom_registers.o
                0x0100a284                        . = PROJECT_SECURE_OR_FLAT?(__OPTION_SETTING_S_Start + 0x84):__OPTION_SETTING_S_Start
 *(.option_setting_ofs3_sel)
                0x0100a290                        . = PROJECT_SECURE_OR_FLAT?(__OPTION_SETTING_S_Start + 0x90):__OPTION_SETTING_S_Start
 *fill*         0x0100a284        0xc ff
 *(.option_setting_banksel_sel)
                0x0100a2c0                        . = PROJECT_SECURE_OR_FLAT?(__OPTION_SETTING_S_Start + 0xc0):__OPTION_SETTING_S_Start
 *fill*         0x0100a290       0x30 ff
 *(.option_setting_bps_sel0)
 .option_setting_bps_sel0
                0x0100a2c0        0x4 ./ra/fsp/src/bsp/mcu/all/bsp_rom_registers.o
                0x0100a2c4                        . = PROJECT_SECURE_OR_FLAT?(__OPTION_SETTING_S_Start + 0xc4):__OPTION_SETTING_S_Start
 *(.option_setting_bps_sel1)
 .option_setting_bps_sel1
                0x0100a2c4        0x4 ./ra/fsp/src/bsp/mcu/all/bsp_rom_registers.o
                0x0100a2c8                        . = PROJECT_SECURE_OR_FLAT?(__OPTION_SETTING_S_Start + 0xc8):__OPTION_SETTING_S_Start
 *(.option_setting_bps_sel2)
 .option_setting_bps_sel2
                0x0100a2c8        0x4 ./ra/fsp/src/bsp/mcu/all/bsp_rom_registers.o
                0x0100a2cc                        . = PROJECT_SECURE_OR_FLAT?(__OPTION_SETTING_S_Start + 0xcc):__OPTION_SETTING_S_Start
 *(.option_setting_bps_sel3)
 .option_setting_bps_sel3
                0x0100a2cc        0x4 ./ra/fsp/src/bsp/mcu/all/bsp_rom_registers.o
                0x0100a2d0                        __OPTION_SETTING_S_End = .
                0x0100a2d0                        __tz_OPTION_SETTING_S_N = __OPTION_SETTING_S_End
OUTPUT(JP200.elf elf32-littlearm)
LOAD linker stubs

.rel.dyn        0x0100a2d0        0x0
 .rel.iplt      0x0100a2d0        0x0 c:/renesas/ra/e2studio_v2023-10_fsp_v5.0.0/toolchains/gcc_arm/12.2.mpacbti-rel1/bin/../lib/gcc/arm-none-eabi/12.2.1/thumb/v8-m.main+fp/hard/crtbegin.o

.ARM.attributes
                0x00000000       0x36
 .ARM.attributes
                0x00000000       0x26 c:/renesas/ra/e2studio_v2023-10_fsp_v5.0.0/toolchains/gcc_arm/12.2.mpacbti-rel1/bin/../lib/gcc/arm-none-eabi/12.2.1/thumb/v8-m.main+fp/hard/crti.o
 .ARM.attributes
                0x00000026       0x38 c:/renesas/ra/e2studio_v2023-10_fsp_v5.0.0/toolchains/gcc_arm/12.2.mpacbti-rel1/bin/../lib/gcc/arm-none-eabi/12.2.1/thumb/v8-m.main+fp/hard/crtbegin.o
 .ARM.attributes
                0x0000005e       0x3a ./src/adc_temp.o
 .ARM.attributes
                0x00000098       0x3a ./src/angle.o
 .ARM.attributes
                0x000000d2       0x3a ./src/control_table.o
 .ARM.attributes
                0x0000010c       0x3a ./src/crc8.o
 .ARM.attributes
                0x00000146       0x3a ./src/global_variables.o
 .ARM.attributes
                0x00000180       0x3a ./src/hal_entry.o
 .ARM.attributes
                0x000001ba       0x3a ./src/interpolation.o
 .ARM.attributes
                0x000001f4       0x3a ./src/monitor.o
 .ARM.attributes
                0x0000022e       0x3a ./src/packet.o
 .ARM.attributes
                0x00000268       0x3a ./src/pid.o
 .ARM.attributes
                0x000002a2       0x3a ./src/power_monitor.o
 .ARM.attributes
                0x000002dc       0x3a ./src/sintable.o
 .ARM.attributes
                0x00000316       0x3a ./src/usart.o
 .ARM.attributes
                0x00000350       0x3a ./ra_gen/common_data.o
 .ARM.attributes
                0x0000038a       0x3a ./ra_gen/hal_data.o
 .ARM.attributes
                0x000003c4       0x3a ./ra_gen/main.o
 .ARM.attributes
                0x000003fe       0x3a ./ra_gen/pin_data.o
 .ARM.attributes
                0x00000438       0x3a ./ra_gen/vector_data.o
 .ARM.attributes
                0x00000472       0x3a ./ra/fsp/src/r_sci_uart/r_sci_uart.o
 .ARM.attributes
                0x000004ac       0x3a ./ra/fsp/src/r_sci_spi/r_sci_spi.o
 .ARM.attributes
                0x000004e6       0x3a ./ra/fsp/src/r_sci_i2c/r_sci_i2c.o
 .ARM.attributes
                0x00000520       0x3a ./ra/fsp/src/r_rtc/r_rtc.o
 .ARM.attributes
                0x0000055a       0x3a ./ra/fsp/src/r_ioport/r_ioport.o
 .ARM.attributes
                0x00000594       0x3a ./ra/fsp/src/r_gpt/r_gpt.o
 .ARM.attributes
                0x000005ce       0x3a ./ra/fsp/src/r_flash_hp/r_flash_hp.o
 .ARM.attributes
                0x00000608       0x3a ./ra/fsp/src/r_dtc/r_dtc.o
 .ARM.attributes
                0x00000642       0x3a ./ra/fsp/src/r_crc/r_crc.o
 .ARM.attributes
                0x0000067c       0x3a ./ra/fsp/src/r_agt/r_agt.o
 .ARM.attributes
                0x000006b6       0x3a ./ra/fsp/src/r_adc/r_adc.o
 .ARM.attributes
                0x000006f0       0x3a ./ra/fsp/src/bsp/mcu/all/bsp_clocks.o
 .ARM.attributes
                0x0000072a       0x3a ./ra/fsp/src/bsp/mcu/all/bsp_common.o
 .ARM.attributes
                0x00000764       0x3a ./ra/fsp/src/bsp/mcu/all/bsp_delay.o
 .ARM.attributes
                0x0000079e       0x3a ./ra/fsp/src/bsp/mcu/all/bsp_group_irq.o
 .ARM.attributes
                0x000007d8       0x3a ./ra/fsp/src/bsp/mcu/all/bsp_io.o
 .ARM.attributes
                0x00000812       0x3a ./ra/fsp/src/bsp/mcu/all/bsp_irq.o
 .ARM.attributes
                0x0000084c       0x3a ./ra/fsp/src/bsp/mcu/all/bsp_register_protection.o
 .ARM.attributes
                0x00000886       0x3a ./ra/fsp/src/bsp/mcu/all/bsp_rom_registers.o
 .ARM.attributes
                0x000008c0       0x3a ./ra/fsp/src/bsp/cmsis/Device/RENESAS/Source/startup.o
 .ARM.attributes
                0x000008fa       0x3a ./ra/fsp/src/bsp/cmsis/Device/RENESAS/Source/system.o
 .ARM.attributes
                0x00000934       0x26 c:/renesas/ra/e2studio_v2023-10_fsp_v5.0.0/toolchains/gcc_arm/12.2.mpacbti-rel1/bin/../lib/gcc/arm-none-eabi/12.2.1/thumb/v8-m.main+fp/hard\libgcc.a(_arm_addsubdf3.o)
 .ARM.attributes
                0x0000095a       0x26 c:/renesas/ra/e2studio_v2023-10_fsp_v5.0.0/toolchains/gcc_arm/12.2.mpacbti-rel1/bin/../lib/gcc/arm-none-eabi/12.2.1/thumb/v8-m.main+fp/hard\libgcc.a(_arm_muldivdf3.o)
 .ARM.attributes
                0x00000980       0x26 c:/renesas/ra/e2studio_v2023-10_fsp_v5.0.0/toolchains/gcc_arm/12.2.mpacbti-rel1/bin/../lib/gcc/arm-none-eabi/12.2.1/thumb/v8-m.main+fp/hard\libgcc.a(_arm_cmpdf2.o)
 .ARM.attributes
                0x000009a6       0x26 c:/renesas/ra/e2studio_v2023-10_fsp_v5.0.0/toolchains/gcc_arm/12.2.mpacbti-rel1/bin/../lib/gcc/arm-none-eabi/12.2.1/thumb/v8-m.main+fp/hard\libgcc.a(_arm_fixdfsi.o)
 .ARM.attributes
                0x000009cc       0x26 c:/renesas/ra/e2studio_v2023-10_fsp_v5.0.0/toolchains/gcc_arm/12.2.mpacbti-rel1/bin/../lib/gcc/arm-none-eabi/12.2.1/thumb/v8-m.main+fp/hard\libgcc.a(_arm_fixunsdfsi.o)
 .ARM.attributes
                0x000009f2       0x26 c:/renesas/ra/e2studio_v2023-10_fsp_v5.0.0/toolchains/gcc_arm/12.2.mpacbti-rel1/bin/../lib/gcc/arm-none-eabi/12.2.1/thumb/v8-m.main+fp/hard\libgcc.a(_aeabi_ldivmod.o)
 .ARM.attributes
                0x00000a18       0x38 c:/renesas/ra/e2studio_v2023-10_fsp_v5.0.0/toolchains/gcc_arm/12.2.mpacbti-rel1/bin/../lib/gcc/arm-none-eabi/12.2.1/thumb/v8-m.main+fp/hard\libgcc.a(_udivmoddi4.o)
 .ARM.attributes
                0x00000a50       0x26 c:/renesas/ra/e2studio_v2023-10_fsp_v5.0.0/toolchains/gcc_arm/12.2.mpacbti-rel1/bin/../lib/gcc/arm-none-eabi/12.2.1/thumb/v8-m.main+fp/hard\libgcc.a(_dvmd_tls.o)
 .ARM.attributes
                0x00000a76       0x38 c:/renesas/ra/e2studio_v2023-10_fsp_v5.0.0/toolchains/gcc_arm/12.2.mpacbti-rel1/bin/../lib/gcc/arm-none-eabi/12.2.1/thumb/v8-m.main+fp/hard\libg_nano.a(libc_a-itoa.o)
 .ARM.attributes
                0x00000aae       0x38 c:/renesas/ra/e2studio_v2023-10_fsp_v5.0.0/toolchains/gcc_arm/12.2.mpacbti-rel1/bin/../lib/gcc/arm-none-eabi/12.2.1/thumb/v8-m.main+fp/hard\libg_nano.a(libc_a-strtol.o)
 .ARM.attributes
                0x00000ae6       0x38 c:/renesas/ra/e2studio_v2023-10_fsp_v5.0.0/toolchains/gcc_arm/12.2.mpacbti-rel1/bin/../lib/gcc/arm-none-eabi/12.2.1/thumb/v8-m.main+fp/hard\libg_nano.a(libc_a-utoa.o)
 .ARM.attributes
                0x00000b1e       0x38 c:/renesas/ra/e2studio_v2023-10_fsp_v5.0.0/toolchains/gcc_arm/12.2.mpacbti-rel1/bin/../lib/gcc/arm-none-eabi/12.2.1/thumb/v8-m.main+fp/hard\libg_nano.a(libc_a-ctype_.o)
 .ARM.attributes
                0x00000b56       0x38 c:/renesas/ra/e2studio_v2023-10_fsp_v5.0.0/toolchains/gcc_arm/12.2.mpacbti-rel1/bin/../lib/gcc/arm-none-eabi/12.2.1/thumb/v8-m.main+fp/hard\libg_nano.a(libc_a-findfp.o)
 .ARM.attributes
                0x00000b8e       0x38 c:/renesas/ra/e2studio_v2023-10_fsp_v5.0.0/toolchains/gcc_arm/12.2.mpacbti-rel1/bin/../lib/gcc/arm-none-eabi/12.2.1/thumb/v8-m.main+fp/hard\libg_nano.a(libc_a-memset.o)
 .ARM.attributes
                0x00000bc6       0x38 c:/renesas/ra/e2studio_v2023-10_fsp_v5.0.0/toolchains/gcc_arm/12.2.mpacbti-rel1/bin/../lib/gcc/arm-none-eabi/12.2.1/thumb/v8-m.main+fp/hard\libg_nano.a(libc_a-impure.o)
 .ARM.attributes
                0x00000bfe       0x38 c:/renesas/ra/e2studio_v2023-10_fsp_v5.0.0/toolchains/gcc_arm/12.2.mpacbti-rel1/bin/../lib/gcc/arm-none-eabi/12.2.1/thumb/v8-m.main+fp/hard\libg_nano.a(libc_a-errno.o)
 .ARM.attributes
                0x00000c36       0x38 c:/renesas/ra/e2studio_v2023-10_fsp_v5.0.0/toolchains/gcc_arm/12.2.mpacbti-rel1/bin/../lib/gcc/arm-none-eabi/12.2.1/thumb/v8-m.main+fp/hard\libg_nano.a(libc_a-strcpy.o)
 .ARM.attributes
                0x00000c6e       0x38 c:/renesas/ra/e2studio_v2023-10_fsp_v5.0.0/toolchains/gcc_arm/12.2.mpacbti-rel1/bin/../lib/gcc/arm-none-eabi/12.2.1/thumb/v8-m.main+fp/hard\libg_nano.a(libc_a-aeabi_memcpy.o)
 .ARM.attributes
                0x00000ca6       0x38 c:/renesas/ra/e2studio_v2023-10_fsp_v5.0.0/toolchains/gcc_arm/12.2.mpacbti-rel1/bin/../lib/gcc/arm-none-eabi/12.2.1/thumb/v8-m.main+fp/hard\libg_nano.a(libc_a-aeabi_memclr.o)
 .ARM.attributes
                0x00000cde       0x38 c:/renesas/ra/e2studio_v2023-10_fsp_v5.0.0/toolchains/gcc_arm/12.2.mpacbti-rel1/bin/../lib/gcc/arm-none-eabi/12.2.1/thumb/v8-m.main+fp/hard\libg_nano.a(libc_a-memcpy-stub.o)
 .ARM.attributes
                0x00000d16       0x24 c:/renesas/ra/e2studio_v2023-10_fsp_v5.0.0/toolchains/gcc_arm/12.2.mpacbti-rel1/bin/../lib/gcc/arm-none-eabi/12.2.1/thumb/v8-m.main+fp/hard\libg_nano.a(libc_a-strlen.o)
 .ARM.attributes
                0x00000d3a       0x24 c:/renesas/ra/e2studio_v2023-10_fsp_v5.0.0/toolchains/gcc_arm/12.2.mpacbti-rel1/bin/../lib/gcc/arm-none-eabi/12.2.1/thumb/v8-m.main+fp/hard\libg_nano.a(libc_a-aeabi_memset-soft.o)
 .ARM.attributes
                0x00000d5e       0x38 c:/renesas/ra/e2studio_v2023-10_fsp_v5.0.0/toolchains/gcc_arm/12.2.mpacbti-rel1/bin/../lib/gcc/arm-none-eabi/12.2.1/thumb/v8-m.main+fp/hard/crtend.o
 .ARM.attributes
                0x00000d96       0x26 c:/renesas/ra/e2studio_v2023-10_fsp_v5.0.0/toolchains/gcc_arm/12.2.mpacbti-rel1/bin/../lib/gcc/arm-none-eabi/12.2.1/thumb/v8-m.main+fp/hard/crtn.o

.comment        0x00000000       0x55
 .comment       0x00000000       0x55 ./src/adc_temp.o
                                 0x56 (size before relaxing)
 .comment       0x00000055       0x56 ./src/angle.o
 .comment       0x00000055       0x56 ./src/control_table.o
 .comment       0x00000055       0x56 ./src/crc8.o
 .comment       0x00000055       0x56 ./src/global_variables.o
 .comment       0x00000055       0x56 ./src/hal_entry.o
 .comment       0x00000055       0x56 ./src/interpolation.o
 .comment       0x00000055       0x56 ./src/monitor.o
 .comment       0x00000055       0x56 ./src/packet.o
 .comment       0x00000055       0x56 ./src/pid.o
 .comment       0x00000055       0x56 ./src/power_monitor.o
 .comment       0x00000055       0x56 ./src/sintable.o
 .comment       0x00000055       0x56 ./src/usart.o
 .comment       0x00000055       0x56 ./ra_gen/common_data.o
 .comment       0x00000055       0x56 ./ra_gen/hal_data.o
 .comment       0x00000055       0x56 ./ra_gen/main.o
 .comment       0x00000055       0x56 ./ra_gen/pin_data.o
 .comment       0x00000055       0x56 ./ra_gen/vector_data.o
 .comment       0x00000055       0x56 ./ra/fsp/src/r_sci_uart/r_sci_uart.o
 .comment       0x00000055       0x56 ./ra/fsp/src/r_sci_spi/r_sci_spi.o
 .comment       0x00000055       0x56 ./ra/fsp/src/r_sci_i2c/r_sci_i2c.o
 .comment       0x00000055       0x56 ./ra/fsp/src/r_rtc/r_rtc.o
 .comment       0x00000055       0x56 ./ra/fsp/src/r_ioport/r_ioport.o
 .comment       0x00000055       0x56 ./ra/fsp/src/r_gpt/r_gpt.o
 .comment       0x00000055       0x56 ./ra/fsp/src/r_flash_hp/r_flash_hp.o
 .comment       0x00000055       0x56 ./ra/fsp/src/r_dtc/r_dtc.o
 .comment       0x00000055       0x56 ./ra/fsp/src/r_crc/r_crc.o
 .comment       0x00000055       0x56 ./ra/fsp/src/r_agt/r_agt.o
 .comment       0x00000055       0x56 ./ra/fsp/src/r_adc/r_adc.o
 .comment       0x00000055       0x56 ./ra/fsp/src/bsp/mcu/all/bsp_clocks.o
 .comment       0x00000055       0x56 ./ra/fsp/src/bsp/mcu/all/bsp_common.o
 .comment       0x00000055       0x56 ./ra/fsp/src/bsp/mcu/all/bsp_delay.o
 .comment       0x00000055       0x56 ./ra/fsp/src/bsp/mcu/all/bsp_group_irq.o
 .comment       0x00000055       0x56 ./ra/fsp/src/bsp/mcu/all/bsp_io.o
 .comment       0x00000055       0x56 ./ra/fsp/src/bsp/mcu/all/bsp_irq.o
 .comment       0x00000055       0x56 ./ra/fsp/src/bsp/mcu/all/bsp_register_protection.o
 .comment       0x00000055       0x56 ./ra/fsp/src/bsp/mcu/all/bsp_rom_registers.o
 .comment       0x00000055       0x56 ./ra/fsp/src/bsp/cmsis/Device/RENESAS/Source/startup.o
 .comment       0x00000055       0x56 ./ra/fsp/src/bsp/cmsis/Device/RENESAS/Source/system.o

.debug_info     0x00000000    0x86acc
 .debug_info    0x00000000     0x3252 ./src/adc_temp.o
 .debug_info    0x00003252     0x6be9 ./src/angle.o
 .debug_info    0x00009e3b     0x19f6 ./src/control_table.o
 .debug_info    0x0000b831      0x16d ./src/crc8.o
 .debug_info    0x0000b99e      0x242 ./src/global_variables.o
 .debug_info    0x0000bbe0     0x8c09 ./src/hal_entry.o
 .debug_info    0x000147e9       0xee ./src/interpolation.o
 .debug_info    0x000148d7      0x678 ./src/monitor.o
 .debug_info    0x00014f4f     0x443b ./src/packet.o
 .debug_info    0x0001938a      0x440 ./src/pid.o
 .debug_info    0x000197ca     0x286f ./src/power_monitor.o
 .debug_info    0x0001c039      0x13b ./src/sintable.o
 .debug_info    0x0001c174     0x3e50 ./src/usart.o
 .debug_info    0x0001ffc4     0x11f2 ./ra_gen/common_data.o
 .debug_info    0x000211b6     0xc1e8 ./ra_gen/hal_data.o
 .debug_info    0x0002d39e       0xb1 ./ra_gen/main.o
 .debug_info    0x0002d44f      0xa18 ./ra_gen/pin_data.o
 .debug_info    0x0002de67      0x6b4 ./ra_gen/vector_data.o
 .debug_info    0x0002e51b     0xa00d ./ra/fsp/src/r_sci_uart/r_sci_uart.o
 .debug_info    0x00038528     0x91fe ./ra/fsp/src/r_sci_spi/r_sci_spi.o
 .debug_info    0x00041726     0x4f39 ./ra/fsp/src/r_sci_i2c/r_sci_i2c.o
 .debug_info    0x0004665f     0x4375 ./ra/fsp/src/r_rtc/r_rtc.o
 .debug_info    0x0004a9d4     0x64cf ./ra/fsp/src/r_ioport/r_ioport.o
 .debug_info    0x00050ea3     0xa6e9 ./ra/fsp/src/r_gpt/r_gpt.o
 .debug_info    0x0005b58c     0x7b52 ./ra/fsp/src/r_flash_hp/r_flash_hp.o
 .debug_info    0x000630de     0x29ae ./ra/fsp/src/r_dtc/r_dtc.o
 .debug_info    0x00065a8c     0x1c2f ./ra/fsp/src/r_crc/r_crc.o
 .debug_info    0x000676bb     0x74e4 ./ra/fsp/src/r_agt/r_agt.o
 .debug_info    0x0006eb9f     0xaf05 ./ra/fsp/src/r_adc/r_adc.o
 .debug_info    0x00079aa4     0x52e8 ./ra/fsp/src/bsp/mcu/all/bsp_clocks.o
 .debug_info    0x0007ed8c      0x90e ./ra/fsp/src/bsp/mcu/all/bsp_common.o
 .debug_info    0x0007f69a      0x1d2 ./ra/fsp/src/bsp/mcu/all/bsp_delay.o
 .debug_info    0x0007f86c     0x127d ./ra/fsp/src/bsp/mcu/all/bsp_group_irq.o
 .debug_info    0x00080ae9       0xb2 ./ra/fsp/src/bsp/mcu/all/bsp_io.o
 .debug_info    0x00080b9b     0x1b13 ./ra/fsp/src/bsp/mcu/all/bsp_irq.o
 .debug_info    0x000826ae     0x37c1 ./ra/fsp/src/bsp/mcu/all/bsp_register_protection.o
 .debug_info    0x00085e6f      0x1b8 ./ra/fsp/src/bsp/mcu/all/bsp_rom_registers.o
 .debug_info    0x00086027      0x168 ./ra/fsp/src/bsp/cmsis/Device/RENESAS/Source/startup.o
 .debug_info    0x0008618f      0x93d ./ra/fsp/src/bsp/cmsis/Device/RENESAS/Source/system.o

.debug_abbrev   0x00000000     0x7b03
 .debug_abbrev  0x00000000      0x263 ./src/adc_temp.o
 .debug_abbrev  0x00000263      0x4d1 ./src/angle.o
 .debug_abbrev  0x00000734      0x418 ./src/control_table.o
 .debug_abbrev  0x00000b4c       0xcf ./src/crc8.o
 .debug_abbrev  0x00000c1b       0xbd ./src/global_variables.o
 .debug_abbrev  0x00000cd8      0x5fe ./src/hal_entry.o
 .debug_abbrev  0x000012d6       0x90 ./src/interpolation.o
 .debug_abbrev  0x00001366      0x1e8 ./src/monitor.o
 .debug_abbrev  0x0000154e      0x699 ./src/packet.o
 .debug_abbrev  0x00001be7      0x118 ./src/pid.o
 .debug_abbrev  0x00001cff      0x338 ./src/power_monitor.o
 .debug_abbrev  0x00002037       0xae ./src/sintable.o
 .debug_abbrev  0x000020e5      0x66c ./src/usart.o
 .debug_abbrev  0x00002751      0x133 ./ra_gen/common_data.o
 .debug_abbrev  0x00002884      0x323 ./ra_gen/hal_data.o
 .debug_abbrev  0x00002ba7       0x61 ./ra_gen/main.o
 .debug_abbrev  0x00002c08       0xff ./ra_gen/pin_data.o
 .debug_abbrev  0x00002d07       0xbd ./ra_gen/vector_data.o
 .debug_abbrev  0x00002dc4      0x615 ./ra/fsp/src/r_sci_uart/r_sci_uart.o
 .debug_abbrev  0x000033d9      0x631 ./ra/fsp/src/r_sci_spi/r_sci_spi.o
 .debug_abbrev  0x00003a0a      0x57e ./ra/fsp/src/r_sci_i2c/r_sci_i2c.o
 .debug_abbrev  0x00003f88      0x57d ./ra/fsp/src/r_rtc/r_rtc.o
 .debug_abbrev  0x00004505      0x494 ./ra/fsp/src/r_ioport/r_ioport.o
 .debug_abbrev  0x00004999      0x627 ./ra/fsp/src/r_gpt/r_gpt.o
 .debug_abbrev  0x00004fc0      0x5a6 ./ra/fsp/src/r_flash_hp/r_flash_hp.o
 .debug_abbrev  0x00005566      0x4db ./ra/fsp/src/r_dtc/r_dtc.o
 .debug_abbrev  0x00005a41      0x329 ./ra/fsp/src/r_crc/r_crc.o
 .debug_abbrev  0x00005d6a      0x5a7 ./ra/fsp/src/r_agt/r_agt.o
 .debug_abbrev  0x00006311      0x597 ./ra/fsp/src/r_adc/r_adc.o
 .debug_abbrev  0x000068a8      0x40b ./ra/fsp/src/bsp/mcu/all/bsp_clocks.o
 .debug_abbrev  0x00006cb3      0x188 ./ra/fsp/src/bsp/mcu/all/bsp_common.o
 .debug_abbrev  0x00006e3b      0x10b ./ra/fsp/src/bsp/mcu/all/bsp_delay.o
 .debug_abbrev  0x00006f46      0x256 ./ra/fsp/src/bsp/mcu/all/bsp_group_irq.o
 .debug_abbrev  0x0000719c       0x5e ./ra/fsp/src/bsp/mcu/all/bsp_io.o
 .debug_abbrev  0x000071fa      0x271 ./ra/fsp/src/bsp/mcu/all/bsp_irq.o
 .debug_abbrev  0x0000746b      0x27d ./ra/fsp/src/bsp/mcu/all/bsp_register_protection.o
 .debug_abbrev  0x000076e8       0x4e ./ra/fsp/src/bsp/mcu/all/bsp_rom_registers.o
 .debug_abbrev  0x00007736       0xf5 ./ra/fsp/src/bsp/cmsis/Device/RENESAS/Source/startup.o
 .debug_abbrev  0x0000782b      0x2d8 ./ra/fsp/src/bsp/cmsis/Device/RENESAS/Source/system.o

.debug_aranges  0x00000000      0xbd8
 .debug_aranges
                0x00000000       0x40 ./src/adc_temp.o
 .debug_aranges
                0x00000040       0x40 ./src/angle.o
 .debug_aranges
                0x00000080       0x48 ./src/control_table.o
 .debug_aranges
                0x000000c8       0x28 ./src/crc8.o
 .debug_aranges
                0x000000f0       0x18 ./src/global_variables.o
 .debug_aranges
                0x00000108       0x60 ./src/hal_entry.o
 .debug_aranges
                0x00000168       0x20 ./src/interpolation.o
 .debug_aranges
                0x00000188       0x20 ./src/monitor.o
 .debug_aranges
                0x000001a8       0xf0 ./src/packet.o
 .debug_aranges
                0x00000298       0x38 ./src/pid.o
 .debug_aranges
                0x000002d0       0x50 ./src/power_monitor.o
 .debug_aranges
                0x00000320       0x28 ./src/sintable.o
 .debug_aranges
                0x00000348       0x80 ./src/usart.o
 .debug_aranges
                0x000003c8       0x20 ./ra_gen/common_data.o
 .debug_aranges
                0x000003e8       0x20 ./ra_gen/hal_data.o
 .debug_aranges
                0x00000408       0x20 ./ra_gen/main.o
 .debug_aranges
                0x00000428       0x18 ./ra_gen/pin_data.o
 .debug_aranges
                0x00000440       0x18 ./ra_gen/vector_data.o
 .debug_aranges
                0x00000458       0x88 ./ra/fsp/src/r_sci_uart/r_sci_uart.o
 .debug_aranges
                0x000004e0       0x70 ./ra/fsp/src/r_sci_spi/r_sci_spi.o
 .debug_aranges
                0x00000550       0x70 ./ra/fsp/src/r_sci_i2c/r_sci_i2c.o
 .debug_aranges
                0x000005c0       0x80 ./ra/fsp/src/r_rtc/r_rtc.o
 .debug_aranges
                0x00000640       0x90 ./ra/fsp/src/r_ioport/r_ioport.o
 .debug_aranges
                0x000006d0       0xc8 ./ra/fsp/src/r_gpt/r_gpt.o
 .debug_aranges
                0x00000798       0xb0 ./ra/fsp/src/r_flash_hp/r_flash_hp.o
 .debug_aranges
                0x00000848       0x68 ./ra/fsp/src/r_dtc/r_dtc.o
 .debug_aranges
                0x000008b0       0x48 ./ra/fsp/src/r_crc/r_crc.o
 .debug_aranges
                0x000008f8       0x80 ./ra/fsp/src/r_agt/r_agt.o
 .debug_aranges
                0x00000978       0xa8 ./ra/fsp/src/r_adc/r_adc.o
 .debug_aranges
                0x00000a20       0x70 ./ra/fsp/src/bsp/mcu/all/bsp_clocks.o
 .debug_aranges
                0x00000a90       0x30 ./ra/fsp/src/bsp/mcu/all/bsp_common.o
 .debug_aranges
                0x00000ac0       0x28 ./ra/fsp/src/bsp/mcu/all/bsp_delay.o
 .debug_aranges
                0x00000ae8       0x28 ./ra/fsp/src/bsp/mcu/all/bsp_group_irq.o
 .debug_aranges
                0x00000b10       0x18 ./ra/fsp/src/bsp/mcu/all/bsp_io.o
 .debug_aranges
                0x00000b28       0x20 ./ra/fsp/src/bsp/mcu/all/bsp_irq.o
 .debug_aranges
                0x00000b48       0x28 ./ra/fsp/src/bsp/mcu/all/bsp_register_protection.o
 .debug_aranges
                0x00000b70       0x18 ./ra/fsp/src/bsp/mcu/all/bsp_rom_registers.o
 .debug_aranges
                0x00000b88       0x28 ./ra/fsp/src/bsp/cmsis/Device/RENESAS/Source/startup.o
 .debug_aranges
                0x00000bb0       0x28 ./ra/fsp/src/bsp/cmsis/Device/RENESAS/Source/system.o

.debug_rnglists
                0x00000000     0x295e
 .debug_rnglists
                0x00000000       0x2d ./src/adc_temp.o
 .debug_rnglists
                0x0000002d       0xce ./src/angle.o
 .debug_rnglists
                0x000000fb       0xbc ./src/control_table.o
 .debug_rnglists
                0x000001b7       0x19 ./src/crc8.o
 .debug_rnglists
                0x000001d0      0x133 ./src/hal_entry.o
 .debug_rnglists
                0x00000303       0x14 ./src/interpolation.o
 .debug_rnglists
                0x00000317       0x27 ./src/monitor.o
 .debug_rnglists
                0x0000033e      0x714 ./src/packet.o
 .debug_rnglists
                0x00000a52       0x26 ./src/pid.o
 .debug_rnglists
                0x00000a78       0x3b ./src/power_monitor.o
 .debug_rnglists
                0x00000ab3       0x1b ./src/sintable.o
 .debug_rnglists
                0x00000ace      0x1bb ./src/usart.o
 .debug_rnglists
                0x00000c89       0x13 ./ra_gen/common_data.o
 .debug_rnglists
                0x00000c9c       0x13 ./ra_gen/hal_data.o
 .debug_rnglists
                0x00000caf       0x13 ./ra_gen/main.o
 .debug_rnglists
                0x00000cc2      0x369 ./ra/fsp/src/r_sci_uart/r_sci_uart.o
 .debug_rnglists
                0x0000102b      0x3f5 ./ra/fsp/src/r_sci_spi/r_sci_spi.o
 .debug_rnglists
                0x00001420      0x28e ./ra/fsp/src/r_sci_i2c/r_sci_i2c.o
 .debug_rnglists
                0x000016ae      0x2a4 ./ra/fsp/src/r_rtc/r_rtc.o
 .debug_rnglists
                0x00001952       0xda ./ra/fsp/src/r_ioport/r_ioport.o
 .debug_rnglists
                0x00001a2c      0x302 ./ra/fsp/src/r_gpt/r_gpt.o
 .debug_rnglists
                0x00001d2e      0x3d3 ./ra/fsp/src/r_flash_hp/r_flash_hp.o
 .debug_rnglists
                0x00002101       0xf1 ./ra/fsp/src/r_dtc/r_dtc.o
 .debug_rnglists
                0x000021f2       0xee ./ra/fsp/src/r_crc/r_crc.o
 .debug_rnglists
                0x000022e0      0x1ce ./ra/fsp/src/r_agt/r_agt.o
 .debug_rnglists
                0x000024ae      0x2ca ./ra/fsp/src/r_adc/r_adc.o
 .debug_rnglists
                0x00002778       0xba ./ra/fsp/src/bsp/mcu/all/bsp_clocks.o
 .debug_rnglists
                0x00002832       0x1f ./ra/fsp/src/bsp/mcu/all/bsp_common.o
 .debug_rnglists
                0x00002851       0x19 ./ra/fsp/src/bsp/mcu/all/bsp_delay.o
 .debug_rnglists
                0x0000286a       0x37 ./ra/fsp/src/bsp/mcu/all/bsp_group_irq.o
 .debug_rnglists
                0x000028a1       0x41 ./ra/fsp/src/bsp/mcu/all/bsp_irq.o
 .debug_rnglists
                0x000028e2       0x31 ./ra/fsp/src/bsp/mcu/all/bsp_register_protection.o
 .debug_rnglists
                0x00002913       0x19 ./ra/fsp/src/bsp/cmsis/Device/RENESAS/Source/startup.o
 .debug_rnglists
                0x0000292c       0x32 ./ra/fsp/src/bsp/cmsis/Device/RENESAS/Source/system.o

.debug_line     0x00000000    0x18f7f
 .debug_line    0x00000000      0x3a2 ./src/adc_temp.o
 .debug_line    0x000003a2      0xa49 ./src/angle.o
 .debug_line    0x00000deb      0x9dd ./src/control_table.o
 .debug_line    0x000017c8      0x246 ./src/crc8.o
 .debug_line    0x00001a0e      0x152 ./src/global_variables.o
 .debug_line    0x00001b60     0x1c8f ./src/hal_entry.o
 .debug_line    0x000037ef      0x1ea ./src/interpolation.o
 .debug_line    0x000039d9      0x2ec ./src/monitor.o
 .debug_line    0x00003cc5     0x2897 ./src/packet.o
 .debug_line    0x0000655c      0x2ba ./src/pid.o
 .debug_line    0x00006816      0x581 ./src/power_monitor.o
 .debug_line    0x00006d97      0x2b6 ./src/sintable.o
 .debug_line    0x0000704d     0x1650 ./src/usart.o
 .debug_line    0x0000869d      0x2a5 ./ra_gen/common_data.o
 .debug_line    0x00008942      0x4aa ./ra_gen/hal_data.o
 .debug_line    0x00008dec       0x5e ./ra_gen/main.o
 .debug_line    0x00008e4a      0x21c ./ra_gen/pin_data.o
 .debug_line    0x00009066      0x12c ./ra_gen/vector_data.o
 .debug_line    0x00009192     0x1f6c ./ra/fsp/src/r_sci_uart/r_sci_uart.o
 .debug_line    0x0000b0fe     0x18df ./ra/fsp/src/r_sci_spi/r_sci_spi.o
 .debug_line    0x0000c9dd     0x10c9 ./ra/fsp/src/r_sci_i2c/r_sci_i2c.o
 .debug_line    0x0000daa6     0x1732 ./ra/fsp/src/r_rtc/r_rtc.o
 .debug_line    0x0000f1d8      0xbe0 ./ra/fsp/src/r_ioport/r_ioport.o
 .debug_line    0x0000fdb8     0x1740 ./ra/fsp/src/r_gpt/r_gpt.o
 .debug_line    0x000114f8     0x1f35 ./ra/fsp/src/r_flash_hp/r_flash_hp.o
 .debug_line    0x0001342d      0x932 ./ra/fsp/src/r_dtc/r_dtc.o
 .debug_line    0x00013d5f      0x676 ./ra/fsp/src/r_crc/r_crc.o
 .debug_line    0x000143d5     0x108d ./ra/fsp/src/r_agt/r_agt.o
 .debug_line    0x00015462     0x1675 ./ra/fsp/src/r_adc/r_adc.o
 .debug_line    0x00016ad7      0x8e4 ./ra/fsp/src/bsp/mcu/all/bsp_clocks.o
 .debug_line    0x000173bb      0x2cd ./ra/fsp/src/bsp/mcu/all/bsp_common.o
 .debug_line    0x00017688      0x2ac ./ra/fsp/src/bsp/mcu/all/bsp_delay.o
 .debug_line    0x00017934      0x310 ./ra/fsp/src/bsp/mcu/all/bsp_group_irq.o
 .debug_line    0x00017c44      0x18c ./ra/fsp/src/bsp/mcu/all/bsp_io.o
 .debug_line    0x00017dd0      0x4fd ./ra/fsp/src/bsp/mcu/all/bsp_irq.o
 .debug_line    0x000182cd      0x3b9 ./ra/fsp/src/bsp/mcu/all/bsp_register_protection.o
 .debug_line    0x00018686      0x147 ./ra/fsp/src/bsp/mcu/all/bsp_rom_registers.o
 .debug_line    0x000187cd      0x210 ./ra/fsp/src/bsp/cmsis/Device/RENESAS/Source/startup.o
 .debug_line    0x000189dd      0x5a2 ./ra/fsp/src/bsp/cmsis/Device/RENESAS/Source/system.o

.debug_str      0x00000000    0x140b3
 .debug_str     0x00000000     0x312a ./src/adc_temp.o
                               0x3229 (size before relaxing)
 .debug_str     0x0000312a     0x4306 ./src/angle.o
                               0x6031 (size before relaxing)
 .debug_str     0x00007430      0xa0a ./src/control_table.o
                               0x2658 (size before relaxing)
 .debug_str     0x00007e3a       0x2a ./src/crc8.o
                                0x1d3 (size before relaxing)
 .debug_str     0x00007e64       0xf4 ./src/global_variables.o
                                0x2aa (size before relaxing)
 .debug_str     0x00007f58      0xf14 ./src/hal_entry.o
                               0x71d1 (size before relaxing)
 .debug_str     0x00008e6c       0x17 ./src/interpolation.o
                                0x1b1 (size before relaxing)
 .debug_str     0x00008e83       0x6f ./src/monitor.o
                                0x674 (size before relaxing)
 .debug_str     0x00008ef2      0x259 ./src/packet.o
                                0xb6d (size before relaxing)
 .debug_str     0x0000914b       0x70 ./src/pid.o
                                0x29a (size before relaxing)
 .debug_str     0x000091bb      0x3c4 ./src/power_monitor.o
                               0x2a9e (size before relaxing)
 .debug_str     0x0000957f       0x2f ./src/sintable.o
                                0x1eb (size before relaxing)
 .debug_str     0x000095ae      0x4f5 ./src/usart.o
                               0x40d0 (size before relaxing)
 .debug_str     0x00009aa3       0x39 ./ra_gen/common_data.o
                               0x325a (size before relaxing)
 .debug_str     0x00009adc     0x42e8 ./ra_gen/hal_data.o
                               0xc325 (size before relaxing)
 .debug_str     0x0000ddc4       0x11 ./ra_gen/main.o
                                0x1b5 (size before relaxing)
 .debug_str     0x0000ddd5       0x28 ./ra_gen/pin_data.o
                               0x1d40 (size before relaxing)
 .debug_str     0x0000ddfd      0x126 ./ra_gen/vector_data.o
                               0x16eb (size before relaxing)
 .debug_str     0x0000df23     0x2330 ./ra/fsp/src/r_sci_uart/r_sci_uart.o
                               0x694e (size before relaxing)
 .debug_str     0x00010253      0x156 ./ra/fsp/src/r_sci_spi/r_sci_spi.o
                               0x5075 (size before relaxing)
 .debug_str     0x000103a9      0x207 ./ra/fsp/src/r_sci_i2c/r_sci_i2c.o
                               0x3745 (size before relaxing)
 .debug_str     0x000105b0      0x5a1 ./ra/fsp/src/r_rtc/r_rtc.o
                               0x30a6 (size before relaxing)
 .debug_str     0x00010b51      0x87d ./ra/fsp/src/r_ioport/r_ioport.o
                               0x572c (size before relaxing)
 .debug_str     0x000113ce      0xa87 ./ra/fsp/src/r_gpt/r_gpt.o
                               0x6acf (size before relaxing)
 .debug_str     0x00011e55      0x6a1 ./ra/fsp/src/r_flash_hp/r_flash_hp.o
                               0x46f0 (size before relaxing)
 .debug_str     0x000124f6      0x200 ./ra/fsp/src/r_dtc/r_dtc.o
                               0x2c8e (size before relaxing)
 .debug_str     0x000126f6      0x197 ./ra/fsp/src/r_crc/r_crc.o
                               0x23fa (size before relaxing)
 .debug_str     0x0001288d      0x1e3 ./ra/fsp/src/r_agt/r_agt.o
                               0x4b26 (size before relaxing)
 .debug_str     0x00012a70      0x5f8 ./ra/fsp/src/r_adc/r_adc.o
                               0x7d9d (size before relaxing)
 .debug_str     0x00013068      0x5c3 ./ra/fsp/src/bsp/mcu/all/bsp_clocks.o
                               0x253a (size before relaxing)
 .debug_str     0x0001362b      0x10b ./ra/fsp/src/bsp/mcu/all/bsp_common.o
                               0x1b65 (size before relaxing)
 .debug_str     0x00013736       0x9f ./ra/fsp/src/bsp/mcu/all/bsp_delay.o
                                0x2de (size before relaxing)
 .debug_str     0x000137d5      0x1e4 ./ra/fsp/src/bsp/mcu/all/bsp_group_irq.o
                               0x2076 (size before relaxing)
 .debug_str     0x000139b9       0x23 ./ra/fsp/src/bsp/mcu/all/bsp_io.o
                                0x1de (size before relaxing)
 .debug_str     0x000139dc      0x3af ./ra/fsp/src/bsp/mcu/all/bsp_irq.o
                               0x1f3d (size before relaxing)
 .debug_str     0x00013d8b       0x76 ./ra/fsp/src/bsp/mcu/all/bsp_register_protection.o
                               0x1aab (size before relaxing)
 .debug_str     0x00013e01      0x16f ./ra/fsp/src/bsp/mcu/all/bsp_rom_registers.o
                                0x312 (size before relaxing)
 .debug_str     0x00013f70       0x82 ./ra/fsp/src/bsp/cmsis/Device/RENESAS/Source/startup.o
                                0x246 (size before relaxing)
 .debug_str     0x00013ff2       0xc1 ./ra/fsp/src/bsp/cmsis/Device/RENESAS/Source/system.o
                                0x649 (size before relaxing)

.debug_frame    0x00000000     0x2518
 .debug_frame   0x00000000       0xb0 ./src/adc_temp.o
 .debug_frame   0x000000b0       0xac ./src/angle.o
 .debug_frame   0x0000015c      0x118 ./src/control_table.o
 .debug_frame   0x00000274       0x3c ./src/crc8.o
 .debug_frame   0x000002b0      0x104 ./src/hal_entry.o
 .debug_frame   0x000003b4       0x34 ./src/interpolation.o
 .debug_frame   0x000003e8       0x38 ./src/monitor.o
 .debug_frame   0x00000420      0x450 ./src/packet.o
 .debug_frame   0x00000870       0x80 ./src/pid.o
 .debug_frame   0x000008f0      0x108 ./src/power_monitor.o
 .debug_frame   0x000009f8       0x40 ./src/sintable.o
 .debug_frame   0x00000a38      0x1b0 ./src/usart.o
 .debug_frame   0x00000be8       0x20 ./ra_gen/common_data.o
 .debug_frame   0x00000c08       0x20 ./ra_gen/hal_data.o
 .debug_frame   0x00000c28       0x28 ./ra_gen/main.o
 .debug_frame   0x00000c50      0x1e8 ./ra/fsp/src/r_sci_uart/r_sci_uart.o
 .debug_frame   0x00000e38      0x168 ./ra/fsp/src/r_sci_spi/r_sci_spi.o
 .debug_frame   0x00000fa0      0x118 ./ra/fsp/src/r_sci_i2c/r_sci_i2c.o
 .debug_frame   0x000010b8      0x174 ./ra/fsp/src/r_rtc/r_rtc.o
 .debug_frame   0x0000122c      0x168 ./ra/fsp/src/r_ioport/r_ioport.o
 .debug_frame   0x00001394      0x230 ./ra/fsp/src/r_gpt/r_gpt.o
 .debug_frame   0x000015c4      0x254 ./ra/fsp/src/r_flash_hp/r_flash_hp.o
 .debug_frame   0x00001818       0xfc ./ra/fsp/src/r_dtc/r_dtc.o
 .debug_frame   0x00001914       0x90 ./ra/fsp/src/r_crc/r_crc.o
 .debug_frame   0x000019a4      0x198 ./ra/fsp/src/r_agt/r_agt.o
 .debug_frame   0x00001b3c      0x1bc ./ra/fsp/src/r_adc/r_adc.o
 .debug_frame   0x00001cf8       0xf4 ./ra/fsp/src/bsp/mcu/all/bsp_clocks.o
 .debug_frame   0x00001dec       0x40 ./ra/fsp/src/bsp/mcu/all/bsp_common.o
 .debug_frame   0x00001e2c       0x48 ./ra/fsp/src/bsp/mcu/all/bsp_delay.o
 .debug_frame   0x00001e74       0x3c ./ra/fsp/src/bsp/mcu/all/bsp_group_irq.o
 .debug_frame   0x00001eb0       0x30 ./ra/fsp/src/bsp/mcu/all/bsp_irq.o
 .debug_frame   0x00001ee0       0x48 ./ra/fsp/src/bsp/mcu/all/bsp_register_protection.o
 .debug_frame   0x00001f28       0x38 ./ra/fsp/src/bsp/cmsis/Device/RENESAS/Source/startup.o
 .debug_frame   0x00001f60       0x44 ./ra/fsp/src/bsp/cmsis/Device/RENESAS/Source/system.o
 .debug_frame   0x00001fa4       0xac c:/renesas/ra/e2studio_v2023-10_fsp_v5.0.0/toolchains/gcc_arm/12.2.mpacbti-rel1/bin/../lib/gcc/arm-none-eabi/12.2.1/thumb/v8-m.main+fp/hard\libgcc.a(_arm_addsubdf3.o)
 .debug_frame   0x00002050       0x50 c:/renesas/ra/e2studio_v2023-10_fsp_v5.0.0/toolchains/gcc_arm/12.2.mpacbti-rel1/bin/../lib/gcc/arm-none-eabi/12.2.1/thumb/v8-m.main+fp/hard\libgcc.a(_arm_muldivdf3.o)
 .debug_frame   0x000020a0       0xc4 c:/renesas/ra/e2studio_v2023-10_fsp_v5.0.0/toolchains/gcc_arm/12.2.mpacbti-rel1/bin/../lib/gcc/arm-none-eabi/12.2.1/thumb/v8-m.main+fp/hard\libgcc.a(_arm_cmpdf2.o)
 .debug_frame   0x00002164       0x24 c:/renesas/ra/e2studio_v2023-10_fsp_v5.0.0/toolchains/gcc_arm/12.2.mpacbti-rel1/bin/../lib/gcc/arm-none-eabi/12.2.1/thumb/v8-m.main+fp/hard\libgcc.a(_arm_fixdfsi.o)
 .debug_frame   0x00002188       0x24 c:/renesas/ra/e2studio_v2023-10_fsp_v5.0.0/toolchains/gcc_arm/12.2.mpacbti-rel1/bin/../lib/gcc/arm-none-eabi/12.2.1/thumb/v8-m.main+fp/hard\libgcc.a(_arm_fixunsdfsi.o)
 .debug_frame   0x000021ac       0x44 c:/renesas/ra/e2studio_v2023-10_fsp_v5.0.0/toolchains/gcc_arm/12.2.mpacbti-rel1/bin/../lib/gcc/arm-none-eabi/12.2.1/thumb/v8-m.main+fp/hard\libgcc.a(_aeabi_ldivmod.o)
 .debug_frame   0x000021f0       0x38 c:/renesas/ra/e2studio_v2023-10_fsp_v5.0.0/toolchains/gcc_arm/12.2.mpacbti-rel1/bin/../lib/gcc/arm-none-eabi/12.2.1/thumb/v8-m.main+fp/hard\libgcc.a(_udivmoddi4.o)
 .debug_frame   0x00002228       0x38 c:/renesas/ra/e2studio_v2023-10_fsp_v5.0.0/toolchains/gcc_arm/12.2.mpacbti-rel1/bin/../lib/gcc/arm-none-eabi/12.2.1/thumb/v8-m.main+fp/hard\libg_nano.a(libc_a-itoa.o)
 .debug_frame   0x00002260       0x64 c:/renesas/ra/e2studio_v2023-10_fsp_v5.0.0/toolchains/gcc_arm/12.2.mpacbti-rel1/bin/../lib/gcc/arm-none-eabi/12.2.1/thumb/v8-m.main+fp/hard\libg_nano.a(libc_a-strtol.o)
 .debug_frame   0x000022c4       0x48 c:/renesas/ra/e2studio_v2023-10_fsp_v5.0.0/toolchains/gcc_arm/12.2.mpacbti-rel1/bin/../lib/gcc/arm-none-eabi/12.2.1/thumb/v8-m.main+fp/hard\libg_nano.a(libc_a-utoa.o)
 .debug_frame   0x0000230c      0x144 c:/renesas/ra/e2studio_v2023-10_fsp_v5.0.0/toolchains/gcc_arm/12.2.mpacbti-rel1/bin/../lib/gcc/arm-none-eabi/12.2.1/thumb/v8-m.main+fp/hard\libg_nano.a(libc_a-findfp.o)
 .debug_frame   0x00002450       0x20 c:/renesas/ra/e2studio_v2023-10_fsp_v5.0.0/toolchains/gcc_arm/12.2.mpacbti-rel1/bin/../lib/gcc/arm-none-eabi/12.2.1/thumb/v8-m.main+fp/hard\libg_nano.a(libc_a-memset.o)
 .debug_frame   0x00002470       0x20 c:/renesas/ra/e2studio_v2023-10_fsp_v5.0.0/toolchains/gcc_arm/12.2.mpacbti-rel1/bin/../lib/gcc/arm-none-eabi/12.2.1/thumb/v8-m.main+fp/hard\libg_nano.a(libc_a-errno.o)
 .debug_frame   0x00002490       0x20 c:/renesas/ra/e2studio_v2023-10_fsp_v5.0.0/toolchains/gcc_arm/12.2.mpacbti-rel1/bin/../lib/gcc/arm-none-eabi/12.2.1/thumb/v8-m.main+fp/hard\libg_nano.a(libc_a-strcpy.o)
 .debug_frame   0x000024b0       0x20 c:/renesas/ra/e2studio_v2023-10_fsp_v5.0.0/toolchains/gcc_arm/12.2.mpacbti-rel1/bin/../lib/gcc/arm-none-eabi/12.2.1/thumb/v8-m.main+fp/hard\libg_nano.a(libc_a-aeabi_memcpy.o)
 .debug_frame   0x000024d0       0x20 c:/renesas/ra/e2studio_v2023-10_fsp_v5.0.0/toolchains/gcc_arm/12.2.mpacbti-rel1/bin/../lib/gcc/arm-none-eabi/12.2.1/thumb/v8-m.main+fp/hard\libg_nano.a(libc_a-aeabi_memclr.o)
 .debug_frame   0x000024f0       0x28 c:/renesas/ra/e2studio_v2023-10_fsp_v5.0.0/toolchains/gcc_arm/12.2.mpacbti-rel1/bin/../lib/gcc/arm-none-eabi/12.2.1/thumb/v8-m.main+fp/hard\libg_nano.a(libc_a-memcpy-stub.o)

.debug_loclists
                0x00000000     0xf300
 .debug_loclists
                0x00000000      0x2a5 ./src/angle.o
 .debug_loclists
                0x000002a5      0x32d ./src/control_table.o
 .debug_loclists
                0x000005d2       0xe8 ./src/crc8.o
 .debug_loclists
                0x000006ba      0x642 ./src/hal_entry.o
 .debug_loclists
                0x00000cfc       0xcf ./src/interpolation.o
 .debug_loclists
                0x00000dcb       0x9b ./src/monitor.o
 .debug_loclists
                0x00000e66     0x2dc5 ./src/packet.o
 .debug_loclists
                0x00003c2b      0x2a7 ./src/pid.o
 .debug_loclists
                0x00003ed2       0xf2 ./src/sintable.o
 .debug_loclists
                0x00003fc4     0x183a ./src/usart.o
 .debug_loclists
                0x000057fe     0x1412 ./ra/fsp/src/r_sci_uart/r_sci_uart.o
 .debug_loclists
                0x00006c10     0x13df ./ra/fsp/src/r_sci_spi/r_sci_spi.o
 .debug_loclists
                0x00007fef      0x9bf ./ra/fsp/src/r_sci_i2c/r_sci_i2c.o
 .debug_loclists
                0x000089ae      0xb5a ./ra/fsp/src/r_rtc/r_rtc.o
 .debug_loclists
                0x00009508      0x724 ./ra/fsp/src/r_ioport/r_ioport.o
 .debug_loclists
                0x00009c2c     0x155f ./ra/fsp/src/r_gpt/r_gpt.o
 .debug_loclists
                0x0000b18b     0x166e ./ra/fsp/src/r_flash_hp/r_flash_hp.o
 .debug_loclists
                0x0000c7f9      0x360 ./ra/fsp/src/r_dtc/r_dtc.o
 .debug_loclists
                0x0000cb59      0x447 ./ra/fsp/src/r_crc/r_crc.o
 .debug_loclists
                0x0000cfa0      0xe56 ./ra/fsp/src/r_agt/r_agt.o
 .debug_loclists
                0x0000ddf6      0xf8c ./ra/fsp/src/r_adc/r_adc.o
 .debug_loclists
                0x0000ed82      0x1e1 ./ra/fsp/src/bsp/mcu/all/bsp_clocks.o
 .debug_loclists
                0x0000ef63       0x20 ./ra/fsp/src/bsp/mcu/all/bsp_common.o
 .debug_loclists
                0x0000ef83      0x110 ./ra/fsp/src/bsp/mcu/all/bsp_delay.o
 .debug_loclists
                0x0000f093       0x6d ./ra/fsp/src/bsp/mcu/all/bsp_group_irq.o
 .debug_loclists
                0x0000f100       0xad ./ra/fsp/src/bsp/mcu/all/bsp_irq.o
 .debug_loclists
                0x0000f1ad       0xa1 ./ra/fsp/src/bsp/mcu/all/bsp_register_protection.o
 .debug_loclists
                0x0000f24e       0xb2 ./ra/fsp/src/bsp/cmsis/Device/RENESAS/Source/system.o

.debug_line_str
                0x00000000      0x20b
 .debug_line_str
                0x00000000       0xe2 c:/renesas/ra/e2studio_v2023-10_fsp_v5.0.0/toolchains/gcc_arm/12.2.mpacbti-rel1/bin/../lib/gcc/arm-none-eabi/12.2.1/thumb/v8-m.main+fp/hard\libgcc.a(_arm_addsubdf3.o)
 .debug_line_str
                0x000000e2       0xe2 c:/renesas/ra/e2studio_v2023-10_fsp_v5.0.0/toolchains/gcc_arm/12.2.mpacbti-rel1/bin/../lib/gcc/arm-none-eabi/12.2.1/thumb/v8-m.main+fp/hard\libgcc.a(_arm_muldivdf3.o)
 .debug_line_str
                0x000000e2       0xe2 c:/renesas/ra/e2studio_v2023-10_fsp_v5.0.0/toolchains/gcc_arm/12.2.mpacbti-rel1/bin/../lib/gcc/arm-none-eabi/12.2.1/thumb/v8-m.main+fp/hard\libgcc.a(_arm_cmpdf2.o)
 .debug_line_str
                0x000000e2       0xe2 c:/renesas/ra/e2studio_v2023-10_fsp_v5.0.0/toolchains/gcc_arm/12.2.mpacbti-rel1/bin/../lib/gcc/arm-none-eabi/12.2.1/thumb/v8-m.main+fp/hard\libgcc.a(_arm_fixdfsi.o)
 .debug_line_str
                0x000000e2       0xe2 c:/renesas/ra/e2studio_v2023-10_fsp_v5.0.0/toolchains/gcc_arm/12.2.mpacbti-rel1/bin/../lib/gcc/arm-none-eabi/12.2.1/thumb/v8-m.main+fp/hard\libgcc.a(_arm_fixunsdfsi.o)
 .debug_line_str
                0x000000e2        0x8 c:/renesas/ra/e2studio_v2023-10_fsp_v5.0.0/toolchains/gcc_arm/12.2.mpacbti-rel1/bin/../lib/gcc/arm-none-eabi/12.2.1/thumb/v8-m.main+fp/hard\libgcc.a(_aeabi_ldivmod.o)
                                 0xdd (size before relaxing)
 .debug_line_str
                0x000000ea        0xc c:/renesas/ra/e2studio_v2023-10_fsp_v5.0.0/toolchains/gcc_arm/12.2.mpacbti-rel1/bin/../lib/gcc/arm-none-eabi/12.2.1/thumb/v8-m.main+fp/hard\libgcc.a(_dvmd_tls.o)
                                 0xe1 (size before relaxing)
 .debug_line_str
                0x000000f6       0xff c:/renesas/ra/e2studio_v2023-10_fsp_v5.0.0/toolchains/gcc_arm/12.2.mpacbti-rel1/bin/../lib/gcc/arm-none-eabi/12.2.1/thumb/v8-m.main+fp/hard\libg_nano.a(libc_a-strlen.o)
 .debug_line_str
                0x000001f5       0x16 c:/renesas/ra/e2studio_v2023-10_fsp_v5.0.0/toolchains/gcc_arm/12.2.mpacbti-rel1/bin/../lib/gcc/arm-none-eabi/12.2.1/thumb/v8-m.main+fp/hard\libg_nano.a(libc_a-aeabi_memset-soft.o)
                                0x102 (size before relaxing)
